:100000000C94D72A0D94100B0D94E50A0D94BA0A9E
:100010000D948F0A0D94640A0D94390A0D940E0AFA
:100020000C940FD10C94082B0C94082B0C94082BD7
:100030000C94082B0C9432DD0C94082B0C94082B98
:100040000C94082B0C948EC90C94082B0C94082B40
:100050000C94082B0C94082B0C9404C80D943B0BA7
:100060000C94082B0C9455D00C94082B0C94082B52
:100070000C94082B0C94082B0C94082B0C94082B34
:100080000C94082B0C94082B0C94082B0C94082B24
:100090000C94082B0C94082B0C94082B0C94082B14
:1000A0000C94082B0C94082B0C94082B0C94082B04
:1000B0000C94082B0C94082B0C94082B0C94082BF4
:1000C0000C94082B0C94082B0C94082B0C94082BE4
:1000D0000C94082B0C94082B0C94082B0C94082BD4
:1000E0000C94082BBB46BE46AD46B146B746F54616
:1000F000C246C646CC46D046D446DA46DE46E2463E
:10010000F546E846EC46F046447744774B774B7724
:100110004B775277527752775F775977597759777C
:1001200089D08FD0A0D0ABD0B3D0C8D0B7D0C8D0F2
:10013000BBD0BFD0C8D0C5D099D19ED1A3D1ADD1AD
:10014000B7D130D2C1D1C9D1D1D1DBD1E5D1EFD135
:10015000FED108D230D212D21CD226D2084AD73BC6
:100160003BCE016E84BCBFFDC12F3D6C74319ABD86
:1001700056833DDA3D00C77F11BED9E4BB4C3E91AA
:100180006BAAAABE000000803F05A84CCDB2D44E99
:10019000B93836A9020C50B9918688083CA6AAAA9B
:1001A0002ABE000000803F000D946D080D948F1151
:1001B0000D944A100D94780620746F6F206C6F6E4A
:1001C0006720657874727573696F6E2070726576DA
:1001D000656E7465640A0020636F6C6420657874D2
:1001E000727573696F6E2070726576656E74656482
:1001F0000A0047322F4733206261642070617261C8
:100200006D65746572730A00205A3A200020593ACD
:10021000200042656420583A20004C756C7A426F89
:1002200074204D696E69204C434420726561647985
:100230002E00526573756D696E67207072696E74F9
:1002400000436C69636B20746F20726573756D6514
:100250002E2E2E00456E642066696C65206C6973D5
:10026000740A00426567696E2066696C65206C6976
:1002700073740A004D3132350046696C652064653F
:100280006C657465643A0044656C6574696F6E20D2
:100290006661696C65642C2046696C653A20006F64
:1002A00070656E206661696C65642C2046696C65BA
:1002B0003A20002569730025696D202569730025A2
:1002C00069682025696D20256973002569642025EA
:1002D00069682025696D20256973002569792025C5
:1002E0006964202569682025696D2025697300509F
:1002F00072696E742074696D653A20004578747275
:1003000075646572202573004C756C7A426F742099
:100310004D696E69204C43442072656164792E00FA
:100320006F6B00436F6F6C696E6720646F6E652E34
:100330000048656174696E6720646F6E652E0020E9
:10034000573A004578747275646572202573004CC5
:10035000756C7A426F74204D696E69204C4344205D
:1003600072656164792E0042656420646F6E652E4B
:100370000020573A004265642068656174696E67C1
:100380002E0042656420636F6F6C696E672E007A81
:100390005F6D61783A20007A5F6D696E3A2000796E
:1003A0005F6D61783A2000795F6D696E3A20007860
:1003B0005F6D61783A2000785F6D696E3A20005277
:1003C00065706F7274696E6720656E6473746F70A8
:1003D000207374617475730A0020643A0020693ACE
:1003E0000020703A0020643A0020693A0020703AF8
:1003F0000043290A0061626C656420286D696E20E3
:1004000074656D702000436F6C642065787472753C
:100410006465732061726520004B6420002364656D
:1004200066696E65202044454641554C545F004B3B
:1004300069200023646566696E6520204445464155
:10044000554C545F004B70200023646566696E65EF
:10045000202044454641554C545F005049442041BA
:1004600075746F74756E652066696E69736865640E
:10047000212050757420746865206C617374204B62
:10048000702C204B6920616E64204B6420636F6E7A
:100490007374616E74732066726F6D2062656C6F29
:1004A0007720696E746F20436F6E6669677572613D
:1004B00074696F6E2E680A00504944204175746F4C
:1004C00074756E65206661696C6564212074696D60
:1004D000656F75740A00504944204175746F7475D6
:1004E0006E65206661696C6564212054656D706578
:1004F00072617475726520746F6F20686967680A2D
:1005000000204B643A2000204B693A2000204B70B9
:100510003A20000A20436C61737369632050494498
:10052000200A002054753A2000204B753A20002004
:100530006D61783A2000206D696E3A200020643A9F
:10054000200020626961733A2000426564204C6596
:1005500076656C696E6720004661696C656420741D
:100560006F20656E61626C6520426564204C657623
:10057000656C696E670A00426564204C6576656C3F
:1005800020436F7272656374696F6E204D6174727F
:1005900069783A003A20007A5F6D696E3A20202D22
:1005A00032207A5F6D61783A202035005A204F66FC
:1005B0006673657420004E6F2063617365206C69FB
:1005C0006768740A004163746976652045787472BF
:1005D000756465723A2000556E6B6E6F776E20639E
:1005E0006F6D6D616E643A202200434F4D4D554E44
:1005F00049434154494F4E0044525952554E0045CB
:1006000052524F525300494E464F004543484F0007
:10061000000020002300260029002C002F003200BB
:1006200000010000030106010901000000000000B4
:10063000C0C0000000C00000254300003F43000090
:100640001F432F2F20004361703A454D45524745C7
:100650004E43595F5041525345523A310A0043616B
:10066000703A434153455F4C494748545F425249B1
:100670004748544E4553533A300A004361703A5448
:100680004F47474C455F4C49474854533A300A005E
:100690004361703A534F4654574152455F504F574C
:1006A00045523A300A004361703A4C4556454C4930
:1006B0004E475F444154413A310A004361703A5A0F
:1006C0005F50524F42453A310A004361703A4155FA
:1006D000544F4C4556454C3A310A004361703A50EC
:1006E00052494E545F4A4F423A310A004361703AD0
:1006F00050524F47524553533A300A004361703AC3
:100700004155544F5245504F52545F54454D503A05
:10071000310A004361703A454550524F4D3A310A13
:10072000004649524D574152455F4E414D453A4D65
:1007300061726C696E20204649524D574152455FA7
:1007400056455253494F4E3A312E312E352E3434C0
:100750002045585452554445525F545950453A53D8
:10076000696E676C65457874727564657220534F65
:10077000555243455F434F44455F55524C3A687468
:100780007470733A2F2F636F64652E616C657068A7
:100790006F626A656374732E636F6D2F646966663A
:1007A0007573696F6E2F4D41524C494E2050524F18
:1007B000544F434F4C5F56455253494F4E3A312E9A
:1007C00030204D414348494E455F545950453A4CBD
:1007D000756C7A426F74204D696E69204C434420D9
:1007E00045585452554445525F434F554E543A3143
:1007F00020555549443A30383366363866312D3005
:100800003238652D343934632D393865312D6632EF
:10081000653064666165653961350A004D3134358E
:1008200020533C696E6465783E206F7574206F6656
:100830002072616E67652028302D31290A000B0671
:100840000606FF05F805EA056F6666004445425551
:10085000473A0020706F736974696F6E206F75740A
:10086000206F662072616E67652E0A003F50726FBE
:100870006265200020204E6F7A7A6C653A20002055
:100880000066696C616D656E7420756E6C6F616475
:10089000005761697420666F72005052494E5420AF
:1008A0005041555345440020204E6F7A7A6C653A8A
:1008B00020006368616E6765006F6620746865205C
:1008C00066696C616D656E74005761697420666F4E
:1008D00072207374617274005052494E542050411A
:1008E000555345440020204E6F7A7A6C653A2000BB
:1008F00020004261636B004D696E696D756D205417
:10090000656D70206973203132302E004865617446
:10091000696E67206661696C65640025753A2530EB
:10092000327500253032753A2530327500257564F0
:1009300020253032753A253032750000060900FE58
:10094000000000000001090008FE0000050808067C
:10095000000040F0C8888898781005080806000054
:10096000C0F88888888888F80505050600012030C9
:10097000F830200508080600002070F8202020200C
:10098000E00509090600FF2070A8A8B88888702033
:100990000509090600FFE080C0B0A8283028280516
:1009A00009090600FFF8A88888888888A8F8050A39
:1009B0000A0600FE205050505088A8A888700303F3
:1009C0000306000340A04000060900FE0701920351
:1009D0002120FFFF08FF07FF0000000600000107BD
:1009E00007060200808080808000800302020601EA
:1009F00005A0A00507070600005050F850F8505019
:100A00000507070600002078A07028F020050707DA
:100A1000060000C0C810204098180507070600000F
:100A20006090A040A89068020303060104C04080C3
:100A3000030707060100204080808040200307074D
:100A400006010080402020204080050505060001A9
:100A500020A870A8200505050600012020F8202008
:100A60000203030602FFC04080050101060003F8EF
:100A7000020202060200C0C00505050600010810BA
:100A800020408005070706000070888888888870E5
:100A900003070706010040C040404040E00507074B
:100AA000060000708808708080F8050707060000BF
:100AB000F81020100808F005070706000010305055
:100AC00090F81010050707060000F880F008088865
:100AD00070050707060000708080F08888700507A1
:100AE00007060000F8081020202020050707060050
:100AF0000070888870888870050707060000708875
:100B00008878080870020505060200C0C000C0C051
:100B10000206060602FFC0C000C0408004070706A8
:100B2000000010204080402010050303060002F85A
:100B300000F80407070601008040201020408005CF
:100B40000707060000708808102000200507070628
:100B5000000070880868A8A87005070706000070E4
:100B60008888F8888888050707060000F08888F0DC
:100B70008888F005070706000070888080808870EC
:100B8000050707060000F08888888888F0050707B1
:100B9000060000F88080F08080F805070706000056
:100BA000F88080F08080800507070600007088804C
:100BB000B8888870050707060000888888F8888844
:100BC00088010707060200808080808080800507FA
:100BD0000706000038101010109060050707060087
:100BE000008890A0C0A090880507070600008080BC
:100BF00080808080F805070706000088D8A88888CC
:100C000088880507070600008888C8A8988888058E
:100C1000070706000070888888888870050707061F
:100C20000000F08888F080808005070706000070CB
:100C3000888888A89068050707060000F08888F073
:100C4000A09088050707060000788080700808F0EB
:100C5000050707060000F8202020202020050707B0
:100C600006000088888888888870050707060000C5
:100C700088888888885020050707060000888888AB
:100C80008888A850050707060000888850205088EB
:100C9000880507070600008888885020202005075F
:100CA00007060000F80810204080F8030707060137
:100CB00000E08080808080E005050506000180401E
:100CC000201008030707060100E02020202020E074
:100CD000050303060004205088050101060000F802
:100CE00002020206020580400505050600007008A4
:100CF0007888780507070600008080B0C88888F0EB
:100D0000050505060000708080887005070706004D
:100D1000000808689888887805050506000070882E
:100D2000F880700507070600003048E0404040406A
:100D30000506060600FF7088887808700507070614
:100D400000008080B0C888888801070706020080FC
:100D50000080808080800308080601FF200020209A
:100D60002020A040040707060000808090A0C0A0BB
:100D700090030707060100C04040404040E00505E1
:100D800005060000D0A8A8A8A8050505060000B023
:100D9000C888888805050506000070888888700561
:100DA00006060600FFF08888F0808005060606002B
:100DB000FF788888780808050505060000B0C88017
:100DC000808005050506000070807008F0040707A4
:100DD0000600004040E040404030050505060000A8
:100DE000888888986805050506000088888850204E
:100DF0000505050600008888A8A850050505060019
:100E00000088502050880506060600FF88888878EC
:100E10000870050505060000F8102040F8030707D4
:100E200006010020404080404020010707060200E4
:100E3000808080808080800307070601008040401A
:100E40002040408005020206000268900000000673
:100E50000000000000060000000000060000000086
:100E60000006000000000006000000000006000070
:100E70000000000600000000000600000000000660
:100E80000000000000060000000000060000000056
:100E90000006000000000006000000000006000040
:100EA0000000000600000000000600000000000630
:100EB0000000000000060000000000060000000026
:100EC0000006000000000006000000000006000010
:100ED0000000000600000000000600000000000600
:100EE00000000000000600000000000600000000F6
:100EF00000060000000000060000000000060000E0
:100F000000000006000000000006000000000006CF
:100F10000000000000060000010707060200800034
:100F200080808080800507070600002070A8A0A8A8
:100F30007020050707060000304040E04050A8053B
:100F40000505060000887050708805070706000038
:100F5000885020F820F820010707060200808080D2
:100F6000008080800508080600003048205050208E
:100F70009060030101060107A0050707060000F8BD
:100F800088B8B8B888F8050707060001700878889F
:100F90007800F80505050600012850A05028050333
:100FA00003060001F8080802020206020640800556
:100FB0000707060000F888A88898A8F80501010628
:100FC0000006F8040404060003609090600507071B
:100FD0000600002020F8202000F804050506000384
:100FE00060902040F0030505060003E020E020E0CB
:100FF00002020206020640800508080600FF8888F3
:10100000888898E880800507070600007898987817
:10101000181818020202060202C0C00202020602EA
:10102000FF408003050506000340C04040E005077F
:1010300007060001708888887000F805050506001D
:1010400001A0502850A00507070600008890A85866
:10105000B808080507070600008890B848982038A7
:10106000050808060000C040C048D8380808050731
:101070000706000020002040808870050808060050
:10108000004020007088F8888805080806000010D5
:1010900020007088F88888050808060000205000A5
:1010A0007088F88888050808060000689000708835
:1010B000F888880508080600005000708888F888BD
:1010C000880508080600002050207088F8888805E8
:1010D00007070600003860A0B8E0A0B805080806B9
:1010E00000FF708880808870206005080806000076
:1010F000402000F880F080F805080806000008107D
:1011000000F880F080F8050808060000205000F87C
:1011100080F080F80507070600005000F880F08096
:10112000F8030808060100804000E0404040E0036A
:101130000808060100204000E0404040E0030808A5
:1011400006010040A000E0404040E0030707060120
:1011500000A000E0404040E005070706000070489E
:1011600048E848487005080806000068900088C8EC
:10117000A89888050808060000402070888888889C
:10118000700508080600001020708888888870059F
:10119000080806000020500070888888700508083C
:1011A00006000068900070888888700508080600AE
:1011B0000050007088888888700505050600018841
:1011C000502050880508080600FF1070A8A8A8A89D
:1011D00070400508080600004020888888888870CC
:1011E000050808060000102088888888887005088F
:1011F00008060000205000888888887005080806C6
:10120000000050008888888888700508080600005B
:1012100010208850202020200509090600FFC0402A
:10122000704848704040E00408080601FF60909054
:10123000A09090E08005080806000040200070089B
:101240007888780508080600001020007008788863
:101250007805080806000020500070087888780596
:10126000080806000068900070087888780507076D
:10127000060000500070087888780508080600000D
:101280002050207008788878050606060000D028CF
:1012900078A0A8500506060600FF708088702060C0
:1012A0000508080600004020007088F880700508D6
:1012B000080600001020007088F8807005080806F5
:1012C00000002050007088F88070050707060000B5
:1012D00050007088F8807003080806010080400004
:1012E00040C04040E003080806010020400040C024
:1012F0004040E003080806010040A00040C0404014
:10130000E0030707060100A00040C04040E00507D9
:1013100007060000A040A0107888700508080600A5
:1013200000689000B0C8888888050808060000405A
:1013300020007088888870050808060000102000CA
:1013400070888888700508080600002050007088A2
:1013500088887005080806000068900070888888F2
:101360007005070706000050007088888870050522
:10137000050600012000F800200507070600FF1001
:1013800070A8A8A870400508080600004020008842
:10139000888898680508080600001020008888885A
:1013A000986805080806000020500088888898681A
:1013B0000507070600005000888888986805090915
:1013C0000600FF102000888888F8087004070706C8
:1013D00001FFC04060506040E00508080600FF5073
:1013E000008888887808705A005900580009200041
:1013F0000000000000000000000000007FFFE0008F
:1014000000000000000000000000007000E000008C
:101410000000000000000000000061F86000000013
:1014200000000000000000000041F8200000000063
:10143000000000000000000040F02000000000005C
:1014400000000000000000406020000000000000DC
:101450000000000000005801A07F80000000000094
:1014600000004104005C63A0FFC000000000000019
:10147000002082005EF7A0FFC00000000000000016
:101480002082005EF7A0FFC00000000000000041C5
:1014900004005C63A07F8000000000000000820860
:1014A000005801A07F80000000000000010410002F
:1014B000406020FFC0000000000000010410004058
:1014C000F020FFC00000000000000082080041F88A
:1014D00020FFC00000000000000041040061F8602F
:1014E0003F00000000000000000000007000E01E4F
:1014F0000000000000000001FFFF807FFFE00C0003
:1015000000000000000001FFFF800000000000005C
:101510000000000000000000007FFFE0000000006D
:1015200000000000000000007000E000000000006B
:1015300000000000000000630C60000000000000DC
:10154000000000000000470E200000000000000026
:1015500000000000004F0F2000000000000000000D
:10156000000000005F0FA00000000000000000006D
:101570000000005E07A07F80000000000000004126
:101580000400406020FFC000000000000000208236
:101590000040F020FFC0000000000000002082009A
:1015A00040F020FFC00000000000000041040040A7
:1015B00060207F80000000000000008208005E07BD
:1015C000A07F80000000000000010410005F0FA059
:1015D000FFC0000000000000010410004F0F20FFBA
:1015E000C000000000000000820800470E20FFC07D
:1015F00000000000000000410400630C603F000098
:101600000000000000000000007000E01E0000006C
:101610000000000001FFFF807FFFE00C00000000E1
:1016200000000001FFFF800000007C3C3E5E2B3D7F
:101630003F2F5B5D3B2C2A225C0043616E6E6F7412
:10164000206F70656E2073756264697220000105F9
:101650000800FF060121023520FFFF07FF06FF09F2
:101660000050221656808080800080153353A0A041
:10167000A00257575050F850F8505002575720705A
:10168000A07028702013355580A040A02002475735
:1016900040A0A040A0A05025135380808012265661
:1016A000408080808040122656804040404080022A
:1016B00045559060F060900255552020F82020118B
:1016C0003353604080044151F011335340E04002F5
:1016D000465610102040808012365640A0A0A0A090
:1016E0004012365640C0404040E0024656609010DE
:1016F0006080F0024656F02060109060024656204E
:1017000060A0F02020024656F080E0109060024673
:10171000566080E0909060024656F01020204040D5
:1017200002465660906090906002465660909070BD
:101730001060122555C0C000C0C011365660600050
:10174000604080123656204080804020034353F092
:1017500000F012365680402020408012365640A0BD
:1017600020400040015858304898A8A890403002C6
:101770004656609090F09090024656E090E090902F
:10178000E0024656609080809060024656E090905D
:101790009090E0024656F080E08080F0024656F0DD
:1017A00080E0808080024656609080B09060024663
:1017B000569090F0909090123656E040404040E0B5
:1017C00002465670202020A04002465690A0C0A09D
:1017D000A0900246568080808080F002465690F0AD
:1017E000F090909002465690D0F0B0B090024656DD
:1017F000609090909060024656E09090E08080016A
:101800004757609090D0B06010024656E09090E04C
:101810009090024656609040209060123656E0400C
:10182000404040400246569090909090600246564C
:10183000909090906060024656909090F0F09002E8
:1018400046569090606090900256568888502020AE
:1018500020024656F010204080F0123656E080807C
:101860008080E0024656808040201010123656E0FC
:1018700020202020E016325240A0014151F01622D3
:10188000528040024454709090700246568080E02E
:101890009090E012345460808060024656101070C0
:1018A00090907002445460B0C06002465620504090
:1018B000E0404001455560907010600246568080BF
:1018C000E09090901236564000C04040E0113757EB
:1018D0002000202020A040024656808090E090907A
:1018E000123656C040404040E0025454D0A8A8A848
:1018F000024454E0909090024454609090600145FE
:1019000055E090E0808001455570907010100244C1
:1019100054A0D0808012345460C020C0024656408B
:1019200040E040502002445490909070123454A0F3
:10193000A0A04002545488A8A8500244549060606B
:10194000900145559090709060024454F02040F012
:10195000024757304020C0204030221656808080F9
:10196000808080024757C02040304020C00642524D
:1019700050A0FFFFFFFFFFFFFFFFFFFFFFFFFFFF85
:10198000FFFFFFFFFFFFFFFFFFFFFFFFFFFFFFFF67
:10199000FFFFFF09005022165680008080808001E2
:1019A00046562070A0A070200246562050E04050BD
:1019B000A002555588705070880256568850F820FD
:1019C000F82022175780808000808080024757705F
:1019D00080E0907010E0173151A002565670A8C8F0
:1019E000C8A87014355560A06000E003435350A0B0
:1019F00050123353E02020143151E002565670E863
:101A0000D8E8D870173151E015335340A040123553
:101A10005540E04000E014355540A02040E014352A
:101A200055C020C020C016225240800145559090DC
:101A300090E08002565678E8E86828282411518002
:101A4000112252408014355540C04040E0143555B5
:101A500040A04000E0034353A050A00247578080BD
:101A600080A060F0200247578080A0D01020700234
:101A7000475780408060A0F02012365640004080DA
:101A8000A04002475740206090F0909002475720B6
:101A9000406090F0909002475760906090F0909076
:101AA00002475750A06090F0909002475790006016
:101AB00090F0909002475760906090F090900246AE
:101AC0005670A0A0F0A0B001475760908080906051
:101AD000400247574020F080E080F0024757204006
:101AE000F080E080F00247576090F080E080F002E4
:101AF00047579000F080E080F01237578040E04078
:101B00004040E01237572040E0404040E012375755
:101B100040A0E0404040E0123757A000E040404085
:101B2000E00256567048E848487002475750A09067
:101B3000D0B090900247574020609090906002474C
:101B4000572040609090906002475760906090905E
:101B5000906002475750A060909090600247579065
:101B6000006090909060123353A040A002465670DF
:101B7000B0B0D0D0E00247574020909090906002E3
:101B80004757204090909090600247576090909007
:101B90009090600247579000909090906002575745
:101BA0001020885020202002465680E09090E0804F
:101BB0000246566090A0A090A002475740200070B7
:101BC00090907002475720400070909070024757E5
:101BD0002050007090907002475750A00070909075
:101BE00070024656500070909070024757609060A7
:101BF00070909070025454F068B078113555608040
:101C000080604002475740200060B0C060024757E4
:101C100020400060B0C06002475760900060B0C0D4
:101C200060024656500060B0C060123757804000D6
:101C3000C04040E0123757204000C04040E012371B
:101C40005740A000C04040E0123656A000C04040BF
:101C5000E0024757A040A01070906002475750A084
:101C600000E0909090024757402000609090600202
:101C70004757204000609090600247576090006096
:101C800090906002475750A00060909060024656C6
:101C90009000609090601235554000E00040024492
:101CA0005470B0D0E00247574020009090907002EE
:101CB00047572040009090907002475760900090E6
:101CC0009090700246569000909090700148582075
:101CD000400090907090600147578080E090E080D5
:101CE000800147579000909070906001050700FEBA
:101CF0000500FB01F220FFFE05FE05FE020040028A
:101D000015258080800080053242A0A002556550D4
:101D1000F850F8500146562070C030E0200255655A
:101D20009010204048025565608068906805122236
:101D300080800225354080808040022535804040EB
:101D40004080043343A040A003334340E0400122DD
:101D5000324080043141E0021121800255650810B3
:101D60002040800245556090909060022535C0402B
:101D7000404040024555E0106080F0024555E010BB
:101D80006010E00245552060A0F020024555F0802B
:101D9000E010E00245556080E09060024555F0108B
:101DA000204040024555609060906002455560902B
:101DB0007010600313238000800214248000808050
:101DC0000235452040804020033343E000E00235E7
:101DD000458040204080024555E01060004002559B
:101DE000657088B8A870024555609090F0900245E3
:101DF00055E090E090E002354560808080600245CB
:101E000055E0909090E0023545E080E080E00235BA
:101E100045E080E080800245557080B090700245BA
:101E2000559090F09090023545E0404040E00245EA
:101E300055301010906002455590A0C0A09002351A
:101E40004580808080E002556588D8A88888024552
:101E50005590D0B0909002455560909090600245AA
:101E600055E09090E080014656609090906010029E
:101E70004555E09090E09002455570806010E0027A
:101E80003545E040404040024555909090906002BA
:101E900045559090A0A04002556588A8A8A850027A
:101EA000455590906090900245559090701060025A
:101EB0003545E0204080E0022535C0808080C002AA
:101EC00055658040201008022535C0404040C005BF
:101ED000324240A0024151F0052232804002445477
:101EE0007090907002455580E09090E0023444601C
:101EF000808060024555107090907002445460B02C
:101F0000C0600235452040E0404000465670909049
:101F100070106002455580E0909090021525800079
:101F20008080800027374000404040408002455577
:101F30008090A0E09002152580808080800254640B
:101F4000F0A8A8A8024454E09090900244546090F5
:101F50009060004656E09090E08080004656709079
:101F600090701010023444A0C0808002445470C0AD
:101F700030E002354540E0404020024454909090CB
:101F8000700244549090A040025464A8A85050029B
:101F90003444A04040A000465690909070106002DB
:101FA0004454F02040F00235456040804060021506
:101FB000258080808080023545C0402040C0054299
:101FC0005250A0FFFFFFFFFFFFFFFFFFFFFFFFFFDC
:101FD000FFFFFFFFFFFFFFFFFFFFFFFFFFFFFFFF11
:101FE000FFFFFFFF020040FFFFFFFFFFFFFFFFFFBC
:101FF000FFFFFFFFFFFFFFFFFFFFFFFFFFFFFFFFF1
:10200000FFFFFFFFFFFFFFFFFFFFFFFFFFFFFFFFE0
:10201000FFFFFFFFFFFFFFFFFFFFFFFFFFFFFFFFD0
:10202000FFFFFFFFFFFFFFFFFFFFFFFFFFFFFFFFC0
:10203000FFFFFFFFFFFFFFFFFFFFFFFFFFFFFFFFB0
:10204000FFFFFFFFFFFF01060D00FE09016602D63C
:1020500020FFFE0BFE0AFE0D0060221969808080C1
:10206000808080800080183363A0A0A00357675051
:1020700050F850F850500259692078A0A0702828D4
:10208000F02002596948A85010204050A8900258EA
:102090006840A0A040A098906828136380808011B9
:1020A0003B6B2040408080808080404020113B6B13
:1020B000804040202020202040408006556520A8F8
:1020C00070A8200455652020F8202011336360405B
:1020D00080065161F811336340E0400259690808F5
:1020E00010102040408080025969205088888888DC
:1020F0008850200259692060A02020202020F8026A
:1021000059697088880810204080F8025969F808D9
:1021100010207008088870025969101030505090D3
:10212000F81010025969F88080B0C8080888700259
:10213000596970888080F088888870025969F80829
:1021400010102020404040025969708888887088AB
:1021500088887002596970888888780808887011A2
:10216000386840E040000040E04011386840E040FE
:102170000000604080025969081020408040201013
:1021800008045464F80000F80259698040201008DF
:102190001020408002596970888808102020002093
:1021A00002596970888898A8A8B080780259692077
:1021B00050888888F8888888025969F048484870AB
:1021C000484848F002596970888080808080887013
:1021D000025969F048484848484848F0025969F8A7
:1021E000808080F0808080F8025969F8808080F0DB
:1021F000808080800259697088808080988888708B
:1022000002596988888888F888888888123969E03E
:1022100040404040404040E00259693810101010E2
:1022200010109060025969888890A0C0A09088889A
:102230000259698080808080808080F80259698896
:1022400088D8A8A88888888802596988C8C8A8A892
:1022500098988888025969708888888888888870E2
:10226000025969F0888888F080808080015A6A70FD
:10227000888888888888A87008025969F0888888C2
:10228000F0A090888802596970888080700808885A
:1022900070025969F820202020202020200259694E
:1022A000888888888888888870025969888888889A
:1022B000505050202002596988888888A8A8A8A86A
:1022C00050025969888850502050508888025969B6
:1022D000888850502020202020025969F8081010CA
:1022E00020404080F8113B6BE080808080808080BF
:1022F0008080E00259698080404020101008081159
:102300003B6BE0202020202020202020E008536389
:10231000205088015161F82A22628040025666707E
:102320000878889868025969808080F08888888851
:10233000F002566670888080887002596908080823
:102340007888888888780256667088F88088700255
:10235000596930484040F04040404000586870881B
:10236000888878088870025969808080B0C8888819
:1023700088881238684000C040404040E0004A6A07
:102380001000301010101090906002596980808009
:1023900090A0C0A09088123969C0404040404040A1
:1023A00040E0025666D0A8A8A8A888025666B0C821
:1023B000888888880256667088888888700058687F
:1023C000F0888888F08080800058687888888878CD
:1023D000080808025666B0C8808080800256667081
:1023E00088601088700258684040F0404040483093
:1023F0000256668888888898680256668888885059
:1024000050200256668888A8A8A8500256668850B0
:10241000202050880058688888889868088870024A
:102420005666F810204080F8015B6B1820202020B1
:10243000C020202020182219698080808080808020
:102440008080015B6BC0202020201820202020C02D
:1024500008536348A890FFFFFFFFFFFFFFFFFFFF48
:10246000FFFFFFFFFFFFFFFFFFFFFFFFFFFFFFFF7C
:10247000FFFFFFFFFFFFFF0D006022196980008052
:102480008080808080800358682070A8A0A0A870F9
:102490002002596930484040E0404048B003566649
:1024A00088705050708802596988885050F820F818
:1024B0002020221969808080800080808080124ADC
:1024C0006A609080609090601090601A3262A0A064
:1024D0000359697088A8D8C8D8A88870045767704D
:1024E0000878887800F80356662850A0A050280481
:1024F0005363F80808163161E00359697088E8D819
:10250000D8E8D888700A5161F817446460909060E8
:102510000357672020F8202000F807356540A020E9
:1025200040E007356540A04020C02A22624080007C
:1025300058688888888898E8808002596978E8E82F
:10254000E8E868282828262161C020226240800708
:10255000356540C04040E004576770888888700047
:10256000F8035666A050282850A0025A6A40C0407E
:1025700040E00818283808025A6A40C04040E0107D
:1025800028081038025A6A40A04020A0481828386D
:1025900008025969200020204080888870025A6A09
:1025A00040200020508888F88888025A6A1020004D
:1025B00020508888F88888025A6A3048002050885D
:1025C00088F88888025A6A28500020508888F8883D
:1025D00088025A6A50500020508888F88888025A29
:1025E0006A20502020508888F8888802596958A0AD
:1025F000A0A0B0E0A0A0B8005B6B70888080808055
:102600008088702040025A6A402000F88080F08064
:1026100080F8025A6A102000F88080F08080F8026A
:102620005A6A304800F88080F08080F8025A6A5078
:102630005000F88080F08080F8123A6A804000E014
:102640004040404040E0123A6A204000E0404040B4
:102650004040E0124A6A609000E04040404040E064
:10266000123A6AA0A000E04040404040E0025969B0
:10267000F0484848E8484848F0025A6A285000881C
:1026800088C8A8988888025A6A402000708888887C
:10269000888870025A6A102000708888888888703C
:1026A000025A6A30480070888888888870025A6A9E
:1026B00028500070888888888870025A6A505000B4
:1026C00070888888888870035565885020508801F4
:1026D0005B6B08709898A8A8A8C8C87080025A6A4E
:1026E00040200088888888888870025A6A102000F4
:1026F00088888888888870025A6A30480088888864
:1027000088888870025A6A5050008888888888882B
:1027100070025A6A10200088885020202020025918
:102720006980F0888888F080808002596960909084
:10273000A0A0908888B0025969402000700878886D
:1027400098680259691020007008788898680259C2
:1027500069304800700878889868025969285000E4
:102760007008788898680259695050007008788815
:102770009868025A6A304830007008788898680271
:102780005666702870A0A8500058687088808088AD
:102790007020400259694020007088F880887002DB
:1027A00059691020007088F8808870025969304893
:1027B000007088F88088700259695050007088F85D
:1027C000808870123969804000C040404040E0126B
:1027D0003969204000C040404040E01249696090A3
:1027E00000C040404040E0123969A0A000C0404015
:1027F0004040E0025A6A50206010708888888870D3
:10280000025969285000B0C88888888802596940F0
:1028100020007088888888700259691020007088AC
:102820008888887002596930480070888888887064
:102830000259692850007088888888700259695048
:102840005000708888888870035767202000F8003F
:102850002020015868087098A8A8C870800259699B
:10286000402000888888889868025969102000886C
:1028700088888898680259693048008888888898CC
:1028800068025969505000888888889868005B6B96
:102890001020008888889868088870005A6A8080AC
:1028A000B0C88888C8B08080005B6B5050008888B2
:1028B0008898680888700000000000000000000090
:1028C0000000000000000000000000000000000008
:1028D0000000000000000000000C000000000000EC
:1028E000000C0000000000000012000000000000CA
:1028F0000023000000000000002100000000000094
:10290000004C800000000000005E8000000000001D
:10291000009240000000000000A140000000000004
:102920000121200000000000027F90000000000054
:10293000020010000000000007FFF8000000000087
:10294000040008000000000008000400000000006F
:102950000800060000000000100002000000000057
:10296000301E010000000000207F810000000000F8
:1029700041FFE0800000000043FCF0800000000008
:10298000873B7840000000018EDBFC600000000106
:102990000FEBCC20000000021FEDB610000000027B
:1029A0001FDEB6100000000439CD7F0800000004CF
:1029B00036E0FF08000000087EC0BB84000000185D
:1029C0007F005D86000000107FC0ED8200000020C7
:1029D0003CC07301000000203B337F010000007009
:1029E0001BE77E03800000C81DEEDE04C0000088E7
:1029F0000FDEDC04400001240FDF3C09200001262B
:102A000007DBF8192000027203E7F013900002516F
:102A100001FFE02290000489007F8024480009041F
:102A2000801E004824000BFE400000DFF400100070
:102A30004000008002001FFFFFFFFFFFFE000000BC
:102A40000000000000000000000000000000000086
:102A50000000000000001022103C3C0E1F0010225D
:102A60001004221104001022100822110400102268
:102A700010083C1104001022101022110400102232
:102A80001020221104001E1C1E3C3C0E04000000FD
:102A90000000000000000000000000000000000036
:102AA0000000000000000000000000000000000026
:102AB0000000000000000000000000000000000016
:102AC0000000000000000000000000000000000006
:102AD00000000000000000000000000000000000F6
:102AE00000000000000000000000000000000000E6
:102AF000000000000A003B20454550524F4D204940
:102B00006E6465783A20005570646174696E672060
:102B10007A6F666673657420696E20454550524F22
:102B20004D3A2000060006000600060006000600DA
:102B30000600060006003FC01F800F0006000600CA
:102B40000F001F803FC006000600060006000600BA
:102B5000060006000600060007F8000C0C00100234
:102B6000002001006001804000804003E04001C07F
:102B70004000804000004000006000002000001085
:102B800000000C0C0007F80001FE00030300040025
:102B9000800800401800601000207C0020380020D1
:102BA0001000200000200000200000600000400015
:102BB000008003030001FE00FFFFFF7F80FFC0FFD6
:102BC000C0FFC07F807F80FFC0FFC0FFC03F001EEE
:102BD000000C005A204F6666736574004D6F766571
:102BE0002058004D6F76652059004D6F7665205A4C
:102BF0000045787472756465720052657769706912
:102C00006E670050726F62696E67206661696C65FD
:102C1000640050726F62696E67206661696C6564FA
:102C20000050524F4245204641494C20434C4541BB
:102C30004E204E4F5A5A4C450A00526577697069CA
:102C40006E670A005265776970696E670050726F2F
:102C500062696E67206661696C65640050726F62BC
:102C6000696E67206661696C65640050524F424529
:102C7000204641494C20434C45414E204E4F5A5A24
:102C80004C450A005265776970696E670A00507298
:102C90006F62696E67206661696C65640A005072D4
:102CA0006F62696E67206661696C656400205A3ADC
:102CB000200020593A200042656420583A20000A3A
:102CC0000A426564204C6576656C20436F727265BC
:102CD0006374696F6E204D61747269783A00202BBD
:102CE000000A436F727265637465642042656420F4
:102CF0004865696768742076732E204265642054A5
:102D00006F706F6C6F67793A0A00202B000A42657A
:102D1000642048656967687420546F706F677261DA
:102D20007068793A0A2020202B2D2D2D2042414316
:102D30004B202D2D2B0A2020207C202020202020FD
:102D400020202020207C0A204C207C2020202028AD
:102D50002B29202020207C20520A2045207C202066
:102D60002020202020202020207C20490A204620CE
:102D70007C20282D29204E20282B29207C20470A22
:102D80002054207C20202020202020202020207C57
:102D900020480A2020207C20202020282D292020A7
:102DA00020207C20540A2020207C2020202020204D
:102DB00020202020207C0A2020204F2D2D2046522C
:102DC0004F4E54202D2D2B0A2028302C30290A005C
:102DD0004D65616E206F662073616D706C65642057
:102DE000706F696E74733A200020643A200020628C
:102DF0003A200045716E20636F6566666963696598
:102E00006E74733A20613A200052756E6E696E6777
:102E100020696E204452592D52554E206D6F6465C5
:102E20000A00473239204175746F20426564204C96
:102E30006576656C696E670A0028422961636B00DC
:102E4000284629726F6E74002852296967687400D9
:102E5000284C29656674003F4E756D626572206F5F
:102E6000662070726F626520706F696E747320697E
:102E70007320696D706C61757369626C65202832AE
:102E8000206D696E696D756D292E0A003F285629DF
:102E90006572626F7365206C6576656C206973205E
:102EA000696D706C61757369626C652028302D34B2
:102EB000292E0A00656E7175657565696E67202239
:102EC000004572726F722077726974696E67207440
:102ED0006F20454550524F4D210A00486F6D6520C7
:102EE00025732573257320666972737400206669E3
:102EF0007273740A005A0059005800486F6D6520BB
:102F00000020746F6F206C6F6E6720657874727527
:102F100073696F6E2070726576656E7465640A0001
:102F200020636F6C6420657874727573696F6E20AE
:102F300070726576656E7465640A00436172642020
:102F400072656D6F766564004361726420696E73AB
:102F5000657274656400506C656173652072657399
:102F60006574005052494E5445522048414C5445D6
:102F700044005072696E7465722068616C74656497
:102F80002E206B696C6C28292063616C6C65642150
:102F90000A006265640A002C2073797374656D20E1
:102FA00073746F7070656421204865617465725F29
:102FB00049443A2000544845524D414C2052554E08
:102FC000415741592042454400546865726D616C17
:102FD0002052756E6177617900544845524D414CDD
:102FE0002052554E415741592045310054484552D1
:102FF0004D414C2052554E415741592045300048D3
:10300000656174696E67206661696C65642042451C
:10301000440048656174696E67206661696C656427
:103020000048656174696E67206661696C6564005B
:1030300048656174696E67206661696C65642045E6
:10304000300057726974696E6720746F2066696C0E
:10305000653A20006F70656E206661696C65642C4E
:103060002046696C653A20006F70656E2066616964
:103070006C65642C2046696C653A200046696C6575
:103080002073656C65637465640A002053697A6512
:103090003A200046696C65206F70656E65643A2061
:1030A000006F70656E206661696C65642C204669EE
:1030B0006C653A20002066696C653A20004E6F7797
:1030C00020002220706F73002220706172656E7480
:1030D0003A2200535542524F5554494E45204341E0
:1030E0004C4C207461726765743A22004B494C4C19
:1030F00045442E2000747279696E6720746F2063D6
:10310000616C6C207375622D67636F6465206669FE
:103110006C6573207769746820746F6F206D616EC1
:1031200079206C6576656C732E204D4158206C6556
:1031300076656C2069733A000000000000003F4390
:1031400000001F435761726E696E673A20486F6DC9
:10315000696E672042756D702044697669736F727D
:10316000203C20310A000202040000A0400000A020
:1031700040000000400000254300004543000021BE
:10318000430000F0410000F0410000004100000059
:1031900000FF01014C756C7A426F74204D696E69B5
:1031A000204C4344204F66662E004F6666004F6EEB
:1031B0002000456E6473746F702061626F727400DA
:1031C00053746570732F6D6D004A65726B004163B7
:1031D00063656C65726174696F6E0056656C6F63D0
:1031E000697479005A204F6666736574004164768D
:1031F000616E6365642053657474696E677300560D
:1032000054726176206D696E005654726176206D3D
:10321000696E005654726176206D696E00566D6954
:103220006E00566D696E00566D696E00566D617860
:10323000204500566D6178204500566D6178204527
:1032400000566D6178205A00566D6178205A0056FC
:103250006D6178205A00566D6178205900566D6175
:1032600078205900566D6178205900566D6178209C
:103270005800566D6178205800566D6178205800CE
:103280004D6F74696F6E004573746570732F6D6D4B
:10329000004573746570732F6D6D005A737465709B
:1032A000732F6D6D005A73746570732F6D6D0059B7
:1032B00073746570732F6D6D005973746570732F1F
:1032C0006D6D005873746570732F6D6D0058737455
:1032D0006570732F6D6D004D6F74696F6E00534490
:1032E0002063617264206F6B0A006F70656E526FAD
:1032F0006F74206661696C65640A00766F6C756D29
:10330000652E696E6974206661696C65640A005394
:103310004420696E6974206661696C0A0043616EBD
:103320006E6F7420656E7465722073756264697265
:103330003A2000022E2E004D61696E004D6F7665B9
:1033400020302E316D6D004D6F766520316D6D0032
:103350004D6F76652031306D6D004D6F7665206163
:10336000786973004578747275646572004D6F7684
:1033700065205A004D6F76652059004D6F766520A7
:103380005800746F20726573756D650057616974BC
:1033900020666F72207072696E74005052494E54EC
:1033A000205041555345440045787472756465203A
:1033B0006D6F726500526573756D65207072696E10
:1033C0007400524553554D45204F5054494F4E536C
:1033D0003A0020204E6F7A7A6C653A200020005027
:1033E0006C6561736520776169742E2E2E004865C7
:1033F0006174696E67206E6F7A7A6C65005052490D
:103400004E54205041555345440020204E6F7A7A47
:103410006C653A2000200068656174206E6F7A7ACE
:103420006C652E00507265737320627574746F6ED4
:1034300020746F005052494E54205041555345441A
:103440000020204E6F7A7A6C653A20002000666971
:103450006C616D656E742065787472756465005773
:1034600061697420666F72005052494E5420504179
:10347000555345440020204E6F7A7A6C653A2000FF
:10348000200066696C616D656E74206C6F6164000C
:103490005761697420666F72005052494E54205033
:1034A00041555345440020204E6F7A7A6C653A208E
:1034B00000746F20636F6E74696E75652E2E2E001A
:1034C000616E6420707265737320627574746F6EC0
:1034D00000496E736572742066696C616D656E7407
:1034E000005052494E542050415553454400004D20
:1034F0003234005072696E742070617573656400B7
:103500004D313235004D363030204230004D3234AE
:10351000004D3233202573006175746F25692E6765
:10352000004578747275646572004D6F7665205A37
:10353000004D6F76652059004D6F76652058004D1F
:103540006F76656D656E74004D6F76652061786984
:10355000730044697361626C652073746570706593
:103560007273004D383400426564204C6576656C9A
:10357000696E67004732382058590A4D313039207A
:10358000533137350A473238205A0A4D3130392005
:10359000523134350A4731320A4732390A4D313017
:1035A00034205330004175746F20686F6D6500479B
:1035B0003238004D61696E001000C90210012C0103
:1035C0004001220170011801B0010E01F001040157
:1035D0005002FA00B002F0003003E600D003DC0035
:1035E0009004D2007005C800A006BE000008B40018
:1035F000B009AA00D00BA000600E960060118C00EC
:103600000015820020197800C01D6E00A022640001
:10361000B0275A00902C500000314600E0343C00A6
:1036200010383200903A2800603C1E00A03D140083
:10363000803E0A00203F00001000AD0330016A0107
:1036400050022B0170030A019004F500B005E5005B
:10365000D006D800F007CE001009C500300ABE0021
:10366000500BB700700CB100900DAB00B00EA6006F
:10367000D00FA200F0109D00101299003013950099
:103680005014920070158E0090168B00B0178700B2
:10369000D0188400F0198100101B7E00301C7B00C4
:1036A000501D7900701E7600901F7300B0207000CE
:1036B000D0216E00F0226B001024690030256600D6
:1036C000502663007027610090285E00B0295C00DE
:1036D000D02A5900F02B5600102D5400302E5100E6
:1036E000502F4E0070304B0090314800B0324500F2
:1036F000D0334200F0343E0010363B003037370004
:103700005038330070392E00903A2900B03B230026
:10371000D03C1B00F03D1100103F0100F03F0000C5
:103720004E6F206D6F76652E004B494C4C45442EF4
:10373000200024F4D43050C38E20C2A24017828BC4
:103740007011127A910D816CD90AA861E108C758ED
:103750006607615143061E4B5D05C145A7041A412A
:103760001104093D9803713931034036DB0265339A
:103770009102D4305402802E1D02632CEE01752A72
:10378000C501B028A001102781018F2564012B24D9
:103790004B01E0223401AC211F018D200D01801F5F
:1037A000FC00841EED00971DDF00B81CD200E61B54
:1037B000C600201BBC00641AB200B219A8000A1986
:1037C000A0006A189900D117910040178B00B51618
:1037D000840031167E00B31579003A157300C714C2
:1037E0006F0058146A00EE136600881363002513F7
:1037F0005E00C7125B006C12570015125400C11115
:10380000510070114F0021114B00D61049008D104E
:1038100047004610440002104200C00F4000800FD5
:103820003E00420F3C00060F3B00CB0E3800930ECB
:1038300037005C0E3500270E3400F30D3200C10D49
:103840003100900D3000600D2E00320D2D00050D61
:103850002C00D90C2B00AE0C2900850C29005C0C27
:103860002700350C27000E0C2600E80B2400C40BA3
:103870002400A00B23007D0B23005A0B2100390BE1
:103880002100180B2000F80A1F00D90A1E00BB0AED
:103890001E009D0A1D00800A1D00630A1C00470AC5
:1038A0001B002C0A1B00110A1A00F7091A00DD0977
:1038B0001900C4091900AB091900920917007B0906
:1038C0001800630917004C09160036091600200974
:1038D00016000A091500F5081500E0081400CC08C8
:1038E0001400B8081400A4081400900813007D0800
:1038F00012006B0813005808120046081200340822
:103900001100230811001208110001081100F0072E
:103910001000E0071000D0071000C0071000B0072B
:103920000F00A107100091070E0083070F00740716
:103930000F0065070E0057070E0049070E003B07F2
:103940000D002E070E0020070D0013070D000607BF
:103950000D00F9060C00ED060D00E0060C00D40683
:103960000C00C8060C00BC060C00B0060C00A40637
:103970000B0099060C008D060B0082060B007706E3
:103980000B006C060B0061060A0057060B004C0684
:103990000A0042060A0038060A002E060A0024061B
:1039A0000A001A060A001006090007060A00FD05AB
:1039B0000900F4050900EB050900E2050900D90535
:1039C0000900D0050900C7050900BE050900B505B5
:1039D0000800AD050800A50509009C050800940530
:1039E00008008C050800840508007C0508007405A3
:1039F00008006C050700650508005D050700560511
:103A000008004E0507004705070040050800380577
:103A10000700310507002A050700230507001C05DC
:103A20000600160507000F05070008050600020539
:103A30000700FB040600F5040700EE040600E80496
:103A40000600E2040700DB040600D5040600CF04EC
:103A50000600C9040600C3040600BD040600B7043E
:103A60000600B1040500AC040600A6040600A0048C
:103A700005009B04060095040500900406008A04D6
:103A8000050085040500800406007A04050075041D
:103A90000500700405006B04050066040500610460
:103AA00005005C04050057040500520405004D04A0
:103AB000050048040500430405003E0404003A04E0
:103AC000050035040500300404002C04050027041B
:103AD0000400230405001E0404001A040400160454
:103AE0000500110404000D04040009040500040489
:103AF000040000040400FC030400F8030400F403C1
:103B00000400F0030400EC030400E8030400E403F1
:103B10000400E0030400DC030400D8030400D40321
:103B20000400D0030400CC030400C8030300C50351
:103B3000030024F404D9201BC40C5C0E9804C409AF
:103B40005F0265077101F405F900FB04B300480446
:103B50008700C10369005803550003034500BE02F6
:103B60003A008402310053022A002902250004028F
:103B70002000E4011C00C8011900AF0117009801E2
:103B80001400840113007101100061011000510143
:103B90000E0043010D0036010B002B010B0020012C
:103BA0000B00150109000C01090003010800FB00CE
:103BB0000800F3000800EB000700E4000600DE0048
:103BC0000600D8000600D2000600CC000500C700A1
:103BD0000500C2000500BD000400B9000400B500E6
:103BE0000400B1000400AD000400A9000400A50019
:103BF0000300A20003009F0004009B000300980044
:103C000003009500020093000300900003008D0064
:103C100002008B000300880002008600020084007E
:103C20000300810002007F0002007D0002007B0093
:103C300002007900020077000100760002007400A3
:103C4000020072000100710002006F0002006D00AE
:103C500001006C0002006A000100690002006700B8
:103C600001006600010065000100640002006200BE
:103C7000010061000100600001005F0002005D00C2
:103C800001005C0001005B0001005A0001005900C6
:103C900001005800010057000100560001005500C6
:103CA00001005400010053000000530001005200C5
:103CB000010051000100500001004F0001004E00C2
:103CC00000004E0001004D0001004C0001004B00BF
:103CD00000004B0001004A000100490001004800BB
:103CE00000004800010047000100460000004600B7
:103CF00001004500000045000100440001004300B0
:103D000000004300010042000000420001004100A9
:103D1000000041000100400001003F0000003F00A2
:103D200001003E0000003E0001003D0000003D009B
:103D300001003C0000003C0000003C0001003B0092
:103D400000003B0001003A0000003A000100390089
:103D50000000390001003800000038000000380081
:103D60000100370000003700010036000000360077
:103D7000000036000100350000003500000035006D
:103D80000100340000003400000034000100330062
:103D90000000330000003300010032000000320058
:103DA000000032000100310000003100000031004D
:103DB00001003000000030000000300001002F0042
:103DC00000002F0000002F0000002F0001002E0037
:103DD00000002E0000002E0001002D0000002D002C
:103DE00000002D0000002D0001002C0000002C0020
:103DF00000002C0000002C0001002B0000002B0014
:103E000000002B0000002B0001002A0000002A0007
:103E100000002A0000002A000100290000002900FB
:103E200000002900000029000000290001002800EE
:103E300000002800000028000000280000002800E2
:103E400001002700000027000000270000002700D5
:103E500000002700010026000000260000002600C8
:103E600000002600000026000100250000002500BB
:103E700000002500000025000000250000002500AE
:103E800001002400000024000000240000002400A1
:103E90000000240001002300000023000000230094
:103EA0000000230000002300000023000000230086
:103EB0000100220000002200000022000000220079
:103EC000000022000000220001002100000021006B
:103ED000000021000000210000002100000021005E
:103EE0000000210001002000000020000000200050
:103EF0000000200000002000000020000000200042
:103F00000000200001001F0000001F0000001F0033
:103F100000001F0000001F0000001F0000001F0025
:103F200001001E0000001E0000001E0000001E0018
:103F300000004D383420582059205A204500457241
:103F4000723A204D494E54454D5020424544004D53
:103F5000494E54454D5020747269676765726564B7
:103F6000004572723A204D494E54454D502045311E
:103F7000004572723A204D494E54454D502045300F
:103F8000004572723A204D415854454D50204245EB
:103F900044004D415854454D50207472696767651F
:103FA000726564004572723A204D415854454D5037
:103FB000204531004572723A204D415854454D50CC
:103FC0002045300000060900FE06018902FE20FFA0
:103FD000FE07FE06FE0000000600070106060602B8
:103FE00000808080800080030303060103A0A0A05E
:103FF0000507070600FF5050F850F8505005090912
:104000000600FE2070A8A07028A8702006080806E8
:1040100000FF40A84810204854080507070600FF85
:10402000609090609890680103030602038080808E
:104030000207070602FF4080808080804002070759
:104040000602FF8040404040408005050506000014
:104050008850F850880505050600002020F820202B
:104060000204040602FEC040408005010106000271
:10407000F8020202060200C0C00406060601001093
:104080001020408080040606060100609090909009
:104090006003060606010040C0404040E0040606FA
:1040A0000601006090102040F0040606060100F0B2
:1040B00020601010E005060606000010305090F851
:1040C00010040606060100F080E01010E004060669
:1040D0000601006080E0909060040606060100F092
:1040E0001010204040040606060100609060909089
:1040F00060040606060100609090701060020505DD
:10410000060200C0C000C0C00207070602FEC0C011
:1041100000C040408005050506000018608060185A
:10412000050303060001F800F8050505060000C0B8
:10413000300830C00407070601006090106040009E
:10414000400506060600007090A8B08070050606BF
:10415000060000205088F88888050606060000F052
:1041600088F08888F0040606060100609080809040
:1041700060040606060100E090909090E0040606B8
:10418000060100F080E08080F0040606060100F0E1
:1041900080E0808080040606060100609080B09078
:1041A000600406060601009090F0909090030606C9
:1041B000060100E040404040E005060606000038E9
:1041C000101010906004060606010090A0C0A09098
:1041D000900406060601008080808080F0050606B7
:1041E00006000088D8A8A888880406060601009062
:1041F000D0B09090900506060600007088888888E8
:1042000070040606060100E09090E0808004070735
:104210000601FF609090D0B0601004060606010011
:10422000E09090E090900406060601006090402027
:104230009060050606060000F820202020200406D5
:10424000060601009090909090600406060601001A
:10425000909090F060600506060600008888A8A887
:10426000D8880506060600008850202050880506DC
:10427000060600008888502020200406060601005B
:10428000F010204080F0030606060100E0808080E8
:1042900080E004060606010080804020101003061E
:1042A00006060100E020202020E0050303060003AD
:1042B0002050880501010600FEF8020202060204F1
:1042C0008040040404060100709090700406060605
:1042D00001008080E09090E00404040601007080FA
:1042E000807004060606010010107090907004049F
:1042F0000406010060B0C0700406060601002050EC
:1043000040E040400406060601FE60909070106098
:104310000406060601008080E090909003060606E1
:1043200001004000C04040E00308080601FE2000F4
:1043300060202020A0400406060601008080A0C066
:10434000A090030606060100C040404040E005047E
:1043500004060000D0A8A888040404060100E09028
:104360009090040404060100609090600406060624
:1043700001FEE09090E080800406060601FE709049
:1043800090701010040404060100A0D08080040482
:104390000406010070C030E004060606010040403B
:1043A000E040502004040406010090909070040442
:1043B000040601009090606005040406000088A8CF
:1043C000A8500404040601009060609004060606EC
:1043D00001FE909090709060040404060100F020AB
:1043E00040F00307070601002040408040402001C4
:1043F00007070602FF808080808080800307070611
:104400000100804040204040800402020601035029
:10441000A0FFFFFFFFFFFFFFFFFFFFFFFFFFFFFF0B
:10442000FFFFFFFFFFFFFFFFFFFFFFFFFFFFFFFF9C
:10443000FFFF0000000600070106060602008000DC
:10444000808080800406060601FF2070A0A07020F6
:104450000507070600FF304840F04040F805050515
:10446000060000A8508850A80506060600008850DF
:10447000F820F8200107070602FF80808000808076
:10448000800407070601FF708060906010E0030160
:1044900001060105A0060707060000788494A4948D
:1044A000847803050506010160A06000E0050505AC
:1044B0000600002850A05028040303060100F01055
:1044C00010040101060102F00607070600007884C7
:1044D000B4A4A48478040101060105F004030306D2
:1044E00001026090600507070600FF2020F82020E9
:1044F00000F803050506010140A02040E003050582
:10450000060101C0204020C00202020602044080D1
:104510000405050601FF9090B0D080050606060050
:104520000078E8E8682828010101060202800202FA
:10453000020602FE408003050506010140C040401E
:10454000E003050506010140A04000E00505050661
:104550000000A0502850A00508080600FF40C040F9
:1045600050703078100508080600FF40C0405068C1
:104570000810380508080600FFC0204030F03078E9
:1045800010040707060100200020608090600507E6
:1045900007060000402020507088880507070600A5
:1045A0000010202050708888050707060000205062
:1045B000205070888805070706000028502050709A
:1045C000888805070706000050002050708888057D
:1045D0000707060000205020507088880506060650
:1045E000000078A0F0A0A0B80408080601FE6090C2
:1045F0008080906020400407070601004020F08082
:10460000E080F00407070601002040F080E080F021
:104610000407070601002050F080E080F00407073F
:104620000601005000F080E080F00307070601005B
:104630008040E0404040E00307070601002040E0E2
:10464000404040E003070706010040A0E040404032
:10465000E0030707060100A000E0404040E0050637
:10466000060600007048E848487004070706010085
:1046700050A090D0B0909004070706010040206041
:104680009090906004070706010020406090909091
:1046900060040707060100205060909090600407B6
:1046A0000706010050A06090909060040707060183
:1046B000005000609090906005050506000088504D
:1046C0002050880408080601FF1070B0B0D0D0E078
:1046D0008004070706010040209090909060040736
:1046E00007060100204090909090600407070601A3
:1046F0000020509090909060040707060100500041
:1047000090909090600507070600001020885020C8
:10471000202004060606010080E09090E080040658
:10472000060601006090A0A090A004070706010003
:1047300040200070909070040707060100204000A0
:104740007090907004070706010020500070909050
:104750007004070706010050A000709090700406D6
:1047600006060100500070909070040707060100D3
:104770002050207090907005040406000070A8B0CE
:10478000780406060601FE7080807020400407074A
:1047900006010040200060B0C07004070706010059
:1047A00020400060B0C070040707060100205000E0
:1047B00060B0C070040606060100500060B0C07012
:1047C000030707060100804000C04040E0030707E0
:1047D000060100204000C04040E00307070601003A
:1047E00040A000C04040E0030606060100A000C053
:1047F0004040E004070706010030601070909060B0
:1048000004070706010050A000E0909090040707FD
:104810000601004020006090906004070706010038
:1048200020400060909060040707060100205000BF
:104830006090906004070706010050A0006090900F
:1048400060040606060100500060909060050505B2
:104850000600002000F8002004040406010070B0E7
:10486000D0E00407070601004020009090907004FB
:10487000070706010020400090909070040707068B
:104880000100205000909090700406060601005030
:1048900000909090700409090601FE20400090905D
:1048A000907090600408080601FE8080E09090E01F
:1048B00080800408080601FE50009090907090607F
:1048C00000002200250028002B002E0031003400BB
:1048D00002010000050108010B0100002100240075
:1048E00027002A002D0030003300010100000401E0
:1048F00007010A0105050505070508080808020261
:1049000002020A0A08080404040401010101010169
:1049100001010303030303030303040707070C0C4C
:104920000C0C0C0C0C0C0202020206060606060613
:1049300006060B0B0B0B0B0B0B0B010210202008B8
:1049400008102040102040800201020108040201EA
:104950000102040810204080804020100804020159
:1049600080040201804020100804020108040201B2
:104970000102040810204080010204081020408039
:1049800000000A0B02090C0D0E08070304010000C9
:104990000000000000000000000000000000000017
:1049A00000000000000000000000000012111000D4
:1049B00000000000000000000000000000000000F7
:1049C000000000000000000125301D0C1E24311CD9
:1049D0000B18232F1B0A17FFFF040806FF06222BC4
:1049E0001A4142043803FF362829452744435072B0
:1049F0006F7465637465642050696E0A00021FFF5E
:104A0000FFFFFFFFFF600000000001FF400000000B
:104A10000000FF8000000000007F83CF00000C300A
:104A20003F87FF80000C301F867980000C000F8CC0
:104A300030C7838C30E78C30CFC7CC31F38C30DC7F
:104A4000ECEC33B98C30D86C6C33198C30D06C0CE6
:104A500033198C30D86C0C33198C30DC6C0E3B194C
:104A60008C30CF7C079F198C30C77C038F19400096
:104A70000000000002600000000000061FFFFFFFB2
:104A8000FFFFF82020506C616E6E6572427566669D
:104A9000657242797465733A20002046726565201C
:104AA0004D656D6F72793A2000436F6D70696C656A
:104AB000643A204E6F7620323120323031370A008E
:104AC000207C20417574686F723A2028416C6570B3
:104AD00068204F626A6563747320496E632E2C20D0
:104AE0004C756C7A426F7420476974205265706F00
:104AF0007369746F7279290A004E6F762032312003
:104B00003230313731333A32373A333200204C6168
:104B1000737420557064617465643A2000312E31DD
:104B20002E350A004D61726C696E0020536F6674F9
:104B3000776172652052657365740A00205761744D
:104B40006368646F672052657365740A002042725F
:104B50006F776E206F75742052657365740A00203C
:104B600045787465726E616C2052657365740A00D5
:104B7000506F77657255700A0073746172740A0021
:104B80006572726F722077726974696E6720746FD4
:104B90002066696C650A004572726F723A00456E54
:104BA0006473746F70732025632025632025632050
:104BB000256300205A3A0020593A0020583A0065EF
:104BC0006E6473746F7073206869743A2000656353
:104BD000686F3A00446F6E6520736176696E672076
:104BE00066696C652E0A004D32390045303A200066
:104BF0005A3A2000593A2000583A20004D53312C9F
:104C00004D53322050696E730A002042002050003C
:104C10006F6B00526573656E643A2000290A0020AC
:104C200062797465733B206372632000536574740A
:104C3000696E67732053746F72656420280056652F
:104C40002D6A65726B0056652D6A65726B0056653C
:104C50002D6A65726B00567A2D6A65726B00567A02
:104C60002D6A65726B0056792D6A65726B005679F4
:104C70002D6A65726B0056792D6A65726B005678E5
:104C80002D6A65726B0056782D6A65726B005678D6
:104C90002D6A65726B004D6F74696F6E004D363012
:104CA0003020486F74656E6420746F6F20636F6C82
:104CB0006420746F206368616E67652066696C614B
:104CC0006D656E740A00526573746F72652066615B
:104CD000696C73616665004D3530320A4D35303090
:104CE000004C6F61642073657474696E6773005360
:104CF000746F72652073657474696E6773004164C4
:104D000076616E6365642053657474696E677300C1
:104D10004D61696E00536C6565702E2E2E005072C9
:104D2000696E742061626F727465640041626F75B0
:104D300074204669726D77617265004E6F2053442E
:104D40002063617264005072696E742066726F6DC8
:104D50002053440053746F70207072696E74005257
:104D60006573756D65207072696E7400506175733E
:104D700065207072696E7400436F6E666967757244
:104D80006174696F6E0054656D70657261747572DF
:104D900065004D6F76656D656E74004368616E6782
:104DA000652066696C616D656E740054756E650092
:104DB000496E666F2073637265656E0020496E767A
:104DC000616C696420657874727564657220005343
:104DD00044207072696E74696E6720627974652010
:104DE000004E6F74205344207072696E74696E6750
:104DF0000A00205A00205900580020204D61783ABE
:104E00002000205A00205900580020204D696E3A99
:104E100020004F6E20004F666600536F6674206559
:104E20006E6473746F70733A200053657474696EA6
:104E3000672054726176656C20416363656C6572AE
:104E40006174696F6E3A200053657474696E6720EF
:104E50005265747261637420416363656C6572614D
:104E600074696F6E3A200053657474696E672050E0
:104E700072696E7420416363656C65726174696FF9
:104E80006E3A200053657474696E67205072696EC3
:104E90007420616E642054726176656C2041636396
:104EA000656C65726174696F6E3A20002045002060
:104EB0005A0020204D3930372058005374657070E7
:104EC0006572206D6F746F722063757272656E7497
:104ED000733A0A0020204D383531205A005A2D509F
:104EE000726F6265204F666673657420286D6D2948
:104EF0003A0A0020440020490020204D333034205D
:104F0000500020440020490020204D3330312050F3
:104F1000005049442073657474696E67733A0A00DF
:104F200020460020420020480020204D313435200A
:104F300053004D6174657269616C206865617475B8
:104F40007020706172616D65746572733A0A002039
:104F5000204D3432302053004175746F2042656417
:104F6000204C6576656C696E673A0A00205A00200D
:104F7000590020204D323036205800486F6D652092
:104F80006F66667365743A0A00204500205A002057
:104F9000590020580020420020540020204D32307B
:104FA00035205300416476616E6365643A20533C5A
:104FB0006D696E5F66656564726174653E20543C20
:104FC0006D696E5F74726176656C5F66656564724B
:104FD0006174653E20423C6D696E5F7365676D6507
:104FE0006E745F74696D655F6D733E20583C6D61D2
:104FF000785F78795F6A65726B3E205A3C6D6178A4
:105000005F7A5F6A65726B3E20453C6D61785F65D3
:105010005F6A65726B3E0A00205400205200202017
:105020004D323034205000416363656C65726174A9
:10503000696F6E2028756E6974732F7332293A2058
:10504000503C7072696E745F616363656C3E2052A0
:105050003C726574726163745F616363656C3E206A
:10506000543C74726176656C5F616363656C3E0A83
:1050700000204500205A0020590020204D323031B8
:105080002058004D6178696D756D20416363656CD2
:1050900065726174696F6E2028756E6974732F7301
:1050A00032293A0A00204500205A002059002020C9
:1050B0004D3230332058004D6178696D756D206632
:1050C00065656472617465732028756E6974732FE9
:1050D00073293A0A00204500205A00205900202058
:1050E0004D393220580053746570732070657220FA
:1050F000756E69743A0A0020204D323030204430F9
:105100000A0020204D323030204400204469736171
:10511000626C65640A0046696C616D656E7420732B
:10512000657474696E67733A0020204D31343920FC
:1051300043203B20556E69747320696E2043656C73
:10514000736975730A002020473231202020203BEC
:1051500020556E69747320696E206D6D0A004F666C
:105160006673657473206170706C69656400457264
:10517000723A20546F6F206661722100546F6F2065
:105180006661722066726F6D207265666572656E0B
:10519000636520706F696E740A0048617264636FA2
:1051A0006465642044656661756C7420536574742D
:1051B000696E6773204C6F616465640A0028230080
:1051C000002823000064000000E8030000000096AF
:1051D000430000964300000041000020420000C947
:1051E000420000C9420000C84400405044202863E7
:1051F000616C63756C6174656429210A0020213D2E
:105200002000454550524F4D20435243206D697355
:105210006D61746368202D202873746F7265642932
:105220002000290A002062797465733B2063726351
:1052300020002073746F7265642073657474696EE6
:105240006773207265747269657665642028002032
:105250004D61726C696E3D563430290A002845450F
:1052600050524F4D3D00454550524F4D207665728E
:1052700073696F6E206D69736D61746368200020BF
:105280002F002042403A0020403A004E6F204C69E7
:105290006E65204E756D6265722077697468206353
:1052A0006865636B73756D2C204C617374204C6959
:1052B0006E653A200053544F505045442E20005004
:1052C00072696E7465722073746F707065642064A7
:1052D000756520746F206572726F72732E20466937
:1052E0007820746865206572726F7220616E642028
:1052F000757365204D39393920746F207265737468
:105300006172742E202854656D70657261747572B7
:10531000652069732072657365742E20536574204F
:105320006974206166746572207265737461727449
:10533000696E67290A004E6F20436865636B737559
:105340006D2077697468206C696E65206E756D627A
:1053500065722C204C617374204C696E653A200094
:10536000636865636B73756D206D69736D617463DC
:10537000682C204C617374204C696E653A20004C97
:10538000696E65204E756D626572206973206E6F5F
:1053900074204C617374204C696E65204E756D628B
:1053A00065722B312C204C617374204C696E653A08
:1053B00020004D313130004D3331004D383420580C
:1053C0002059205A204500534420726561642065AD
:1053D00072726F720A00446F6E65207072696E742B
:1053E000696E672066696C650A004B494C4C454400
:1053F0002E20004B494C4C2063617573656420621C
:1054000079204B494C4C20627574746F6E2F706913
:105410006E0A004B494C4C45442E20004B494C4CE5
:105420002063617573656420627920746F6F206DED
:1054300075636820696E6163746976652074696D4F
:1054400065202D2063757272656E7420636F6D6DBB
:10545000616E643A20005A204F6666736574004698
:105460006C6F7700466C6F770046616E20737065D5
:1054700065640046616E2073706565640042656412
:1054800000426564004E6F7A7A6C65004E6F7A7ADE
:105490006C65005370656564005370656564004D0C
:1054A00061696E00416D6178204500416D61782031
:1054B0004500416D6178205A00416D6178205A00A5
:1054C000416D6178205900416D6178205900416D2E
:1054D0006178205800416D6178205800412D747228
:1054E0006176656C00412D74726176656C00412DAA
:1054F0007265747261637400412D726574726163C8
:105500007400416363656C00416363656C004D6FBB
:1055100074696F6E00205A3A0020593A0020436F98
:10552000756E7420583A0020453A00205A3A0020FF
:10553000593A00583A00436F6F6C646F776E0046BB
:10554000616E2073706565640046616E20737065DE
:1055500065640042656400426564004E6F7A7A6C4F
:1055600065004E6F7A7A6C65004D61696E004E4140
:105570004E494E495459494E46CDCCCC3D0AD723CD
:105580003C17B7D13877CC2B329595E6241FB14F15
:105590000A000020410000C84200401C4620BCBE5A
:1055A0004CCA1B0E5AAEC59D7400D600F0D0112413
:1055B0001FBECFEFD1E2DEBFCDBF00E00CBF14E0D5
:1055C000A0E0B2E0EEE8FCE302E00BBF02C007900F
:1055D0000D92AC32B107D9F725E1ACE2B4E001C0DD
:1055E0001D92A230B207E1F715E5CCEAD5E500E05F
:1055F00006C022970109FE010BBF0F94C71DCA3ACE
:10560000D10780E00807A9F70E9467D80D94361EDD
:105610000C9400002F923F924F925F926F927F9274
:105620008F929F92AF92BF92CF92DF92EF92FF92B2
:105630000F931F93CF93DF93CDB7DEB7C958D1092E
:105640000FB6F894DEBF0FBECDBF00918B1020E6E1
:10565000029F80011124055F104F8091BE0680FFDC
:105660001AC0EEECFBE484917F013FEFE31AF30AEA
:10567000811102C0780104C00E947D48F701F3CF78
:10568000D7018D917D01882319F00E947D48F8CFC4
:105690008AE00E947D481092700610926F068FE398
:1056A0008093BD061092BC061092BB061092460471
:1056B000109247041092480410924904F801808126
:1056C0000F5F1F4F8032D1F38E34B1F4818190EDA2
:1056D000980F9A3020F08D3211F08B3269F43296A7
:1056E000DF0131962C9120532A30D0F3CD01FC01FB
:1056F000019620812032D9F3F093B506E093B406E9
:105700007F01BFEFEB1AFB0A10816AE270E0C7016C
:105710000F94071E009739F0DC0111978C918032AD
:10572000E1F311961C921D3429F0143519F0173449
:1057300009F0CAC0F7014E2F9F2F81918032D9F313
:1057400080538A3008F0C0C01093BD062091BB067C
:105750003091BC06E42FF92F6AE0AF014F5F5F4F35
:10576000629FC001639F900D1124208130E020537F
:105770003109820F931F218120532A3030F09093FA
:10578000BC068093BB069A0103C09C01FA01E5CFD9
:10579000D9012F5F3F4F4C914032D1F31D34D1F4EA
:1057A0008E31910591F03CF48731910571F08C3187
:1057B000910581F40AC08537910564F0873791051A
:1057C00024F0803AE3E09E0729F4B0937006A0939A
:1057D0006F067AC01092700610926F06D090B406D1
:1057E00041E050E0FD0131962C91222309F46CC078
:1057F0002132A1F41D3491F48032910579F4F093B3
:105800007006E0936F0663E270E0CF010F94071E0D
:10581000009709F459C0DC011C9256C00FEB020F2F
:105820000A31A0F59F01F90160812F5F3F4F60327F
:10583000D1F320ED260F2A3040F023ED260F223041
:1058400020F06B3211F00C94CF409F01602F70E07C
:10585000DB01B595A795B595A795B595A795AA5BD5
:10586000BB4F07707A01002E01C0EE0C0A94EAF7D4
:10587000FC90FE28FC922115310511F02D1901C074
:1058800020E0DB01A45DBB4F2C930AC020916F0682
:1058900030917006232B21F4B0937006A0936F060D
:1058A000208121542A3110F4DF019CCFDF01319691
:1058B0006C9160536A30D0F39D01F9012F5F3F4F27
:1058C00060816032D1F3F0CF8091BD068D3409F450
:1058D0004FC4843511F40C947B40873411F00C9440
:1058E000B5408091BB069091BC068A31910509F4C0
:1058F000F2C2BCF48430910544F4823091050CF07E
:105900001FC197FF2BC00C94CC408430910509F443
:10591000DEC20C9711F00C94CC400E94EC600C9409
:10592000CC408E31910509F471C33CF48C31910562
:1059300009F45AC30CF4D6C25CC38B35910509F443
:105940000EC48C35910509F40FC48A35910511F008
:105950000C94CC401092BA060C94CC408091140266
:10596000882311F40C94CC400E94434D8AE494E0C7
:105970000E94104A0E9434508091BE0683FD8FC061
:10598000C0905604D0905704E0905804F090590409
:105990002091E50E3091E60E4091E70E5091E80E11
:1059A000C701B6010F949916882309F478C0809135
:1059B0007706811138C06091120270911302882716
:1059C00077FD8095982F0F949F169B01AC016091F5
:1059D00090067091910680919206909193060F9493
:1059E000991687FF20C0C092E50ED092E60EE09295
:1059F000E70EF092E80EEEECFBE484918F010F5F6E
:105A00001F4F882321F00E947D48F801F6CFE7ED73
:105A1000F1E084918F010F5F1F4F882321F00E94D6
:105A20007D48F801F6CFC0905604D0905704E0901E
:105A30005804F09059042091E50E3091E60E409103
:105A4000E70E5091E80EC701B6010F94CB1A20E083
:105A500030E048E453E40F94F21C181604F5C092A9
:105A6000E50ED092E60EE092E70EF092E80EEEEC34
:105A7000FBE484918F010F5F1F4F882321F00E9468
:105A80007D48F801F6CFE8EBF1E084918F010F5FDC
:105A90001F4F882321F00E947D48F801F6CF209106
:105AA0004A0430914B0440914C0450914D04609154
:105AB000D90E7091DA0E8091DB0E9091DC0E0F946E
:105AC000991681111DC020914E0430914F044091D0
:105AD0005004509151046091DD0E7091DE0E809162
:105AE000DF0E9091E00E0F949916811109C060911C
:105AF0000A0270910B0280910C0290910D021AC063
:105B00006091AE027091AF02882777FD8095982F43
:105B10000F949F1620910A0230910B0240910C02C3
:105B200050910D020F94FE162AE037ED43E25CE33C
:105B30000F94FE160E947B8E0E946F4A0C94CC40FC
:105B400020911402222311F40C94CC4011E002970E
:105B500009F010E00E94434D19821A821B821C82B8
:105B60001D821E821F82188682E50E94214C882396
:105B700009F45EC10E948E496B017C012091D90E0F
:105B80003091DA0E4091DB0E5091DC0E63962CAF13
:105B90003DAF4EAF5FAF63978090DD0E9090DE0E0D
:105BA000A090DF0EB090E00E80914A0490914B04DB
:105BB000A0914C04B0914D0467968CAF9DAFAEAFF1
:105BC000BFAF679720914E0430914F04409150042D
:105BD000509151046B962CAF3DAF4EAF5FAF6B97BA
:105BE00020E030E0A901C701B6010F94991688237F
:105BF00009F434C163962CAD3DAD4EAD5FAD6397F6
:105C000067966CAD7DAD8EAD9FAD67970F9499167D
:105C100081110DC0A50194016B966CAD7DAD8EAD6B
:105C20009FAD6B970F949916882309F417C120E054
:105C300030E0A901C701B6010F949916881F882783
:105C4000881F181759F080E090E0A0E8BFEBAB96F2
:105C50008CAF9DAFAEAFBFAFAB970AC020E030E0D6
:105C600040E85FE3AB962CAF3DAF4EAF5FAFAB9775
:105C700063962CAD3DAD4EAD5FAD639767966CAD51
:105C80007DAD8EAD9FAD67970F94CB1AA3966CAF89
:105C90007DAF8EAF9FAFA397A50194016B966CADBE
:105CA0007DAD8EAD9FAD6B970F94CB1AA7966CAF61
:105CB0007DAF8EAF9FAFA797A3962CAD3DAD4EADF8
:105CC0005FADA397CA01B9010F94FE162B013C01E9
:105CD000A7962CAD3DAD4EAD5FADA797CA01B901FA
:105CE0000F94FE169B01AC01C301B2010F94CC1AB4
:105CF0000F94371D6F966CAF7DAF8EAF9FAF6F97D0
:105D000020E030E040E05FE30F94FE162B013C0101
:105D1000A7019601C701B6010F94FE166B017C0125
:105D2000A3019201C301B2010F94FE169B01AC01C5
:105D3000C701B6010F94CB1A0F94371D9B01AC011C
:105D4000AB966CAD7DAD8EAD9FADAB970F94FE164F
:105D50006B017C0167962CAD3DAD4EAD5FAD679795
:105D600063966CAD7DAD8EAD9FAD63970F94CC1AED
:105D700020E030E040E05FE30F94FE162B013C0191
:105D8000A7966CAD7DAD8EAD9FADA79790586F96E1
:105D90002CAD3DAD4EAD5FAD6F970F94A81B9B0131
:105DA000AC01C701B6010F94FE169B01AC01C30103
:105DB000B2010F94CC1A63962CAD3DAD4EAD5FADE4
:105DC00063970F94CB1A69837A838B839C836B963A
:105DD0002CAD3DAD4EAD5FAD6B97C501B4010F94D9
:105DE000CC1A20E030E040E05FE30F94FE162B0178
:105DF0003C016F962CAD3DAD4EAD5FAD6F97A39658
:105E00006CAD7DAD8EAD9FADA3970F94A81B9B018C
:105E1000AC01C701B6010F94FE169B01AC01C30192
:105E2000B2010F94CC1AA50194010F94CB1A12C0A1
:105E300089E40E94214C882331F00E948E496983B5
:105E40007A838B839C838AE40E94214C882331F0DF
:105E50000E948E496D837E838F83988720E030E097
:105E6000A90169817A818B819C810F949916811196
:105E70000BC020E030E0A9016D817E818F81988583
:105E80000F949916882349F0612FCE0101960E9444
:105E900096A00E9434500C94CC40E7E9FBE4849136
:105EA0008F010F5F1F4F882321F00E947D48F8016A
:105EB000F6CFE2EFF1E084918F010F5F1F4F88234F
:105EC00011F40C94CC400E947D48F801F4CF0E945C
:105ED0009DF00C94CC4081E0809314021092B206A5
:105EE0000C94CC400E94C97581110C94CC4080E583
:105EF0000E94214C882321F00E945E49462F01C058
:105F000040E06091E10E7091E20E8091E30E90917D
:105F1000E40E00E010E020E231E409831A832B83D1
:105F20003C8300E010E025E333E40D831E832F83E0
:105F3000388700E010E020EA31E409871A872B87D0
:105F40003C8700E010E020EC3FE70D871E872F879D
:105F5000388B413071F1423021F518A219A21AA2F2
:105F60001BA220E030E040EA51E40F94CC1A7B0100
:105F70008C0120E030E04FE153E40F94F21C18163E
:105F800024F4E12CF12C0FE113E4A701B8014BAF8D
:105F90005CAF6DAF7EAFBE01605E7F4FCE01CB9632
:105FA00011C020E030E040EA51E40F94991687FFD9
:105FB0000BC018A219A21AA21BA2BE01605E7F4FDD
:105FC000CE0109960E9405EB18A219A21AA21BA2E3
:105FD000AE01405E5F4FBE016B5F7F4FCE01019609
:105FE0000E9401EB0C94CC4080E00E948EA40C94A3
:105FF000CC4081E08093CC0E24982C9A0E949D6422
:106000001092CC0E249A2C980C94CC4020E030E0D6
:10601000A9016091D90E7091DA0E8091DB0E9091FA
:10602000DC0E0F94CC1A182F88E5C957DF4F688310
:10603000C758D040C857DF4F7883C858D040C7579B
:10604000DF4F9883C958D0400E94214CC957DF4F79
:106050006881C758D040C857DF4F7881C858D040B2
:10606000C757DF4F9881C958D040882321F00E943C
:106070008E499B0102C09B01812FA901BC0148A34D
:1060800059A36AA37BA320E030E0A9016091DD0E53
:106090007091DE0E8091DF0E9091E00E0F94CC1A7D
:1060A0005B018C0189E50E94214C882321F00E942C
:1060B0008E495B018C01A501B80149835A836B832A
:1060C0007C8340905E0450905F0460906004709008
:1060D000610420915A0430915B0440915C0450911A
:1060E0005D0468A179A18AA19BA10F94CB1A6B01D1
:1060F0007C012FE632E143E85AEB0F94F21C87FF54
:1061000002C00C94CC4022E430E045E253E4C701E5
:10611000B6010F949916181614F40C94CC40A301F0
:106120009201B501C8010F94CB1A6B017C0121E3E8
:1061300038E040EC50EC0F94F21C87FF02C00C9446
:10614000CC4022E430E04FE353E4C701B6010F94A2
:106150009916181614F40C94CC400C94E04081E08D
:106160008093BA060C94CC400E94F3ED0C94CC4082
:106170008091BB069091BC068837910509F4ECC666
:106180000CF0E5C08C34910509F4F2C40CF062C047
:106190008831910509F49AC26CF58231910509F4B0
:1061A000CDC584F497FF02C00C94CC408230910599
:1061B0000CF4BEC1419711F00C94CC400E949FC0DA
:1061C0000C94CC408531910509F476C23CF4449797
:1061D00011F00C94CC40E3E6F2E02DC2863191053B
:1061E00009F46EC2479711F00C94CC400E948DBC0C
:1061F0000C94CC408E31910509F4A7C2C4F48A31C5
:10620000910509F490C20CF480C28B31910509F418
:1062100098C24C9711F00C94CC4040E060E0809123
:106220006F06909170060E942D930C94CC408032A2
:10623000910509F4ADC30CF4F6C38A32910509F453
:1062400093C48B34910511F00C94CC400E94A97634
:106250000C94CC408A36910509F460C5CCF58435A0
:10626000910509F46BC5E4F48135910509F45EC527
:106270004CF48D34910511F00C94CC400E94607662
:106280000C94CC408235910509F454C583359105B1
:1062900011F00C94CC4081E08093B9060C94CC4072
:1062A0008C35910509F47DC54CF48535910511F0C7
:1062B0000C94CC400E940B4C0C94CC408836910539
:1062C00009F45AC48936910509F4B0C40C94CC4041
:1062D0008237910509F469C5DCF48D36910509F41E
:1062E000E8C44CF48B36910511F00C94CC400E941C
:1062F000014D0C94CC408E36910509F48FC48F3635
:10630000910511F00C94CC400E942D4C0C94CC4083
:106310008537910509F44FC54CF48337910511F089
:106320000C94CC400E94BA480C94CC40863791051E
:1063300009F44AC58737910511F00C94CC4081E0EF
:106340008093CC0E24982C9AEFEBF3E041C58F326A
:1063500031E0930711F40C942F3A0CF06EC08C3C92
:10636000910509F44EC6D4F58B39910509F478C42A
:10637000ECF48D37910509F4D5C45CF489379105A7
:1063800011F00C94CC401092C80E109271060C942F
:10639000CC408C38910509F445C48139910511F040
:1063A0000C94CC400E94964C0C94CC40883C9105B7
:1063B00009F4D9C534F48E3B910509F498C40C94C2
:1063C000CC40893C910509F418C68B3C910511F02D
:1063D0000C94CC400E94EE4B0C94CC408D3D91052A
:1063E00009F41FC69CF48E3C910509F412C60CF406
:1063F0000CC6833D910509F410C68C3D910511F042
:106400000C94CC400E942B4D0C94CC408C3251E02B
:10641000950709F453C634F4823E910509F405C684
:106420000C94CC408D32B1E09B0709F471C68E32DA
:10643000914009F4BEC70C94CC40843FF1E09F0723
:1064400011F40C944D3EDCF5803931E0930711F4E2
:106450000C94ED3DE4F48E3551E0950711F40C9465
:10646000DC3F34F48033914009F426C70C94CC40CF
:106470008F35E1E09E0711F40C9410408336914073
:1064800011F00C94CC40E7E9FBE40C9452408239C3
:1064900021E0920711F40C94F43D14F40C94F03DB7
:1064A000843A41E0940711F40C94F83D8C3A914001
:1064B00011F00C94CC400F9450000C94CC408835D3
:1064C000A2E09A0711F40C94A03EB4F4863FE1E0F8
:1064D0009E0711F40C94533E14F40C94503E873FE5
:1064E00021E0920711F40C94563E8C31924011F445
:1064F0000C94643E0C94CC408B3843E0940711F428
:106500000C94A33F4CF48335934011F00C94CC4091
:10651000EEECFBE40C946F3E803AB3E09B0709F489
:1065200075C2873E934011F40C9469400C94CC40A2
:1065300000916F061091700680E50E94214C88231F
:1065400069F00E944E496B017C01BB24B394611534
:1065500071058105910531F4B12C04C0B12CC12C19
:10656000D12C760183E50E94214C8823F9F00E940A
:106570008E4920E030E04AE754E40F94FE160F9471
:10658000151C6B017C01B11013C0611571058105EB
:10659000910571F40115110559F0D8018C918823EA
:1065A00039F061E0C8010E9472C007C0BB2091F3BE
:1065B00060E081E492E00E9482C081E08093000963
:1065C0000E9495F70E943450C114D104E104F104F3
:1065D000D1F08090660490906704A0906804B09019
:1065E00069048C0C9D1CAE1CBF1C0E94454F681991
:1065F00079098A099B0997FF1AC0809100098111C6
:106600000C94354114C080910009882321F080E06A
:106610000F94C104F8CF80914B1260E0882319F0E9
:1066200082E392E002C08AE192E00E9482C010926E
:1066300000090C94CC4084918F010F5F1F4F882379
:1066400021F00E947D48F801F6CF1092F71440E047
:1066500050E0BA0183EA92E10E94BCD68BE1E3EA02
:10666000F2E1DE01159601900D928A95E1F7809195
:10667000A1129091A2129C838B8387E793E09A8367
:10668000898340E050E0BE016F5F7F4F82E094E07D
:106690000E94DB5ECE0101960E9457ACE4E5F2E079
:1066A00084918F010F5F1F4F882311F40C94CC400D
:1066B0000E947D48F801F4CF0E940AAB0C94CC40B4
:1066C00010924B1210924C120C94CC4019821A82E8
:1066D0001B821C8218A219A21AA21BA28091A506D5
:1066E000882341F040E0BE016F5F7F4FCE0180966E
:1066F0000E94EEE580914C12882319F081E080938E
:106700004B120E94A9760C94CC4010924B120E941E
:10671000207784E792E090938509809384090E9412
:10672000A4B90C94CC4080914C12882311F40C94A1
:10673000CC4083E50E94214C81110C943A410C9489
:10674000CC400E94F0F00C94CC4080914C128823F5
:1067500011F40C94CC408DE394E10E94F5A68DE3F6
:1067600094E10E94F8AA10924A1210924912E09005
:106770006F06F090700680914C12882311F40C94EF
:10678000CC400E9400AB1D8218861C821B8287E7CA
:1067900093E09A8389838FE992E19093BF1280936B
:1067A000BE12F70180818F3209F06BC06FE270E09A
:1067B000C7010F94071E8C010F5F1F4F9E012F5FB3
:1067C0003F4F59010115110509F461C06FE270E0F6
:1067D000C8010F94071E6C01009709F459C00817EF
:1067E000190708F055C04C01801A910AA401B8019C
:1067F000CE0180960F94271EE0E2F0E0EC0FFD1F23
:10680000E80DF91D10828E01005E1F4FD8018D9199
:106810008D01882319F00E947D48F8CF8AE00E94FC
:106820007D486091BE127091BF126115710519F01B
:106830006C5F7F4F02C060E070E021E0AE01405E1F
:106840005F4FCE0105960E94E15D811112C0BE012D
:10685000605E7F4F8FE992E00E94217A8EE20E9473
:106860007D488AE00E947D48C5010E9457AC0C9487
:10687000CC40B092BF12A092BE1286010F5F1F4F94
:10688000A1CF80EC92E19093BF128093BE1287015A
:106890006091BE127091BF126115710519F06C5FA5
:1068A0007F4F02C060E070E018A21BA222E0A801A6
:1068B000CE0180960E94E15DF82E882311F1CE0171
:1068C00080960E9433A7F82E8823D9F06CA57DA569
:1068D0008EA59FA541E00E946974F82E882389F057
:1068E000E8A9B0E2EB9FF0011124E659FB4F309785
:1068F00039F085EE80831BA20E94C273F82E01C07E
:10690000F12CCE0180960E9452ACFF2011F149E794
:10691000E42E42E0F42EF7018491882331F0FFEF5A
:10692000EF1AFF0A0E947D48F6CFD8018D918D01A4
:10693000882319F00E947D48F8CF8AE00E947D48A4
:106940001092EE141092EF141092F0141092F114B1
:1069500019C037E8E32E32E0F32EF7018491882343
:1069600031F0FFEFEF1AFF0A0E947D48F6CFD80101
:106970008D918D01882319F00E947D48F8CF8EE219
:106980000E947D48CE0101960E9457AC0C94CC40E9
:1069900080914B1281110E9495F700916F06109122
:1069A000700680E50E94144B882321F00E947F49E5
:1069B000F82E01C0F12C80914C12882311F40C9414
:1069C000CC404F2D61E0C8010E942D9383E50E94C9
:1069D000214C882381F00E945E49AB01BC014093A9
:1069E000EE145093EF146093F0147093F1148DE350
:1069F00094E10E94BCD680914C12882319F081E06A
:106A000080934B12F1100C94CC407BCE80916F069A
:106A10009091700621E020934A1240E060E00E94CD
:106A20002D930C94CC400E9475762CE3C22ED12C71
:106A3000E12CF12CA70196010F946E1A162F072F47
:106A4000CA01B901A70196010F946E1AD62EC72E5E
:106A5000CA01B90128E130E040E050E00F946E1A1D
:106A6000FB01C9016DE671E00F94941D9B014D2D52
:106A70005C2DDE0111967D012115310599F00F93F2
:106A80001F93CF92DF92FF93EF939F938F933F9348
:106A90002F938BED92E09F938F93FF92AF930F9480
:106AA000331612C00097B1F00F931F93CF92DF926D
:106AB000FF93EF939F938F938BEC92E09F938F9331
:106AC000FF92AF930F9433160FB6F894DEBF0FBE4C
:106AD000CDBF30C0309779F00F931F93CF92DF92E4
:106AE000FF93EF938FEB92E09F938F93FF92AF937F
:106AF0000F943316E9CF452B69F00F931F93CF9274
:106B0000DF9287EB92E09F938F93FF92AF930F9466
:106B10003316DACF0F931F9383EB92E09F938F93FB
:106B2000FF92AF930F9433160F900F900F900F902A
:106B30000F900F9060E0C7010E9472C0EEECFBE482
:106B400084918F010F5F1F4F882321F00E947D48A1
:106B5000F801F6CFB7018FEE92E00E94217A8AE029
:106B60000E947D480C94CC400E9439D20C94CC40B9
:106B70000E9420770C94CC4088E690E00E942DF192
:106B800081110C94CC408091BE0683FF02C00C940E
:106B9000CC4083E50E94214C882311F40C94CC4016
:106BA0000E948E490F94101C7093A00E60939F0E4C
:106BB00080E00E94F2C20E948E4920E030E040E76F
:106BC00052E40F94991618163CF00E94607660E02B
:106BD00088E093E00E9482C00E948E492091900636
:106BE0003091910640919206509193060F94F21CB9
:106BF000181614F00C94CC4081EF92E09F938F9381
:106C00008CEF92E09F938F931F920E94AE750F902E
:106C10000F900F900F900F900C94CC400E94354D28
:106C20000C94CC400E946FAD0C94CC4089E690E06F
:106C30000E942DF181110C941B46E0E2F3E0849157
:106C40008F010F5F1F4F882321F00E947D48F801BC
:106C5000F6CF0F9435048AE00E947D480C941B46C1
:106C600083E50E94214C882311F40C94CC400E94AF
:106C70006E4980936E068D3318F08CE380936E0618
:106C80000E94454F6B017C0120916E0630E0A8EE1A
:106C9000B3E00F94BC1AC60ED71EE81EF91EC092B0
:106CA0006A06D0926B06E0926C06F0926D060C9428
:106CB000CC408DE690E00E942DF181110C94CC40E7
:106CC0008091BE0683FF02C00C94CC4083E50E94F5
:106CD000214C60968FAF609781110C944B4182E5F7
:106CE0000E94214C81110C944B410C94CC4080911A
:106CF000BE0683FF02C00C94CC4083E50E94214C69
:106D000068968FAF689781110C94EB4282E50E94E0
:106D1000214C81110C94EB420C94CC400E940E4DFE
:106D20000C94CC400E9480E80C94CC400E9479A442
:106D30000C94CC401092B9060C94CC4083E50E9490
:106D4000214C8823A1F00E948E4920E030E04AE7E0
:106D500054E40F94FE160F94151C60930E0270936A
:106D60000F0280931002909311020C94CC4088E59E
:106D70000E94144B81110C946B4489E50E94144BC2
:106D800081110C946B448AE50E94144B81110C9480
:106D90006B4485E40E94144B81110C946B440C9459
:106DA00089440E9466FF0C94CC400E9495F70F9492
:106DB0008B0F0C94CC4060E080916F069091700630
:106DC0000E9472C00C94CC400E94614B0C94CC4049
:106DD00084918F010F5F1F4F882321F00E947D480F
:106DE000F801F6CFE7EBF3E084918F010F5F1F4FBF
:106DF000882321F00E947D48F801F6CF1E9903C038
:106E00000CE013E002C007E013E0D8018D918D0182
:106E1000882319F00E947D48F8CF8AE00E947D48BF
:106E2000EFEAF3E084918F010F5F1F4F882321F079
:106E30000E947D48F801F6CF379903C00CE013E0BB
:106E400002C007E013E0F80181918F01882319F057
:106E50000E947D48F8CF8AE00E947D48E7EAF3E08F
:106E600084918F010F5F1F4F882321F00E947D487E
:106E7000F801F6CF1D9903C00CE013E002C007E053
:106E800013E0D8018D918D01882319F00E947D486F
:106E9000F8CF8AE00E947D48EFE9F3E084918F010A
:106EA0000F5F1F4F882321F00E947D48F801F6CF25
:106EB000029903C00CE013E002C007E013E0F80100
:106EC00081918F01882319F00E947D48F8CF8AE0D4
:106ED0000E947D48E7E9F3E084918F010F5F1F4F27
:106EE000882321F00E947D48F801F6CF1C9903C049
:106EF0000CE013E002C007E013E0D8018D918D0192
:106F0000882319F00E947D48F8CF8AE00E947D48CE
:106F1000EFE8F3E084918F010F5F1F4F882321F08A
:106F20000E947D48F801F6CF019903C00CE013E000
:106F300002C007E013E0F80181918F01882319F066
:106F40000E947D48F8CF8AE00E947D481092CC0EC6
:106F5000249A2C980C94CC4081E08093C80E8093A6
:106F600071060C94CC4088EC90E00E942DF18111C8
:106F70000C94CC4084E40E94144B8823D1F10E94ED
:106F80008E4911E020E030E0A9010F94991681119B
:106F900001C010E010937606112359F10091980674
:106FA00010E00E948E49F801EE0FFF1FEE0FFF1F49
:106FB000EE58F94F608371838283938320E030E041
:106FC000A901609172067091730680917406909188
:106FD00075060F94991681110CC080E090E0A0E432
:106FE000B0E48093720690937306A0937406B093F6
:106FF00075060E94CB490C94CC400E94424B0C94E5
:10700000CC400E941AF20C94CC400E94924B0C94FB
:10701000CC400F945F010C94CC400E947FF20C9402
:10702000CC400E946DF10C94CC4080E50E94144B42
:10703000882311F40C94CC400E945E49F62E062F52
:10704000172F83E50E94214C882321F00E945E497E
:107050006B0103C0CC24CA94DC2C96012F5F3F4FF8
:107060002330310510F00C94CC4017FF02C00C9473
:10707000CC400E9495F7FFEFCF16DF0631F0CA949F
:10708000CD2871F000E010E00DC08F2D0E94E24E7F
:1070900031E020E0892B09F030E0032F122F02C0ED
:1070A00001E010E08F2D0E94E24E8017910711F44D
:1070B0000C94CC4080E00F94C104F4CF83E50E948F
:1070C000214C882319F00E945E4902C064E071E0FF
:1070D00079A368A380E50E94214C882339F00E949F
:1070E0005E49693833E1730730F402C068EE73E03B
:1070F0007A83698304C088E893E19A838983BE0117
:10710000605E7F4FCE0101960E949E980C94CC4009
:1071100085E40E94214C811110C080E50E94144B2F
:10712000882391F00E948E496093800670938106B7
:10713000809382069093830607C00E946E4988233D
:1071400061F3E7E9FBE471C089E40E94144B8823F2
:1071500081F00E948E492CEA35EC47E25EE30F9401
:10716000FE1660937C0670937D0680937E06909356
:107170007F0684E40E94144B882381F00E948E498C
:107180002CEA35EC47E25EE30F94A81B6093780687
:107190007093790680937A0690937B06EEECFBE47D
:1071A00084918F010F5F1F4F882321F00E947D483B
:1071B000F801F6CF409180065091810660918206D9
:1071C0007091830681EE93E00E94FEF12CEA35EC8B
:1071D00047E25EE360917C0670917D0680917E06B9
:1071E00090917F060F94A81BAB01BC018DED93E03D
:1071F0000E940FF32CEA35EC47E25EE360917806DB
:107200007091790680917A0690917B060F94FE1614
:10721000AB01BC0189ED93E00E940FF38AE00E946C
:107220007D48BAC70E947D48F80184918F010F5FA5
:107230001F4F8111F7CF06E213E0D8018D918D0128
:107240008823B1F10E947D48F8CF8AE50E94144B53
:10725000882309F468C50E948E496B017C0120E0F7
:1072600030E040E050EC0F94F21C87FD4FC520E069
:1072700030E040EA50E4C701B6010F9499161816A1
:107280000CF444C5C0929A06D0929B06E0929C06EC
:10729000F0929D0680E00F94C10E60919A06709165
:1072A0009B0680919C0690919D0642E00E9488F189
:1072B0008AE00E947D4870C780E50E94144B8823B5
:1072C00051F00E948E4960938C0670938D068093D6
:1072D0008E0690938F0689E40E94144B882381F0D8
:1072E0000E948E492CEA35EC47E25EE30F94FE16CD
:1072F000609388067093890680938A0690938B0624
:1073000084E40E94144B882381F00E948E492CEA69
:1073100035EC47E25EE30F94A81B609384067093FC
:1073200085068093860690938706EEECFBE48491B5
:107330008F010F5F1F4F882321F00E947D48F801C5
:10734000F6CF40918C0650918D0660918E0670911B
:107350008F068DEE93E00E94FEF12CEA35EC47E2B9
:107360005EE3609188067091890680918A0690910B
:107370008B060F94A81BAB01BC0189EE93E00E9421
:107380000FF32CEA35EC47E25EE3609184067091DE
:10739000850680918606909187060F94FE16AB01B4
:1073A000BC0185EE93E00E940FF38AE00E947D48C5
:1073B000F3C683E50E94144B182F882371F00E94B6
:1073C0008E490F94101C709313026093120221E0F7
:1073D000672B09F020E02093770680E50E94144B8C
:1073E000882369F08091120290911302892B19F081
:1073F0000E947F4901C081E080937706CDC61111BC
:10740000CBC6EEECFBE484918F010F5F1F4F882306
:1074100021F00E947D48F801F6CF809177068823FD
:1074200019F069E073E002C066E173E086E094E081
:107430000E94217A609112027091130285EF93E00D
:107440000E94C7DFE1EFF3E084918F010F5F1F4FD0
:10745000882309F4A1C60E947D48F801F5CF85E490
:107460000E94214C882321F00E945E491B0102C02A
:10747000212C312C83E40E94214C882349F00E9466
:107480005E49C058DF4F79836883C058D04008C038
:10749000E5E0F0E0C058DF4FF983E883C058D04002
:1074A00085E50E94144B882341F00E947F49CE5706
:1074B000DF4F8883C258D04005C0CE57DF4F1882B7
:1074C000C258D040E12CF12C37FE03C00CE812E486
:1074D00002C006E113E483E50E94214C882321F0D9
:1074E0000E948E497B018C012114310411F4109209
:1074F00098060E94454F2B013C01C101019602975D
:1075000028F4A7E3CA2EA3E0DA2E0BC00AE413E0A6
:10751000D8018D918D01882309F4CACE0E947D483F
:10752000F7CFF60181916F01882319F00E947D4801
:10753000F8CF8AE00E947D480F942C0C8FE7FFEF74
:107540002F163F0619F48093B30E02C08093B50E38
:10755000B701C8010F94101C882777FD8095982FDC
:107560000F949F16AC966FAFAC97AD967FAFAD976B
:10757000AE968FAFAE97AF969FAFAF9781E08093F7
:107580003C02EC964CAE5DAE6EAE7FAEEC97CD5746
:10759000DF4F488259826A827B82C358D040E0968E
:1075A0001FAEE09720E4E1962FAFE1973CE1E29631
:1075B0003FAFE29746E4E3964FAFE397E4961FAE02
:1075C000E497E5961FAEE597E6961FAEE697E79639
:1075D0001FAEE797AB961CAE1DAE1EAE1FAEAB97AF
:1075E000A7961CAE1DAE1EAE1FAEA797C12CD12C08
:1075F0007601FFE78F2E912CA12CB12C8FE790E024
:10760000A0E0B0E06F968CAF9DAFAEAFBFAF6F970D
:10761000C458DF4F188219821A821B82CC57D0407F
:1076200091E0E8969FAFE897A1961FAE1EAEA19796
:1076300010E060961FAE609764961FAE649700E0FE
:1076400080913C02882309F4C1C20E94454F6B9689
:107650006CAF7DAF8EAF9FAF6B978091A30E8823E9
:1076600009F469C10E945495AFEF2A163A0679F4DD
:1076700010919406B09195066096BFAF6097E09127
:1076800096066496EFAF6497009197060EC010912E
:107690009006F09191066096FFAF60972091920658
:1076A00064962FAF649700919306212F60963FADAB
:1076B000609764964FAD6497502FE4966FADE49752
:1076C000E5967FADE597E6968FADE697E7969FAD99
:1076D000E7970F94991687FF12C0E4961FAFE497BF
:1076E00060963FAD6097E5963FAFE59764964FADE6
:1076F0006497E6964FAFE697E7960FAFE797212F8F
:1077000060963FAD609764964FAD6497502FE096BA
:107710006FADE097E1967FADE197E2968FADE2978E
:10772000E3969FADE3970F94F21C181694F4E0963D
:107730001FAFE09760965FAD6097E1965FAFE1970E
:1077400064968FAD6497E2968FAFE297E3960FAFA2
:10775000E397E8969FADE897992309F46EC0AC963D
:107760002FADAC97AD963FADAD97AE964FADAE9702
:10777000AF965FADAF97612F60967FAD60976496CF
:107780008FAD6497902F0F94F21C18160CF0D3C095
:107790006B968CAD9DADAEADBFAD6B978419950961
:1077A000A609B709AC01BD014858534161097109E7
:1077B00077FDC1C06F964CAD5DAD6EAD7FAD6F977F
:1077C000481959096A097B09759567955795479531
:1077D000EFEF2E163E0619F44093B30E02C040930D
:1077E000B50EC458DF4F88839983AA83BB83CC57D7
:1077F000D040AC96FFADAC97E496FFAFE497AD9662
:107800002FADAD97E5962FAFE597AE963FADAE970E
:10781000E6963FAFE697AF964FADAF97E7964FAF7F
:10782000E7976B968CAD9DADAEADBFAD6B97EC960B
:107830008CAF9DAFAEAFBFAFEC97AC962FADAC9712
:10784000AD963FADAD97AE964FADAE97AF965FADEF
:10785000AF97612F60967FAD609764968FAD649708
:10786000902F0F94991687FD02C00C9416466B96C4
:107870008CAD9DADAEADBFAD6B97EC962CAD3DAD77
:107880004EAD5FADEC97821B930BA40BB50BAC0117
:10789000BD01485853416109710977FF02C00C943A
:1078A0001646A1964EAD5FADA197452B11F00C94F5
:1078B0008D446F968CAD9DADAEADBFAD6F97880D0D
:1078C000991DAA1DBB1DB595A79597958795EFEFB7
:1078D0002E163E0611F00C9412468093B30EA1961C
:1078E0002EAD3FADA1972F5F3F4FA1963FAF2EAF7B
:1078F000A197AC963FADAC97E0963FAFE097AD96C1
:107900004FADAD97E1964FAFE197AE965FADAE97B5
:10791000E2965FAFE297AF968FADAF97E3968FAFEA
:10792000E3976B964CAC5DAC6EAC7FAC6B9791E023
:10793000E8969FAFE89720E030E040EA51E4AC964B
:107940006FADAC97AD967FADAD97AE968FADAE9760
:10795000AF969FADAF970F94CC1A9B01AC01612FEE
:1079600060967FAD609764968FAD6497902F0F946B
:10797000F21C18166CF4E6EDF4E084918F010F5FB1
:107980001F4F882309F408C40E947D48F801F5CFF1
:1079900080E398EFAFEFBFEFCD57DF4F28813981FC
:1079A0004A815B81C358D040821B930BA40BB50B5B
:1079B0006B962CAD3DAD4EAD5FAD6B97820F931FB7
:1079C000A41FB51FB7FD13C00F9435048AE00E94B1
:1079D0007D486B968CAD9DADAEADBFAD6B97CD5771
:1079E000DF4F88839983AA83BB83C358D0406B96AB
:1079F0008CAD9DADAEADBFAD6B97880F991FAA1F23
:107A0000BB1F84199509A609B709EC962CAD3DADAD
:107A10004EAD5FADEC97821B930BA40BB50B813879
:107A20009F44A241B10568F0E8EBF4E084918F0136
:107A30000F5F1F4F882309F4AFC30E947D48F801F0
:107A4000F5CFA1964EAD5FADA197C058DF4F8881AD
:107A50009981C058D040841795070CF0B4C0EBE56D
:107A6000F4E084918F010F5F1F4F882321F00E9463
:107A70007D48F801F6CF9FEF2916390619F40AE17F
:107A800013E002C002E014E0B80189E494E00E942F
:107A9000217AB701A60185E494E00E94FEF18AE014
:107AA0000E947D48B80183E394E00E94217AA79662
:107AB0004CAD5DAD6EAD7FADA7978FE294E00E94B7
:107AC000FEF18AE00E947D48B8018DE194E00E94B9
:107AD000217AAB964CAD5DAD6EAD7FADAB9789E1D4
:107AE00094E00E94FEF18AE00E947D48CE57DF4F6D
:107AF000A881C258D040AA2309F44EC32320209461
:107B000089F5C0928C06D0928D06E0928E06F09296
:107B10008F062CEA35EC47E25EE3A7966CAD7DADAF
:107B20008EAD9FADA7970F94FE1660938806709355
:107B3000890680938A0690938B062CEA35EC47E2FF
:107B40005EE3AB966CAD7DAD8EAD9FADAB970F9404
:107B5000A81B609384067093850680938606909395
:107B600087061AC3C0928006D0928106E0928206F0
:107B7000F09283062CEA35EC47E25EE3A7966CAD03
:107B80007DAD8EAD9FADA7970F94FE1660937C06DA
:107B900070937D0680937E0690937F062CEA35ECE9
:107BA00047E25EE3AB966CAD7DAD8EAD9FADAB971E
:107BB0000F94A81B609378067093790680937A06D9
:107BC00090937B06E9C20E94038B3ACD80913C02E0
:107BD0008111E2C20F942C0CDFC20E9495F7DCC227
:107BE00081E00E9417EDD8C280E00E9417EDD4C258
:107BF00086E50E94144B882321F087E795E00F94D7
:107C00004B0F83E50E94144B882321F00E947F498B
:107C1000182F01C010E083E50E94144B882319F04F
:107C2000812F0E94B6ACF0909906111103C0EEECC2
:107C3000FBE41AC0F110FBCFE7E9FBE484918F016C
:107C40000F5F1F4F882321F00E947D48F801F6CF77
:107C5000E8E5F5E084918F010F5F1F4F882339F32A
:107C60000E947D48F801F6CF84918F010F5F1F4F6E
:107C7000882321F00E947D48F801F6CFFF2019F0FB
:107C80006EE173E002C062E273E08AE495E00E9474
:107C9000217A8AE00E947D487FC20E94E1DF7CC297
:107CA0000E947BFA79C20E94FAF876C283E50E94AC
:107CB000144B882319F00E947F4901C081E091E0B4
:107CC00089270E942BF368C283E50E94144B882306
:107CD00009F462C20E947F498093ED0E5DC28491D7
:107CE0008F010F5F1F4F882321F00E947D48F8010C
:107CF000F6CFECEAF5E084918F010F5F1F4F8823E8
:107D000009F4A3CA0E947D48F801F5CFE7E9F5E040
:107D100084918F010F5F1F4F882309F4C9CA0E9405
:107D20007D48F801F5CF40919A0650919B066091ED
:107D30009C0670919D0684E995E00E94FEF1B8CA08
:107D40000E94C975882319F081E00E948EA485E401
:107D50000E94144B882319F00E948E4904C060E0F1
:107D600070E080E090EC2F966CAF7DAF8EAF9FAF50
:107D70002F978AE50E94214C882319F00E948E4992
:107D800004C060E070E080E291E42B966CAF7DAFC0
:107D90008EAF9FAF2B9788E50E94214C882319F066
:107DA0000E948E4904C060E070E080E291E4279672
:107DB0006CAF7DAF8EAF9FAF279789E50E94214CB6
:107DC000882319F00E948E4904C060E070E085E3CA
:107DD00093E423966CAF7DAF8EAF9FAF239785E57D
:107DE0000E94144B882319F00E948E4904C060E061
:107DF00070E088EC92EC6BAF7CAF8DAF9EAF8CE403
:107E00000E94144B882319F00E948E4903C060E041
:107E100070E0CB0168A379A38AA39BA382E40E94AC
:107E2000214C882321F00E945E49F62E02C085E095
:107E3000F82ED0903C128091A50681117EC0CC24F2
:107E4000C394EF2C8E01055C1F4F9E01215C3F4FB8
:107E5000AE014D5B5F4FBE01695B7F4FCE01855B1D
:107E60009F4F0E9416E7882309F467C081E0809342
:107E7000000911E080910009882309F44AC060E0FC
:107E80008F2D0E9414998091A4068823F1F11093FC
:107E90009F0640E050E0BA0185E891EB0E94ACC13A
:107EA00080910009882321F081E00F94C104F8CF6C
:107EB0001092A0061092A1061092A2061092A3069C
:107EC0001092A4060E94F2C20E94E08E10939F06B8
:107ED00040E050E0BA018BED9FEA0E94ACC10E94E5
:107EE000454F685370458F4F9F4F6093A006709326
:107EF000A1068093A2069093A3061092A406109365
:107F0000000961E08F2D0E94149981E00F94C10453
:107F1000B1CF00E010E028E432E409831A832B8318
:107F20003C838091A506882341F04F2DBE016F5FF1
:107F30007F4FCE0180960E94EEE5E1E0DE122CC17B
:107F40000E94A97629C188E50E94144B8823F1F08C
:107F50000E945E498B01222717FD2095322F009346
:107F6000A6061093A7062093A8063093A906DB0166
:107F70002FEF30E00F94C11D20ED37E040E050E0DE
:107F80000F94901AB9018EE20E9475D18AE50E9481
:107F9000144B882329F00E945E4981E00E948F5D86
:107FA00085E40E94144B882309F4F6C00E945E49C0
:107FB00082E00E948F5DF0C083E50E94144B811126
:107FC00004C00FE713E0F12C0FC010E00E946E49CF
:107FD000682F812F0E94A8C71F5F1530B9F7F1CF16
:107FE000F394B4E0FB1671F0D8018D918D010E94DD
:107FF000144B8823A9F30E946E49682F8F2D0E948D
:10800000A8C7EECF82E40E94144B882331F00E946F
:108010006E49682F84E00E94A8C70E9432DFBCC06E
:1080200083E50E94214C8823D1F10E946E49813062
:1080300031F08230A1F50FE713E0F12C21C00FE7FA
:1080400013E0F12CF80181918F010E94214C8823CB
:1080500039F00E946E494FEF682F8F2D0E9429C77B
:10806000F394F4E0FF12EECF82E40E94214C8823C7
:10807000B1F00E946E4913C0F394B4E0FB16A1F373
:10808000D8018D918D010E94214C8823A9F30E9473
:108090006E49482F6FEF8F2D0E9429C7EDCF0E94A8
:1080A00032DF7AC084918F010F5F1F4F882321F048
:1080B0000E947D48F801F6CFE6EBF5E084918F0150
:1080C0000F5F1F4F882309F467C00E947D48F801A5
:1080D000F5CF81E0809314021092B20683E50E94EE
:1080E000144B811103C00E94C8DE56C00E947F4914
:1080F000811152C0F8CFF090BB06FF2001F1EEECE9
:10810000FBE484918F010F5F1F4F882319F0F5D78F
:10811000F801F7CF84E5F1D76F2D70E080E090E0B3
:108120004AE00E94D1DD80E2E8D706E213E0F801E0
:1081300081918F01882309F4BBC8DFD7F8CF109253
:10814000B306EEECFBE484918F010F5F1F4F882391
:1081500019F0D3D7F801F7CF60E070E085EC95E037
:108160000E94C7DF8AE0C9D717C0EEECFBE4849118
:108170008F010F5F1F4F882319F0BFD7F801F7CF8A
:108180006091B4067091B50687ED95E00E94217A62
:1081900082E2B3D78AE0B1D70E945EDE4CC520915F
:1081A0006F0630917006232B39F49F01215031095D
:1081B0003093700620936F0620E030E00C94262C5C
:1081C00080E00E94B6AC0E94575083E50E94144B99
:1081D000882309F448C00E947F4921E0482FBE014E
:1081E0006F5F7F4FCE0180960E943E616B017C01E4
:1081F0009B01AC010F94781D811130C02CEA35EC45
:1082000047E257E368A179A18AA19BA10F94CC1AF8
:10821000AB01BC0182E192E00E940FF32CEA35EC45
:1082200047E257E369817A818B819C810F94CC1A54
:10823000AB01BC018DE092E00E940FF32CEA35EC1B
:1082400047E257E3C701B6010F94CC1AAB01BC015A
:1082500088E092E00E940FF38AE04FD70E943E50E0
:108260000F948B0F99CF81E0B8CF80E00F94C104B9
:108270000C94F5320E945E49AB01BC014093EE14B0
:108280005093EF146093F0147093F1148DE394E124
:108290000E94BCD681CF0E948E490F94101C70930F
:1082A000A00E60939F0E80E00E94F2C20E948E4951
:1082B00020E030E040E752E40F949916181644F09D
:1082C0000E94607660E08FE493E00E9482C002C06A
:1082D0000E94A97660919F0E7091A00E882777FD6D
:1082E0008095982F0F949F162091900630919106BB
:1082F00040919206509193060F94F21C18160CF0C0
:1083000062C181EF92E09F938F9383E493E09F9308
:108310008F931F920E94AE750F900F900F900F9049
:108320000F9081E080933C0267961CAE1DAE1EAE9E
:108330001FAE67976F961CAE1DAE1EAE1FAE6F9739
:1083400010E0A0961FAEA0979CE3A4969FAFA497C1
:10835000ACE1A896AFAFA897B6E4AC96BFAFAC9728
:10836000D12CE12C90E8F92E0FEB812C912C5401AB
:1083700060919F0E7091A00E882777FD8095982FB1
:108380000F949F16762E672E582E492E262F372FA4
:10839000482F592F6D2D7E2D8F2D902F0F949916CC
:1083A0008823D9F020919006309191064091920651
:1083B00050919306672D762D852D942D0F94991647
:1083C000182F111F1127111F6096EFAD6097EE2334
:1083D00041F0112331F011E0E4C07D2C6E2C5F2CB4
:1083E000402E0E94454F6B017C01DC01CB016F9652
:1083F0002CAD3DAD4EAD5FAD6F97821B930BA40BC3
:10840000B50BB7FD38C0D701C60188519C4FAF4F9F
:10841000BF4F6F968CAF9DAFAEAFBFAF6F970F944E
:108420003504EFE3F3E084911F019FEF291A390A25
:10843000882319F062D6F101F6CF81149104A104CA
:10844000B104A9F0C501B40168517C4F8F4F9F4F13
:108450006C197D098E099F0928EE33E040E050E059
:108460000F946E1ACA01B9010E943AD102C08FE37B
:1084700044D68AE042D680E00F94C1040E94345072
:10848000A09190066896AFAF6897209091063090C3
:108490009206009193062A2F322D432D502F672DDF
:1084A000762D852D942D0F94CB1A9F7720E030E008
:1084B00040E251E481149104A104B10429F40F9421
:1084C000991687FD05C006C00F94F21C181614F407
:1084D00046015701112309F44AC067962CAD3DAD02
:1084E0004EAD5FAD6797211531054105510541F04E
:1084F000D701C601821B930BA40BB50BB7FD37C088
:1085000068962FAD6897322D432D502FA0966FADF2
:10851000A097A4967FADA497A8968FADA897AC9688
:108520009FADAC970F94CB1A20E030E040EC5FE3B6
:108530000F94991687FD4FCFD701C601805A9541F8
:10854000AF4FBF4F67968CAF9DAFAEAFBFAF6797D2
:1085500068969FAD6897A0969FAFA097A4962FAE00
:10856000A497A8963FAEA897AC960FAFAC97809112
:108570003C028823B1F081149104A104B10429F4D0
:10858000D72CE62CF52C042DF3CEA8EECA1AA3E0C6
:10859000DA0AE108F108C818D908EA08FB08F7FC6C
:1085A000EFCF80913C02882309F4F6CD60E01123DF
:1085B00029F083E293E00E9482C0EECD81E393E054
:1085C0000E9482C0E9CD6096FFAD6097F111A9CEFF
:1085D0008CEF92E098CEA2D60F94101C67397105EB
:1085E00014F066E970E070939C0E60939B0E0E94FD
:1085F000A7C294D620E030E040EA50E40F94F21C89
:10860000181614F40E94A97660919B0E70919C0E2E
:10861000882777FD8095982F0F949F1620919406B8
:108620003091950640919606509197060F949916B1
:1086300060E087FF03C082E893E002C085E793E033
:108640000E9482C081E080933C028091B3068093B7
:10865000980667961CAE1DAE1EAE1FAE67976F964E
:108660001CAE1DAE1EAE1FAE6F9760961FAE60971C
:10867000A0961FAEA097BCE3A496BFAFA497ECE171
:10868000A896EFAFA897F6E4AC96FFAFAC97C12CD5
:10869000D12C00E8E02E8FEBF82E812C912C540188
:1086A00060919B0E70919C0E882777FD8095982F86
:1086B0000F949F16162F072F782E692E262F372FEF
:1086C000482F592FB601C7010F949916882331F10D
:1086D0002091940630919506409196065091970608
:1086E000612F702F872D962D0F949916881F88273C
:1086F000881F60968FAF609768962FAD689722238A
:1087000089F0882379F080913C02882309F444CDD4
:1087100060E087E693E00E9482C03ECD1C2D0D2DC7
:108720007E2C6F2C0E94454F6B017C01DC01CB013C
:108730006F962CAD3DAD4EAD5FAD6F97821B930B29
:10874000A40BB50BB7FD38C0D701C60188519C4FAB
:10875000AF4FBF4F6F968CAF9DAFAEAFBFAF6F97B0
:108760000F943504E1E7F3E084912F019FEF491A5C
:10877000590A882319F0C1D4F201F6CF811491046B
:10878000A104B104A9F0C501B40168517C4F8F4F19
:108790009F4F6C197D098E099F0928EE33E040E058
:1087A00050E00F946E1ACA01B9010E943AD102C07A
:1087B0008FE3A3D48AE0A1D480E00F94C1040E9487
:1087C0003450209094063090950640909606509034
:1087D00097069101A201612F702F872D962D0F947E
:1087E000CB1A9F7720E030E040EA50E481149104F6
:1087F000A104B10429F40F94991687FD05C006C0A1
:108800000F94F21C181614F4460157016096AFAD90
:108810006097AA2309F443C067962CAD3DAD4EADD9
:108820005FAD6797211531054105510541F0D7012D
:10883000C601821B930BA40BB50BB7FD30C0910191
:10884000A201A0966FADA097A4967FADA497A8961D
:108850008FADA897AC969FADAC970F94CB1A20E044
:1088600030E040EC5FE30F94991687FD4CCFD701C1
:10887000C601805A9541AF4FBF4F67968CAF9DAFF1
:10888000AEAFBFAF6797A0962FAEA097A4963FAEAE
:10889000A497A8964FAEA897AC965FAEAC97809180
:1088A0003C02882309F42FCF81149104A104B10460
:1088B00029F4C12ED02EE72CF62CF2CE98EEC91A50
:1088C00093E0D90AE108F108C818D908EA08FB08BA
:1088D000F7FE19CFEECF0E9495F788E5A5D688233D
:1088E00019F0179A1092C90E89E59ED6882319F0BF
:1088F000169A1092CA0E8AE597D6882319F0159A0F
:108900001092CB0E85E490D6882309F445CC37D558
:1089100043CC0E9495F735D53FCCC458DF4F4880F3
:1089200059806A807B80CC57D040480E591E6A1E01
:108930007B1EC458DF4F288139814A815B81CC5727
:10894000D040281B390B4A0B5B0BCA01B901A501AA
:1089500094010F945F1AA30192010F94901A490198
:108960005A016F968CAD9DADAEADBFAD6F97880EC1
:10897000991EAA1EBB1E94E189169104A104B1049C
:108980001CF1ACEE8A169104A104B1043CF4B0E8E9
:108990008B169104A104B1043CF105C05BEE852E59
:1089A000912CA12CB12C6F968CAE9DAEAEAEBFAE0D
:1089B0006F972EEF30E040E050E0281939094A095E
:1089C0005B0949015A0116C084E190E0A0E0B0E0E3
:1089D0006F968CAF9DAFAEAFBFAF6F9744E1842E63
:1089E000912CA12CB12C06C06F968CAE9DAEAEAE74
:1089F000BFAE6F97E2E4F5E084919F012F5F3F4F98
:108A00008823B9F0C957DF4F2883C758D040C857CB
:108A1000DF4F3883C858D04070D3C957DF4F288103
:108A2000C758D040C857DF4F3881C858D040F901E7
:108A3000E3CF6F966CAD7DAD8EAD9FAD6F970E940D
:108A40003AD1EDE3F5E084919F012F5F3F4F8823FA
:108A5000B9F0C957DF4F2883C758D040C857DF4FF8
:108A60003883C858D04049D3C957DF4F2881C758E9
:108A7000D040C857DF4F3881C858D040F901E3CF04
:108A8000C501B4010E943AD1E0964FADE097E1965E
:108A90005FADE197E2966FADE297E3967FADE39726
:108AA00086E395E00E94FEF1E4964FADE497E596EB
:108AB0005FADE597E6966FADE697E7967FADE797F2
:108AC0008FE295E00E94FEF1A196AEADBFADA197F9
:108AD000139714F40C94593CC501B4010F949F16DC
:108AE00020E030E040E850E40F94FE166B017C017A
:108AF000E0962FADE097E1963FADE197E2964FAD5E
:108B0000E297E3965FADE397E4966FADE497E59661
:108B10007FADE597E6968FADE697E7969FADE79731
:108B20000F94CB1A2BED3FE049E450E40F94FE166E
:108B300020E030E040E05FE30F94FE169B01AC01C3
:108B4000C701B6010F94A81B6B017C01C301B201E0
:108B50000F949F162FE632E143E85AE30F94FE1676
:108B60002B013C01B701A60189E295E00E94FEF1CC
:108B7000B301A20183E295E00E94FEF12AE939E9FE
:108B800049E15FE3C701B6010F94FE166B017C015A
:108B90009B01AC010F94CC1AA30192010F94A81B66
:108BA000A7966CAF7DAF8EAF9FAFA797A301920141
:108BB000C701B6010F94FE1620E030E040E05EE30E
:108BC0000F94FE16AB966CAF7DAF8EAF9FAFAB9799
:108BD000E3E1F5E084913F01BFEF6B1A7B0A882344
:108BE00019F08BD2F301F6CFB701A6018DE095E025
:108BF0000E94FEF1A7964CAD5DAD6EAD7FADA7971F
:108C000087E095E00E94FEF1AB964CAD5DAD6EAD98
:108C10007FADAB9781E095E00E94FEF18AE06DD2D6
:108C20000C94593C8093B50E0C946F3CE8961FAEA3
:108C3000E8970C949B3CC757DF4F0FB6F894DEBF04
:108C40000FBECDBFDF91CF911F910F91FF90EF909D
:108C5000DF90CF90BF90AF909F908F907F906F905C
:108C60005F904F903F902F900895CF92DF92EF92B8
:108C7000FF920F931F93CF93DF937C016A01EB0167
:108C800000E010E00C151D0571F06991D701ED9120
:108C9000FC910190F081E02DC7011995892B19F005
:108CA0000F5F1F4FEFCFC801DF91CF911F910F9141
:108CB000FF90EF90DF90CF900895089580E090E0CE
:108CC000089580E00895FC01E60FF11D849190E085
:108CD000982F88273196E4918E0F911D089508955D
:108CE000DC011696ED91FC91179712968C911297D4
:108CF000481B15968C91483018F0E80FF11D47700D
:108D0000869586958695489F402D1124E40FF11D88
:108D1000362F377080E890E002C0959587953A9598
:108D2000E2F7669566956695E60FF11D3081222380
:108D300011F0832B02C0809583238083089581E006
:108D40000895089590E0FC013197E231F10508F0B3
:108D50004CC0EE58FF4F0D94BB1D809180008F7763
:108D600003C0809180008F7D809380000895809162
:108D70008000877FF9CF84B58F7702C084B58F7D5F
:108D800084BD08958091B0008F7703C08091B000BA
:108D90008F7D8093B0000895809190008F7707C0F9
:108DA000809190008F7D03C080919000877F809399
:108DB000900008958091A0008F7707C08091A00057
:108DC0008F7D03C08091A000877F8093A0000895CD
:108DD000809120018F7707C0809120018F7D03C093
:108DE00080912001877F8093200108953FB7F894F8
:108DF00080918A1190918B11A0918C11B0918D115D
:108E000026B5A89B05C02F3F19F00196A11DB11DE5
:108E10003FBF6627782F892F9A2F620F711D811D02
:108E2000911D42E0660F771F881F991F4A95D1F761
:108E30000895CF93DF932FB7F89494E08902E0016F
:108E40001124FE01E65AF14F608171818281938184
:108E50002FBF0F949F16C251D14F288139814A816B
:108E60005B810F94FE16DF91CF91089580918C0E57
:108E70009FB780FF09C0F89480910B018D7F80938C
:108E80000B019FBF8FEF08C0F89480910B018260A7
:108E900080930B019FBF81E080933D0280918C0EF7
:108EA0009FB781FF09C0F89480910B018160809386
:108EB0000B019FBF8FEF08C0F89480910B018E7F4C
:108EC00080930B019FBF81E080933E0280918C0EC6
:108ED0009FB782FF09C0F89480910B018B7F80932C
:108EE0000B019FBF8FEF08C0F89480910B01846045
:108EF00080930B019FBF81E080933F0280918C0E95
:108F00009FB783FF09C0F89480910B018064809320
:108F10000B019FBF8FEF08C0F89480910B018F7BEE
:108F200080930B019FBF81E08093400208954F9290
:108F30005F926F927F92AF92BF92CF92DF92EF9249
:108F4000FF920F931F93CF93DF938C01EB01FC01F2
:108F500047A050A461A472A4AFA0B8A4C9A4DAA485
:108F60009501A601C301B2010F94991687FF40C075
:108F7000A3019201C301B2010F94FE162B013C0123
:108F8000F80183A994A9A5A9B6A9BC01CD0190585F
:108F90009B01AC010F94CC1AF80127A530A941A977
:108FA00052A90F94FE169B01AC01C301B2010F94AC
:108FB000CB1A0F94371D7B018C019B01AC01B501CD
:108FC000C6010F94991687FF02C0750186019701AB
:108FD000A801B501C6010F949916882349F0A7018D
:108FE000B8014FA358A769A77AA7888181608883B1
:108FF000DF91CF911F910F91FF90EF90DF90CF9075
:10900000BF90AF907F906F905F904F9008958F9238
:109010009F92AF92BF92CF92DF92EF92FF920F9307
:109020001F93CF93DF9300D01F92CDB7DEB755E6E5
:10903000852E51E1952E6EE7A62E67E0B62E0EEB3B
:1090400010E1C12CD12C7601C394F401619171918E
:10905000819191914F01F50121913191419151916E
:109060005F0129833A834B835C830F949D1629818A
:109070003A814B815C810F94FE160F94151CF80108
:1090800061937193819391938F01C616D706E80679
:10909000F90610F46B017C01F5E78F16F1E19F06EC
:1090A000A1F66FEF7FEFCB01A70196010F946E1A27
:1090B00020930A0730930B0740930C0750930D073A
:1090C0000F900F900F900F90DF91CF911F910F9104
:1090D000FF90EF90DF90CF90BF90AF909F908F90D8
:1090E00008958EBD0DB407FEFDCF08958FEF8EBDA0
:1090F0000DB407FEFDCF8EB508959091C00095FF89
:10910000FCCF8093C6000895EF92FF921F93CF93F8
:10911000DF931F92CDB7DEB7182FECE6F8E084910D
:109120007F012FEFE21AF20A882329F09983E5DF05
:10913000F7019981F4CFE12FF92F84917F019FEFFF
:10914000E91AF90A882319F0D8DFF701F6CFE3E529
:10915000F8E084917F01AFEFEA1AFA0A882319F048
:10916000CCDFF701F6CF0F90DF91CF911F91FF90E9
:10917000EF900895CF93DF93E1E2F7E08491EF0160
:109180002196882319F0B9DFFE01F8CFE3E1F7E07B
:109190008491EF012196882319F0AFDFFE01F8CF0B
:1091A000ECEFF6E08491EF012196882319F0A5DF1A
:1091B000FE01F8CFECEEF6E08491EF0121968823D2
:1091C00019F09BDFFE01F8CFEBEDF6E08491EF01A3
:1091D0002196882319F091DFFE01F8CFEAECF6E042
:1091E0008491EF012196882319F087DFFE01F8CFE3
:1091F000EBEBF6E08491EF012196882319F07DDFF7
:10920000FE01F8CFE6EAF6E08491EF01219688238B
:1092100019F073DFFE01F8CFE0E9F6E08491EF0189
:109220002196882319F069DFFE01F8CFEBE7F6E01D
:109230008491EF012196882319F05FDFFE01F8CFBA
:10924000EEE5F6E08491EF012196882319F055DFD1
:10925000FE01F8CFE6E4F6E08491EF012196882341
:1092600019F04BDFFE01F8CFDF91CF9108953FB7A2
:10927000F8942091830980918209821759F0E22F96
:10928000F0E0EE5FF64F808190E02F5F2F77209324
:10929000830902C08FEF9FEF3FBF08958091C506FD
:1092A0009091C606009731F04AE050E060E070E02F
:1092B0000D94D91460E070E0CB0108958091C5064B
:1092C0009091C606009731F04AE050E060E070E00F
:1092D0000D94A81360E070E0CB010895EFDF97FDD7
:1092E0000CC0ECDF6F3F71058105910509F014F4A6
:1092F000E5DF01C06FEF862F089580E0089580912B
:10930000C5069091C606892B39F0E8DF91E08111FE
:1093100001C090E0892F089581E008951F93CF93B5
:10932000DF938091C5069091C6060097E1F0FC019D
:10933000EF011191212F2F7D79F0153411F01536A1
:10934000B9F7188260E070E00F9440121883562F2E
:10935000472F382F292F0BC060E070E0DF91CF91AD
:109360001F910D94401250E040E030E020E0652F66
:10937000742F832F922FDF91CF911F910895149A0C
:109380000895179A1092C90E169A1092CA0E159A3D
:109390001092CB0EF4CFCF92DF92EF92FF92C0905B
:1093A0007206D0907306E0907406F0907506809176
:1093B0007606882321F120E030E0A901C701B6013B
:1093C0000F9499168823D9F020E030E040E05FE365
:1093D000C701B6010F94FE169B01AC010F94FE1657
:1093E0002BED3FE049E450E40F94FE169B01AC01E5
:1093F00060E070E080E89FE30F94A81B04C060E089
:1094000070E080E89FE360930F07709310078093EC
:10941000110790931207FF90EF90DF90CF9008957F
:10942000CF92DF92EF92FF92CF93DF93EC01809186
:109430001502882309F442C0C0909202D090930292
:10944000E0909402F0909502A701960168817981DD
:109450008A819B810F94F21C181624F4C882D98249
:10946000EA82FB82C0909602D0909702E090980228
:10947000F0909902A70196016C817D818E819F8178
:109480000F94F21C181624F4CC82DD82EE82FF8247
:10949000C0909A02D0909B02E0909C02F0909D02B6
:1094A000A7019601688579858A859B850F94F21CB2
:1094B000181624F4C886D986EA86FB86DF91CF91F8
:1094C000FF90EF90DF90CF90089580E1E9EDFEE00E
:1094D000AAE4B4E001900D928A95E1F7089580E145
:1094E000EAE4F4E0A9EDBEE001900D928A95E1F77F
:1094F0000895AF92BF92CF92DF92EF92FF920F93B7
:109500001F93CF93DF93C82FDD27C7FDD0958E0122
:10951000000F111F000F111FF801E353F14F20E05E
:1095200030E0A90160817181828193810F94CC1A0E
:10953000F801ED5AF84F20813181428153810F9417
:10954000CC1A6B017C01F801E65AFB4F60837183F2
:1095500082839383065D194FF8016591759185911A
:1095600094918E01000F111F000F111F98012256B8
:109570003D4F5901A70196010F94CC1AF501608364
:109580007183828393830A5C194FF8016591759109
:1095900085919491CC0FDD1FCC0FDD1FCE56DD4F92
:1095A000A70196010F94CC1A688379838A839B83E1
:1095B000DF91CF911F910F91FF90EF90DF90CF90AF
:1095C000BF90AF9008959091BC10E92FF0E0E75163
:1095D000F14F80839F5F943018F49093BC1002C0C9
:1095E0001092BC1080918C108F5F80938C10089526
:1095F000CF93FC01C62F80818B3399F080918C1022
:10960000843078F42091BC1030E6239FC0011124EF
:10961000BF01855F904F0F94121E8C2FD4DF81E025
:1096200001C080E0CF91089581548A3148F5482FD8
:1096300050E0FA01B3E0F595E795BA95E1F7EA5BFA
:10964000FB4F208130E0877002C0359527958A95C1
:10965000E2F720FF15C0FA01E45DFB4F20812223D1
:1096600039F08091B4069091B506820F911D02C029
:1096700080E090E09093C6068093C50681E008954F
:1096800080E008950F931F93CF93DF93CFE7D3E04C
:1096900005E611E18991C8DF882341F03FDE0F9490
:1096A000151CF80160837183828393830C5F1F4FC5
:1096B000F3E0C338DF0771F7DF91CF911F910F916E
:1096C000A6CCCF93DF9385E4AFDF882369F017DE64
:1096D000882351F0EEECFBE48491EF01219688237E
:1096E00019F00BDDFE01F8CF81E49EDF882369F0DD
:1096F00006DE882351F0E2E4F6E08491EF01219642
:10970000882319F0FADCFE01F8CFC0916F06D091E2
:1097100070068991882311F0F0DCFBCF8AE0DF919D
:10972000CF91EBCC83E580DF882349F0F7DD6093B0
:10973000690770936A0780936B0790936C0784E5C1
:1097400073DF882349F0EADD60936507709366074D
:10975000809367079093680782E466DF882349F067
:109760009DDD6093DB107093DC108093DD1090938F
:10977000DE1088E559DF882349F0D0DD6093991029
:1097800070939A1080939B1090939C1089E54CDF06
:10979000882349F0C3DD60939D1070939E108093E1
:1097A0009F109093A0108AE53FDF882349F0B6DD33
:1097B0006093A1107093A2108093A3109093A410B3
:1097C00085E432DF882349F0A9DD6093A51070930A
:1097D000A6108093A7109093A81008950F931F933D
:1097E000CF93DF93CFE7D3E00DE617E089911CDF3D
:1097F000882331F093DDF801608371838283938342
:109800000C5F1F4FF3E0C338DF0781F7DF91CF9183
:109810001F910F91089583E507DF882389F07EDD8E
:1098200020E030E04AE754E40F94FE160F94151C34
:1098300060935A1170935B1180935C1190935D114A
:109840000895F2DE882339F081E02091C506309139
:10985000C606232B09F480E00895DF92EF92FF9271
:109860000F931F93CF93DF9383E5EBDF882311F0F2
:1098700035DD01C080E08093BE06EEECFBE4849110
:10988000EF012196882319F038DCFE01F8CFECE4D3
:10989000F8E08491EF012196882319F02EDCFE0177
:1098A000F8CF8091BE06882371F10EE318E0C0E086
:1098B000D0E020E08091BE0690E00C2E02C095958D
:1098C00087950A94E2F780FF15C0DD24D394D20E69
:1098D000222311F08CE211DCF80125913491F90179
:1098E00084917901FFEFEF1AFF0A882321F005DC4C
:1098F0009701F5CFD22E21960E5F1F4FC530D105AF
:1099000061F02D2DD7CFE8E4F8E08491EF012196A6
:10991000882319F0F2DBFE01F8CF8AE0DF91CF91C6
:109920001F910F91FF90EF90DF90E7CBCF93DF93E4
:1099300083E587DF882311F0C1DC02C060E070E0BE
:10994000EB01DD27C230D105A8F0E7E9FBE4849103
:10995000EF012196882319F0D0DBFE01F8CFECE16E
:10996000F8E08491EF012196882309F447C0C5DB14
:10997000FE01F7CF88E465DF8823A1F09FDC68371C
:1099800071053CF0633281E078072CF062E271E00F
:1099900002C068E770E0FE01EE0FFF1FE952FF4EC4
:1099A0007183608386E44DDF882391F087DC6F3F0D
:1099B000710519F014F06FEF70E0FE01EE0FFF1F5C
:1099C000E153FF4E77FF02C060E070E07183608377
:1099D00082E437DF882391F071DC6530710534F063
:1099E000683871052CF067E870E002C065E070E04F
:1099F000CC0FDD1FCD52DF4E79836883DF91CF918D
:109A0000089580E51EDF811105C010925F1110924C
:109A10005E11089553DC672BC1F30895CF93DF9354
:109A200083E50FDF882331F049DCEB016F3F7105DF
:109A300019F010F0CFEFD0E080E503DF811105C011
:109A4000D0935F11C0935E1103C048DC8823C1F33B
:109A5000DF91CF91089583E5F4DE882329F02EDC91
:109A60007093AF026093AE0208958EE4EADE88231D
:109A700049F024DC6093DF107093E0108093E110D4
:109A80009093E2100895CF92DF92EF92FF920F939E
:109A90001F93CF93DF933FE7E32E33E0F32E0AE4E7
:109AA00014E0C9EDDEE046EBC42E46E0D42EF7010B
:109AB00081917F01B9DD8823C9F030DCF601208176
:109AC000211104C02091BA06222329F0288139816E
:109AD0004A815B8103C020E030E0A9010F94CC1AD9
:109AE000F801608371838283938309C0888199819F
:109AF000AA81BB81F80180839183A283B3830C5F29
:109B00001F4F2496FFEFCF1ADF0A83E8E81683E0A1
:109B1000F80669F686E495DE8823B9F0FFDB20E0DD
:109B200030E0A9010F94F21C18167CF4F7DB20E05A
:109B300030E040E752E40F94A81B60930A02709350
:109B40000B0280930C0290930D02DF91CF911F9135
:109B50000F91FF90EF90DF90CF90089580911C12AD
:109B600090911D12891B8F7008958CE0E8EFF6E04C
:109B7000A9EDBEE001900D928A95E1F708959FB797
:109B8000F894E2E0F1E080818B7F80839FBF0895AD
:109B90000B96FC01849108950A96FC018491089526
:109BA00068E091C866E08FC8FC0184910895FCDFED
:109BB000882311F0823011F486E0089583E008953F
:109BC000FB014181DC0112962C911297421760F043
:109BD00013962C911397241738F0608115962C91C9
:109BE000621710F424817CC80895FC0120818281D1
:109BF000820F82839181891760F484818F5F8483CF
:109C00008381820F891710F08FEF890F838381E0A2
:109C1000089580E00895FC01128280818150838341
:109C20001482089588E290E00197F1F708952EE9F3
:109C30003FE0009729F0F9013197F1F70197F9CF4B
:109C400008950F93FC010150040F84A996A994175D
:109C500018F0081728F402C0081750F0041740F451
:109C60002150260F83A995A9961720F4281720F4D0
:109C700080E007C0281720F481E0261710F0F8CF05
:109C800081E00F910895DB01ED91FC911994EF9221
:109C9000FF920F931F93CF93DF931F92CDB7DEB741
:109CA0008C01DC011296ED90FC901397D196ED910A
:109CB000FC91D29782E0199520E030E04AE0B701AC
:109CC000C801E1DFF82ED801D196ED91FC91D29731
:109CD00083E01995D801D196ED91FC91D29780E05F
:109CE0001995FF2081F1F801628173819E012F5F38
:109CF0003F4F46E4C801C7DF8981D8018C93129693
:109D00006D917C9113979E012F5F3F4F47E4C801EF
:109D1000BADF8981F80181836281738120E030E0BC
:109D200048E4C801B0DFD8011B968C931B979801BB
:109D30002D5C3F4F12966D917C91139747E1C801BE
:109D4000A2DF81E001C080E00F90DF91CF911F91F1
:109D50000F91FF90EF9008958F929F92AF92BF92D4
:109D6000CF92DF92EF92FF926B017C013FD84B01C3
:109D70005C01C114D104E104F104D9F037D86819A9
:109D800079098A099B09683E73408105910588F32A
:109D900021E0C21AD108E108F10888EE880E83E0BC
:109DA000981EA11CB11CC114D104E104F10431F7C7
:109DB000E0CFFF90EF90DF90CF90BF90AF909F905B
:109DC0008F900895CF93DF93282F30E0F901E0586A
:109DD000F64B8491F901E65CF64BD491F901EC5015
:109DE000F74BC491CC2391F081110E94A246EC2F35
:109DF000F0E0EE0FFF1FE05FF94FA591B4912C91B9
:109E00002D2381E090E021F480E002C080E090E02A
:109E1000DF91CF9108950F931F93CF93DF931F92FC
:109E2000CDB7DEB7282F30E0F901E058F64B84912A
:109E3000F901E65CF64B1491F901EC50F74B0491F3
:109E40000023C9F0882321F069830E94A24669811A
:109E5000E02FF0E0EE0FFF1FE054F74BA591B49117
:109E60009FB7F8948C91611103C01095812301C0B4
:109E7000812B8C939FBF0F90DF91CF911F910F91FA
:109E8000089561E0FC018081C6CF2FB7F8946091FE
:109E90008F117091901180919111909192112FBF1B
:109EA00008950F931F93CF93DF93EB01EEDF8B01A8
:109EB0001DD98F3F41F0E9DF601B710B6C177D07E7
:109EC000B8F380E001C081E0DF91CF911F910F9145
:109ED0000895CF92DF92FF920F931F93CF93DF935A
:109EE00000D01F92CDB7DEB76C01F62EFC01828147
:109EF000982F906A96959CBD80FD06C091E08630B3
:109F000009F490E0892F01C080E08DBD60E0F6018A
:109F1000808129833A834B835C837DDF6CE271E02F
:109F2000C601BFDF8F2D8064DCD808E110E05C81C2
:109F30004B813A812981DA01C901002E04C0B6950E
:109F4000A795979587950A94D2F729833A834B83EF
:109F50005C83C7D80850110929813A814B815C8103
:109F6000083FFFEF1F0739F7FF2029F088E0F816B8
:109F700021F08FEF03C085E901C087E8B2D8ECE09B
:109F8000FE1201C0B3D810E0B1D8F601838387FF79
:109F900004C01F3F11F01F5FF7CF0F900F900F907D
:109FA0000F90DF91CF911F910F91FF90DF90CF9095
:109FB0000895CF92DF92EF92FF920F931F93CF936A
:109FC000DF93EC0162DF0E811F8128853985011541
:109FD00011052105310591F53C853323E1F12A85F1
:109FE00031503C8731E0320F3A874D85341301C040
:109FF0001A86FE0134E0239FE00DF11D1124068531
:10A000001785208931890A831B832C833D836B014B
:10A010007C01C00ED11EE11CF11CCE82DF82E886DD
:10A02000F9868C819D81892BB1F09FB7F89480913E
:10A0300002018460809302019FBF0DC06B017C010F
:10A04000C01AD10AE20AF30AF7FC05C098DD1E82A5
:10A050001F8218861986DF91CF911F910F91FF9073
:10A06000EF90DF90CF90089510DF609366047093B7
:10A070006704809368049093690408958091C106F1
:10A080009091C206A091C306B091C40680930A02C3
:10A0900090930B02A0930C02B0930D028091BF0627
:10A0A0009091C0069093AF028093AE02DDCF809175
:10A0B0000A0290910B02A0910C02B0910D028093C4
:10A0C000C1069093C206A093C306B093C4068091C4
:10A0D000AE029091AF029093C0068093BF0684E6D3
:10A0E00090E09093AF028093AE02BECF0F93CF93D8
:10A0F000DF93C82FD62F04E0262F41E3682F8AE98B
:10A1000091E19FDD8823C9F02D2F41E36C2F8AE96F
:10A1100091E10E9421B78C2F0E9488AD8FEF8D0FA7
:10A120008C0F0E9488AD2D2F44E36C2F8AE991E1BA
:10A13000DF91CF910F910C9421B7DF91CF910F91C7
:10A1400008957F928F929F92AF92BF92CF92DF92AB
:10A15000EF92FF920F931F93CF93DF93CDB7DEB7AC
:10A160002A970FB6F894DEBF0FBECDBF10928911AB
:10A1700080918111882351F00E94305D40E050E0D1
:10A18000BA018EE79EEE0E94ACC1C8C44091AE02F7
:10A190005091AF028091851190918611A091871105
:10A1A000B09188119A01280F391F4436510524F4C3
:10A1B000253631053CF41CC04436510551F0243697
:10A1C0003105B4F484E690E09093AF028093AE0240
:10A1D00013C08B309105A105B1051CF02A5031093F
:10A1E00007C0863F9F4FAF4FBF4F74F4265F3F4F6E
:10A1F0003093AF022093AE02109285111092861117
:10A2000010928711109288118091AE029091AF0246
:10A210008A3091053CF0883E23E092072CF087EECF
:10A2200093E002C08AE090E09093AF028093AE0288
:10A230000E94A8C0782E0E9424D38091CE1185312F
:10A2400098F4772049F080915E1190915F11892BED
:10A2500019F00DE015E102C000EF13E123E14FE03A
:10A2600061E089E00E941AAD8091CE118D3108F035
:10A2700084C1883008F03FC08091A406711002C0EC
:10A28000811139C060919F0E7091A00E882777FDD3
:10A290008095982F0F949F1620E030E040E05FE318
:10A2A0000F94CC1A0F94101C643671052CF46A308C
:10A2B000710524F04CE003C042E101C046E022E118
:10A2C00030E0241B310937FF02C02F5F3F4F359527
:10A2D00027953195219531092B5F2093D11127E0E6
:10A2E0002093D211CB010E94F27C0E9481D38DEE8B
:10A2F00093E10E9474D38091CE118D31D0F580917D
:10A30000D0118531B0F120E030E040E05FE36091B2
:10A3100090067091910680919206909193060F9409
:10A32000CC1A0F94101C9B01643671050CF0F4C21A
:10A330002A3031050CF4EEC24CE022E130E0241B5F
:10A34000310937FF02C02F5F3F4F35952795319573
:10A35000219531092B5F2093D1112CE12093D2114B
:10A36000CB010E94F27C0E9481D38DEE93E10E948A
:10A3700074D38091CE11853140F58091D011813117
:10A3800020F160919F0E7091A00E882777FD809537
:10A39000982F0F949F16209190063091910640912E
:10A3A0009206509193060F94F21C18160CF0B6C248
:10A3B0001092BA1102E022E041E16DE08AE991E1F8
:10A3C0000E94A1B781E08093BA118091CE118830AC
:10A3D00008F03FC08091CA06711002C0811139C0D7
:10A3E00060919B0E70919C0E882777FD8095982F29
:10A3F0000F949F1620E030E040E05FE30F94CC1A0A
:10A400000F94101C643671052CF46A30710524F029
:10A410004CE003C042E101C046E022E130E0241BF1
:10A42000310937FF02C02F5F3F4F35952795319592
:10A43000219531092F5A2093D11127E02093D21171
:10A44000CB010E94F27C0E9481D38DEE93E10E94A9
:10A4500074D38091CE118D31D0F58091D01185319A
:10A46000B0F120E030E040E05FE36091940670914D
:10A47000950680919606909197060F94CC1A0F94AA
:10A48000101C9B01643671050CF053C22A30310553
:10A490000CF44DC24CE022E130E0241B310937FFBF
:10A4A00002C02F5F3F4F3595279531952195310992
:10A4B0002F5A2093D1112CE12093D211CB010E946D
:10A4C000F27C0E9481D38DEE93E10E9474D380913F
:10A4D000CE11853140F58091D011813120F160910C
:10A4E0009B0E70919C0E882777FD8095982F0F9476
:10A4F0009F162091940630919506409196065091B2
:10A5000097060F94F21C18160CF015C21092BA118F
:10A5100002E022E042E168E58AE991E10E94A1B708
:10A5200081E08093BA118091CE118C3130F5809109
:10A53000D011843110F180915E1190915F110196DC
:10A5400044E6489F9001499F300D112437FF02C017
:10A5500021503F4F832F932F990F990B009769F04C
:10A5600028E62093D1112BE12093D2110E94F27C96
:10A570000E9481D385E20E9443D38091CE1184331F
:10A5800028F48091D0118A3208F0DEC18091CE117A
:10A59000853328F48091D011813308F0F9C180917E
:10A5A0004B12882309F44DC08091CE11843308F0FA
:10A5B00048C08091D011823308F443C08091401488
:10A5C000882309F4E9C18091EA149091EB14A091D9
:10A5D000EC14B091ED140097A105B10509F4DCC1AC
:10A5E000BC01CD016D597F4F8F4F9F4F24E630E066
:10A5F00040E050E00F946E1A6091EE147091EF14E9
:10A600008091F0149091F1140F946E1A622F48E427
:10A61000649FB0011124882777FD8095982F0F94AF
:10A620009F162AE037ED43E25CE30F94FE160F9489
:10A63000151C262F02E042E367E38AE991E10E94BC
:10A64000A1B78091CE11813308F05DC08091D01107
:10A65000893208F458C00E9475766B017C018CE346
:10A66000882E912CA12CB12CC701B601A501940113
:10A670000F946E1ACA01B901A50194010F946E1AC4
:10A68000CA01962E872E59018E010F5F1F4F41E898
:10A69000C41641E5D40641E0E406F10408F47EC1A5
:10A6A000B90128E130E040E050E00F946E1A7901E2
:10A6B0008F929F92C50168E170E00F94941D9F9363
:10A6C0008F933F932F932DE239E03F932F931F9366
:10A6D0000F930F9433160FB6F894DEBF0FBECDBFA5
:10A6E0009AE0E916F10408F488C198E0892F880FF0
:10A6F000890F8195855A8093D11180E38093D2117F
:10A70000C8010E9481D3E0919411F0919511848148
:10A710008111CCC06091D90E7091DA0E8091DB0E60
:10A720009091DC0E0F94101CCB010E94897CBC011F
:10A7300080EE96E00F94121E6091DD0E7091DE0E99
:10A740008091DF0E9091E00E0F94101CCB010E94BF
:10A75000897CBC018BED96E00F94121E2CEA35EC3F
:10A7600047E257E36091E10E7091E20E8091E30EB3
:10A770009091E40E0F94CC1A20E030E048EC52E4C3
:10A780000F94FE160F94101C6B017C0197FD19C0ED
:10A7900090E1C91697E2D906E104F104E4F0C7019B
:10A7A000B60120E137E240E050E00F94901ACA0170
:10A7B000B9012AE030E040E050E00F94901A605D6B
:10A7C0000BC0F094E094D094C094C11CD11CE11C47
:10A7D000F11C6DE201C060E26093CC0628EEC21667
:10A7E00023E0D206E104F10494F0C701B60128EE9B
:10A7F00033E040E050E00F94901ACA01B9012AE01A
:10A8000030E040E050E00F94901A605D01C060E2DB
:10A810006093CD06C701B60124E630E040E050E089
:10A820000F94901A9AE0892E912CA12CB12CCA0178
:10A83000B901A50194010F94901A605D6093CE0652
:10A84000C701B601A50194010F94901A162F662333
:10A8500081F08EE28093CF06CA01B901A50194016F
:10A860000F94901A605D6093D006105D1093D1062E
:10A8700017C0CA01B901A50194010F94901A66236B
:10A8800039F08EE28093CF06605D6093D00605C0FC
:10A8900080E28093D0068093CF0680E28093D10639
:10A8A0006CEC76E084ED96E00F94121E8091CE1150
:10A8B0008632A8F48091D0118E3188F008E020E82B
:10A8C0004EE160E08AE991E10E94A1B78091CE114A
:10A8D000863228F48091D0118F3108F090C0809199
:10A8E000CE11823328F48091D0118C3208F0F7C059
:10A8F0008091CE118F3308F011C18091D01188332F
:10A9000008F40CC11092D1118EE38093D2110E94F1
:10A91000D5D304C146E011CD42E10FCD02E022E0E3
:10A9200041E16DE08AE991E10E94A1B74ECD46E098
:10A93000B2CD42E1B0CD02E022E042E168E58AE931
:10A9400091E10E94A1B7EFCD07E028E04AE26AE278
:10A950008AE991E10E94A1B705E022E04CE262E3BE
:10A960008AE991E10E94A1B76AE08AE2BFDB6091C7
:10A970009C1170919D1182E38093B6118BE28093BC
:10A98000B71126EB31E142E38AE991E17CD9FECDB2
:10A990006AE486E3ABDB03CE60E039CE44E6A4167E
:10A9A000B104C0F48F929F92C50168E170E00F94EA
:10A9B000941D9F938F9383E299E09F938F931F93AE
:10A9C0000F930F9433160FB6F894DEBF0FBECDBFB2
:10A9D00095E08CCE8F929F923F932F938BE199E0DD
:10A9E0009F938F931F930F930F9433160FB6F89482
:10A9F000DEBF0FBECDBF96E079CE97E077CE109246
:10AA0000BA1183E08093D11185E28093D21177202F
:10AA100029F08BEE93E10E9474D30DC080915F0703
:10AA2000811102C08FE305C08091C90E8111F1CF61
:10AA300080E20E9443D38BE08093D11115E2109302
:10AA4000D21180EE96E00E9481D38BE28093D111E7
:10AA50001093D211772029F089EE93E10E9474D3EC
:10AA60000DC080916007811102C08FE305C0809105
:10AA7000CA0E8111F1CF80E20E9443D383E3809319
:10AA8000D11115E21093D2118BED96E00E9481D383
:10AA900083E58093D1111093D211772029F087EEAE
:10AAA00093E10E9474D30DC080916107811102C0AF
:10AAB0008FE305C08091CB0E8111F1CF80E20E941F
:10AAC00043D38BE58093D11185E28093D21184ED3D
:10AAD00096E00E9481D381E08093BA1100CF84E098
:10AAE0000E942BD383E08093D11112E31093D211F3
:10AAF00086E00E9462D30E9424D38CE08093D1111F
:10AB00001093D2118091AE029091AF020E94F27C1C
:10AB10000E9481D385E20E9443D3EACE2A960FB6E3
:10AB2000F894DEBF0FBECDBFDF91CF911F910F9183
:10AB3000FF90EF90DF90CF90BF90AF909F908F905D
:10AB40007F9008951F93CF93DF9310928911809186
:10AB5000851190918611A0918711B0918811813053
:10AB60009048A105B10540F0109285111092861110
:10AB70001092871110928811C09185114091C806DA
:10AB8000141604F5842F992787FD909505972C2F8F
:10AB9000332727FD309528173907A4F045301CF0DE
:10ABA000CBEFC40F01C0C0E08C2F992787FD909593
:10ABB000A92FB92F8093851190938611A0938711A7
:10ABC000B0938811C0938211D0E012E0C11109C086
:10ABD0008091B0028823D9F121E041E068ED78E06E
:10ABE00020C0C13049F48091B002882381F120E077
:10ABF00041E069EC78E015C0C23049F48091B002C0
:10AC0000882329F120E041E069EB78E00AC0C330F5
:10AC100061F48091B0028823D1F020E041E062EB42
:10AC200078E08D2F0E9474AF12C0C43081F48091FF
:10AC3000B002882351F021E040E067EA78E08D2FF0
:10AC40000E9474AF8D2F0E948CD31093B002DF5FEF
:10AC5000CF5FD53009F0BACFD093C806DF91CF913E
:10AC60001F9108951F93CF93DF93109289118091C4
:10AC7000851190918611A0918711B0918811813032
:10AC80009048A105B10540F01092851110928611EF
:10AC90001092871110928811C09185114091C706BA
:10ACA000141604F5842F992787FD909505972C2F6E
:10ACB000332727FD309528173907A4F045301CF0BD
:10ACC000CBEFC40F01C0C0E08C2F992787FD909572
:10ACD000A92FB92F8093851190938611A093871186
:10ACE000B0938811C0938211D0E012E0C11109C065
:10ACF0008091B0028823D9F121E041E06AE978E04F
:10AD000020C0C13049F48091B002882381F120E055
:10AD100041E061E978E015C0C23049F48091B002A9
:10AD2000882329F120E041E061E878E00AC0C330DF
:10AD300061F48091B0028823D1F020E041E06FE718
:10AD400078E08D2F0E9474AF12C0C43081F48091DE
:10AD5000B002882351F021E040E064E778E08D2FD5
:10AD60000E9474AF8D2F0E948CD31093B002DF5FCE
:10AD7000CF5FD53009F0BACFD093C706DF91CF911E
:10AD80001F9108950F931F93CF93DF931092891112
:10AD90008091851190918611A0918711B0918811B1
:10ADA00081309048A105B10540F0109285111092B4
:10ADB00086111092871110928811C09185114091CF
:10ADC000C9061416D4F4842F992787FD909501970E
:10ADD0002C2F332727FD30952817390774F0CFEF34
:10ADE000C40F8C2F90E0A0E0B0E080938511909389
:10ADF0008611A0938711B0938811109283118091CE
:10AE00008211C81714F4C09382118091821199277E
:10AE100087FD909504962C2F332727FD30958217B8
:10AE2000930724F48CEF8C0F809382111091821180
:10AE3000D0E081E002E0111123C08823B9F01C1694
:10AE4000ACF04091851150918611609187117091FD
:10AE500088114F5F5F4F6F4F7F4F40938511509325
:10AE600086116093871170938811CF5F8091B00233
:10AE7000882309F469C021E041E06CE079E04EC02C
:10AE8000113019F58823B9F0C230ACF44091851126
:10AE90005091861160918711709188114F5F5F4FBB
:10AEA0006F4F7F4F409385115093861160938711A8
:10AEB00070938811CF5F8091B002882309F444C059
:10AEC00020E040E067EF78E029C01230E9F480919B
:10AED0008111811105C08091B0028823A9F109C0B8
:10AEE000C230C9F70E940AC280918311882399F366
:10AEF00033C081E0C23009F080E024E042EF58E046
:10AF00006D2F0E946DB820C0133061F48091B002A3
:10AF10008823D1F020E041E060EF78E08D2F0E949F
:10AF200074AF12C0143081F48091B002882351F0C4
:10AF300021E040E065EE78E08D2F0E9474AF8D2F08
:10AF40000E948CD30093B002DF5F1F5FD53011F0F9
:10AF500080E071CFD093C906DF91CF911F910F91FF
:10AF600008955F926F927F928F929F92AF92BF925D
:10AF7000CF92DF92EF92FF920F931F93CF93DF93C5
:10AF8000EC01C62ED42EB22EEC80FD80C7010E94AB
:10AF9000D44D182F8C819D810E94D74D982E113051
:10AFA00011F00FEF01C00FE08C819D810E94CC4D0C
:10AFB000182F8C819D810E94C84DA82E8C819D8167
:10AFC0000E94D04D20E62B1530F4009721F0E80EBA
:10AFD000F91E11E610C08C819D810E94D24DE0E4E3
:10AFE000EB1530F4009721F0E80EF91E11E403C0D0
:10AFF000F1E1EF0EF11CAB1430F4188A1B8A1C8AA5
:10B00000198A1A8A99C0A116C0F3A92DB0E0F701D8
:10B0100084918F3F21F4FFEFEF1AFF0A3FC01B110D
:10B0200035C08C819D810E94D44D97012F5F3F4F89
:10B03000F701882311F0823091F484918B8BF90110
:10B0400024912C8BF7013396E491E88BF701349629
:10B05000E491E98BF7013596E491EA8B24C0949151
:10B06000892F8F7082508A8B92959F70998BF901EE
:10B070002491822F8F708C8B22952F702B8BF70150
:10B080003296E491E295EF70E88B0DC0F7013296AD
:10B09000E491E023EE0EF11CEA0EFB1E1A1509F4F2
:10B0A000ACCF1F5FB4CFE114F10409F445C08C812B
:10B0B0009D810E94D74DA82E6B88BC8879887C0C16
:10B0C0009A899B0D1D2D191B0B2D262D412F672DA8
:10B0D000CE010E94214E882369F1EA0CF11CF7E0B1
:10B0E0006F0E669466946694512E5B0C5E012CE1A3
:10B0F000A20EB11C862C912C1515E1F0072D6701CD
:10B100008C2D8E19861590F4F60184916A817B81CD
:10B110000C8F1D8F1F8E8E8F95014BE3CE010E94E9
:10B12000434EFFEFCF1ADF0A085FEACFE80CF91CA5
:10B130001F5FE2CF888901C080E0DF91CF911F912E
:10B140000F91FF90EF90DF90CF90BF90AF909F90C6
:10B150008F907F906F905F900895CF92DF92EF92E3
:10B16000FF920F931F93CF93DF931F92CDB7DEB75C
:10B170006C01DC01DC96EC90DC97DB96FC90DB97B5
:10B180008C010C5F1F4F5996ED91FC915A97C801A5
:10B1900069831995482F4E0D29816F2DC801E1DE75
:10B1A000F60123AD992787FD9095820F911D83AFFE
:10B1B00081E090E00F90DF91CF911F910F91FF9070
:10B1C000EF90DF90CF900895BF92CF92DF92EF92F1
:10B1D000FF920F931F93CF93DF937C018B0120E0AD
:10B1E00030E0F701E20FF31FE491EE2319F02F5F37
:10B1F0003F4FF7CFF801CF01801B910B41914111D7
:10B20000FACFC4E1D0E0C81BD1093327C217D30756
:10B210001CF492E0C92E02C0CC24C39480919B11EF
:10B2200090E06C2D70E06F5F7F4F0F94A81DB62EDD
:10B2300086E0D82ED60E8091CE11D81650F080918F
:10B24000D01190E02D2D30E02B503109821793075B
:10B2500094F5F12C01151105C1F18AE30E9443D345
:10B2600082E0C8120FC0DB0C8091CE11D81668F1B5
:10B270002091D01130E08D2D90E00B9728173907E1
:10B280001CF423C0FF2009F18C2F880F8C0F880F2E
:10B290008093D111D092D21180E20E9443D3C80191
:10B2A000DF91CF911F910F91FF90EF90DF90CF90A2
:10B2B000BF900C9481D31092D111D092D211C701BA
:10B2C0000E9474D3FF24F394C5CFDF91CF911F91D7
:10B2D0000F91FF90EF90DF90CF90BF9008958091F5
:10B2E000851190918611A0918711B0918811B7FFB7
:10B2F00008C0109285111092861110928711109239
:10B30000881180918D1090918E10A0918F10B09126
:10B310009010409185115091861160918711709124
:10B32000881184179507A607B70744F48093851101
:10B3300090938611A0938711B09388118091B002E9
:10B34000882391F020919110309192108091851175
:10B3500090918611820F931F0E94F27CBC01809114
:10B3600097109091981030DF8091811140912C07B7
:10B37000811106C0442311F18091B0028823F1F0BD
:10B3800080919110909192102091851130918611A9
:10B39000820F931FE0919510F0919610309711F065
:10B3A00091838083442329F0E0912D07F0912E07AB
:10B3B00019958091811181110E940AC28091811199
:10B3C00008958091811181110C940AC260918511B8
:10B3D0007091861180918711909188116115710586
:10B3E0008105910571F10F949F162091EB06309124
:10B3F000EC064091ED065091EE060F94FE169B016F
:10B40000AC016091E50E7091E60E8091E70E90918F
:10B41000E80E0F94CC1A6093E50E7093E60E8093BD
:10B42000E70E9093E80E10928511109286111092FB
:10B4300087111092881183E00E94E0C081E0809320
:10B44000B0028091B002882341F085EE9EE00E9418
:10B45000417CBC0181EF9BE2B7CE08953F924F92B1
:10B460005F926F927F928F929F92AF92BF92CF9294
:10B47000DF92EF92FF920F931F93CF93DF9300D051
:10B4800000D0CDB7DEB78C01362E80918111882394
:10B49000C9F026960FB6F894DEBF0FBECDBFDF9180
:10B4A000CF911F910F91FF90EF90DF90CF90BF90C1
:10B4B000AF909F908F907F906F905F904F903F9054
:10B4C0000C940AC28091851190918611A0918711E8
:10B4D000B0918811892B8A2B8B2B09F492C00E9482
:10B4E0003450932DA4E09A02C00111249E838D83D1
:10B4F000FC01E752F14F408051806280738080915F
:10B50000150281110BC020E030E04AE754E4C3018A
:10B51000B2010F94CC1A6B017C0108C0ED81FE8151
:10B52000EE56FD4FC080D180E280F380809185117E
:10B5300090918611A0918711B091881189839A8387
:10B54000AB83BC83BC01CD010F949F162091EB0609
:10B550003091EC064091ED065091EE060F94FE16E8
:10B560009B01AC01C301B2010F94CC1A4B015C01E9
:10B57000AD81BE81A752B14FBE83AD83FD01608313
:10B5800071838283938389819A81AB81BC81B7FF68
:10B5900013C020E030E04AE754E4C301B2010F9445
:10B5A000CB1A6B017C019B01AC01C501B4010F9466
:10B5B000991687FF18C010C089819A81AB81BC8120
:10B5C000892B8A2B8B2B79F0A7019601C501B40139
:10B5D0000F94F21C18163CF4AD81BE81CD92DD9221
:10B5E000ED92FC921397832D0E94E0C0109285117A
:10B5F00010928611109287111092881181E0809329
:10B60000B0028091B002882309F441C02DEC3CECDB
:10B610004CEC5DE36091EB067091EC068091ED06D9
:10B620009091EE060F94F21C232D332727FD3095C1
:10B6300087FD0AC0C901880F991F880F991F87527B
:10B64000914F0E94417C09C0C901880F991F880F42
:10B65000991F8752914F0E94AC79BC01C801269670
:10B660000FB6F894DEBF0FBECDBFDF91CF911F9113
:10B670000F91FF90EF90DF90CF90BF90AF909F9091
:10B680008F907F906F905F904F903F909DCD2696CA
:10B690000FB6F894DEBF0FBECDBFDF91CF911F91E3
:10B6A0000F91FF90EF90DF90CF90BF90AF909F9061
:10B6B0008F907F906F905F904F903F90089562E0E1
:10B6C0008AEE9BE2CBCE61E083EE9BE2C7CE60E0E8
:10B6D0008CED9BE2C3CE8F929F92AF92BF92CF929E
:10B6E000DF92EF92FF920F931F93CF93DF9300D0DF
:10B6F0001F92CDB7DEB780918111882309F448C02D
:10B700008091AA029091AB02181619060CF03BC06A
:10B710009A8389839E012D5F3F4F44E050E06AE9A0
:10B7200076E0CE0101960E946077EEECFBE4849116
:10B730007F019FEFE91AF90A882321F00E947D48D2
:10B74000F701F5CF40919A0650919B0660919C06B7
:10B7500070919D0687E09BE20E94FEF16091AA0233
:10B760007091AB0286EF9AE20E94C7DFE4EFFAE243
:10B7700084917F019FEFE91AF90A882321F00E9442
:10B780007D48F701F5CF10929F060E940AC2DEC0E5
:10B7900081E080939F068090851190908611A09003
:10B7A0008711B090881181149104A104B10409F4A7
:10B7B00057C0109285111092861110928711109225
:10B7C0008811B401882777FD8095982F0F949F16D4
:10B7D0002091F60E3091F70E4091F80E5091F90E2F
:10B7E0000F94FE1620919A0630919B0640919C067C
:10B7F00050919D060F94CC1A6B017C0120E030E043
:10B8000040E050EC0F94F21C87FD2AC020E030E0AD
:10B8100040EA50E4C701B6010F949916181604F1D6
:10B8200080919906882371F08091CB0E882351F086
:10B830008091990E90919A0E880D991D90939A0E71
:10B840008093990EC0929A06D0929B06E0929C0635
:10B85000F0929D0681E00F94C10E82E08093B002C9
:10B860008091B002882341F08AE996E00E94AC7989
:10B87000BC0183ED9BE2A8DCC0909A06D0909B06A9
:10B88000E0909C06F0909D068090E7069090E80678
:10B89000A090E906B090EA06A5019401C701B6019F
:10B8A0000F9499168823C9F0A5019401C701B60128
:10B8B0000F94F21C18161CF481E090E002C08FEF88
:10B8C0009FEF9093E6068093E506C092E706D0923C
:10B8D000E806E092E906F092EA0664E08091E50667
:10B8E000681B0BEB1BE22CE042E082E40E941AADE5
:10B8F00008EB1BE221E043E064E18CE30E941AAD17
:10B9000008E81BE220E143E06FE285E00E941AAD07
:10B9100008E51BE220E143E06FE28AE50E941AADF0
:10B9200060E38091E506681B0EE31BE22DE042E038
:10B930008EE60E941AAD61E38091E506681B04E281
:10B940001BE22DE042E089E10E941AAD0F900F90BA
:10B950000F900F90DF91CF911F910F91FF90EF907B
:10B96000DF90CF90BF90AF909F908F900895CF922F
:10B97000DF92FF920F931F93CF93DF931F921F923B
:10B98000CDB7DEB7082F162FE091AF11F091B011AF
:10B990008AE991E149835A831995180F4981C42E88
:10B9A0005A81D52EF12CD6012D916D01222341F023
:10B9B000412F602F8AE991E1D4DA080FF80EF3CF16
:10B9C0008F2D0F900F90DF91CF911F910F91FF90CE
:10B9D000DF90CF9008950F931F930F94F70B06EB12
:10B9E00018E220E448E060E080E00E941AAD86E4BE
:10B9F00090E20E94D7D243E853E061E18DE3B7DFE4
:10BA00008BEE9CE10E94D7D24CE853E06CE18EE3D0
:10BA1000AEDF8EE496E10E94D7D24CE953E069E2B2
:10BA20008FE3A5DF8EE496E10E94D7D248EA53E087
:10BA30006EE38EE39CDF4AEA53E06EE383E497DF34
:10BA40000E949DD28111CBCF1F910F9108958091BB
:10BA50008111882321F010929F060C940AC2BBCF5B
:10BA6000CF93DF931F92CDB7DEB78091D3118111B1
:10BA700007C081E08093D3118AE991E10E94474E8B
:10BA800060919C1170919D1119829E012F5F3F4F13
:10BA90004FE08AE991E10E94434E9DDF0F90DF91D4
:10BAA000CF910895DDDFE4E0F1E080818D7F808338
:10BAB0009FB7F894E5E0F1E08081826080839FBFCA
:10BAC000E4E0F1E080818B7F80839FB7F894E5E02C
:10BAD000F1E08081846080839FBFE1E0F1E08081BC
:10BAE0008F7B80839FB7F894E2E0F1E080818064EF
:10BAF00080839FBFE4E0F1E080818E7F80839FB7E9
:10BB0000F894E5E0F1E08081816080839FBF82E06E
:10BB1000809329070E94FDBF109223070895DB013F
:10BB2000833078F494E0899FF0011124EA55F94FAD
:10BB3000AB01662757FD6095762F40835183628362
:10BB40007383813089F018F08230D9F008952FEF97
:10BB500030E00F94C11D20ED37E040E050E00F943D
:10BB6000901AB9018EE219C02FEF30E00F94C11D79
:10BB700020ED37E040E050E00F94901AB9018DE2DB
:10BB80000CC02FEF30E00F94C11D20ED37E040E0F6
:10BB900050E00F94901AB9018CE20C9475D1609129
:10BBA000A6067091A70680E0BADF6091AA067091A0
:10BBB000AB0681E0B4DF6091AE067091AF0682E023
:10BBC000AECF2F923F924F925F926F927F928F9261
:10BBD0009F92AF92BF92CF92DF92EF92FF920F931C
:10BBE0001F93CF93DF93CDB7DEB7C454D1090FB6FF
:10BBF000F894DEBF0FBECDBF4C015B017A01322E3F
:10BC00001C8E1F8E19821C826115710511F410E0C3
:10BC1000AFC0FC0183818111FACFFA0180818F329C
:10BC200061F4CA017C010196F70120812F32D1F322
:10BC3000F50183818250823010F465010BC0618D63
:10BC4000728DCE0101960E9416D8882301F3CE0191
:10BC500001966C018E01045E1F4F280147E3642E9C
:10BC6000712C6C0E7D1E9BE0690E711CFE013196DD
:10BC70002496FFAFEEAF249725960FAF2597212E80
:10BC800037C080E28193E615F705D9F7D70120E0A8
:10BC900097E04A2F3B2F8D9181112DC08FA98032C3
:10BCA00009F4B5CF842F932F7C01FC0120810196EC
:10BCB0002F32D1F3222309F452C021E0AE01495CB6
:10BCC0005F4FB601C8010E9473A7882309F49FCF74
:10BCD000CA14DB0419F0C6010E94F8AA0415150560
:10BCE000B9F125969FAD2597822D6801092F182F50
:10BCF000FE01F796C6CF8F3289F28E3219F0EAE252
:10BD0000F6E10AC09A3009F482CF28E09AE0C1CF68
:10BD10003196381709F47BCF34913111F9CF92174E
:10BD200008F475CF813208F472CF8F3709F46FCFE2
:10BD300031E0320FE7E3F0E0EC0FFD1FE20FF11D01
:10BD40002FE9280F2A3108F480528083232FA1CFB6
:10BD500023969FAD239724968FAD2497C6CF232D8E
:10BD6000AE01495C5F4FB601C4010E9473A7182F52
:10BD7000CE0101960E9452ACCE014C960E9452AC6C
:10BD8000812FCC5BDF4F0FB6F894DEBF0FBECDBF67
:10BD9000DF91CF911F910F91FF90EF90DF90CF90A7
:10BDA000BF90AF909F908F907F906F905F904F90DB
:10BDB0003F902F9008952F923F924F925F926F92F3
:10BDC0007F928F929F92AF92BF92CF92DF92EF922B
:10BDD000FF920F931F93CF93DF93CDB7DEB7C0577A
:10BDE000D1090FB6F894DEBF0FBECDBF7C016B0149
:10BDF0004A012DB73EB7AF963FAF2EAFAF97AD9686
:10BE00001FAEAD9734E0C30ED11C8E01015A1F4FF7
:10BE100067E7662E63E0762E70E4272E312C2C0E19
:10BE20003D1E84E0280E311C4BE552E1BE016F5FE0
:10BE30007F4FC6010E9436D618160CF059C12C85CA
:10BE4000922F9871903109F0CFC08091F7148150F2
:10BE5000823008F4C9C04DB65EB6BE016F5F7F4F39
:10BE6000C8010E9491C281E0F70190819111B4C094
:10BE7000E1E0F0E0D8010D900020E9F7E01BF10BC4
:10BE8000EA0FFB1F31962DB73EB72E1B3F0B0FB6A7
:10BE9000F8943EBF0FBE2DBFEDB7FEB731965F01E0
:10BEA000882319F063EB73E001C0B701C5010F945B
:10BEB000121EB801C5010F94FC1D63EB73E0C501B0
:10BEC0000F94FC1D25961FAE259728961FAE289728
:10BED00024961FAE1EAE249722967FAE6EAE22979A
:10BEE00021E0A801B601C1016CDE81114DC0809135
:10BEF000F714811149C0EEECFBE484919F012F5FA0
:10BF00003F4F882381F0E0962FAFE097E1963FAF57
:10BF1000E1970E947D48E0962FADE097E1963FAD16
:10BF2000E197F901EACFEAE3F6E184919F012F5FFF
:10BF30003F4F811102C0980110C0E0962FAFE097EB
:10BF4000E1963FAFE1970E947D48E0962FADE097E4
:10BF5000E1963FADE197F901E8CFF90181919F01A9
:10BF6000882379F0E0962FAFE097E1963FAFE19715
:10BF70000E947D48E1963FADE197E0962FADE097B6
:10BF8000ECCF8AE00E947D488BE1FE01EC5BFF4F25
:10BF9000DE01959601900D928A95E1F724968EAD7B
:10BFA0009FAD24979CA38BA37AA269A240E050E0A6
:10BFB000BE016F5D7F4FC501FEDECE0181960E94FE
:10BFC00057ACCE01805C9F4F0E9457AC0FB6F894DF
:10BFD0005EBE0FBE4DBE28CF80E001900020E9F785
:10BFE0003197EE19FF0946CF8981882309F480C073
:10BFF000853E09F419CF8E3209F416CF80915B1279
:10C000008E3209F411CF2A7009F00ECF81E0903101
:10C0100009F080E080934D12811108C08985873432
:10C0200009F002CF8A858E3709F4FECE8091F7148D
:10C03000813021F068F08230A9F1F6CE8091F814B9
:10C040009091F91401969093F9148093F814ECCE22
:10C05000BE016F5F7F4F8EE492E10E9491C2570153
:10C06000F50181915F01882319F00E947D48F8CF86
:10C070005EE4A52E52E1B52EF50181915F01882382
:10C0800019F00E947D48F8CF80E20E947D486D8DB6
:10C090007E8D8F8D98A14AE00E94D1DD8AE00E94BA
:10C0A0007D48C2CEBE016F5F7F4F8EE492E10E9459
:10C0B00091C28114910441F06EE472E1C4010F94C5
:10C0C000E91D892B69F414C0AD96FFADAD972F2FF4
:10C0D00030E08091F8149091F9142817390741F055
:10C0E000AD963FADAD973F5FAD963FAFAD979CCE60
:10C0F000AF962EAD3FADAF970FB6F8943EBF0FBED3
:10C100002DBFC059DF4F0FB6F894DEBF0FBECDBFB5
:10C11000DF91CF911F910F91FF90EF90DF90CF9023
:10C12000BF90AF909F908F907F906F905F904F9057
:10C130003F902F900895EF92FF920F931F93CF930C
:10C14000DF93CDB7DEB76F970FB6F894DEBF0FBEA3
:10C15000CDBF7B010EEB12E120EC32E1F80131831F
:10C16000208322E02093F7149093F9148093F8141D
:10C1700040E050E0BA0184EC92E10E94BCD6F801A4
:10C18000808191812BE1FC013496DE0115960190AE
:10C190000D922A95E1F7FC01828193819C838B8328
:10C1A00087E793E09A838983A701BE016F5F7F4F82
:10C1B00082E094E000DECE0101960E9457AC6F96BB
:10C1C0000FB6F894DEBF0FBECDBFDF91CF911F91A8
:10C1D0000F91FF90EF900895CF93DF93CDB7DEB727
:10C1E00027970FB6F894DEBF0FBECDBF0E94C9756A
:10C1F00081113BC080E50E94214C882319F00E94E8
:10C200005E4901C060E06F8383E50E94214C882372
:10C2100019F00E945E4901C06CE06E8384E50E94C3
:10C22000214C882319F00E945E4901C063E06D83B0
:10C2300082E50E94214C882319F00E948E4904C097
:10C2400060E070E080ED90E469837A838B839C8367
:10C250009E012B5F3F4FAE014F5F5F4FBE016A5F94
:10C260007F4FCE0107960E940CEB27960FB6F894ED
:10C27000DEBF0FBECDBFDF91CF9108952F923F92C9
:10C280004F925F926F927F928F929F92AF92BF92E6
:10C29000CF92DF92EF92FF920F931F93CF93DF9392
:10C2A000CDB7DEB768970FB6F894DEBF0FBECDBF2F
:10C2B0009C8B8B8B1B014D8B2E8BFC0160817181C4
:10C2C000828193816D877E878F87988BF101C080F3
:10C2D000D180E280F380C986DA86EB86FC864090C6
:10C2E0005E0450905F04609060047090610420913F
:10C2F0005A0430915B0440915C0450915D040F94AA
:10C30000CB1A4B015C012FE632E143E85AEB0F9464
:10C31000F21C87FD24C022E430E045E253E4C5016D
:10C32000B4010F9499161816D4F0A3019201C70115
:10C33000B6010F94CB1A6B017C0121E338E040EC8D
:10C3400050EC0F94F21C87FD0AC022E430E04FE36A
:10C3500053E4C701B6010F94991618162CF4612CFA
:10C36000712C00EC1FE7CEC2C0900A02D0900B02E5
:10C37000E0900C02F0900D028091F006811107C050
:10C38000809115028093EF0681E08093F006809102
:10C39000160290911702A0911802B0911902809391
:10C3A0000A0290930B02A0930C02B0930D02198223
:10C3B0001A821B821C82AE014F5F5F4FBE01675F16
:10C3C0007F4FCE010D960E9401EB81E00E9417ED98
:10C3D00081111DC20E94345004E010E0812C912C88
:10C3E000A12C61E4B62E412C512C70E2672E71E431
:10C3F000772E60E070E080EF93E40E94A3ED882345
:10C4000009F4C4C0015011090115110509F084C0D7
:10C41000EBE6FCE284918F010F5F1F4F882321F030
:10C420000E947D48F801F6CF60E08CE59CE20E9416
:10C4300082C040E7C42E43E0D42EDE82CD8259E193
:10C44000E52EF12CFA82E982BE016B5F7F4FCE01AF
:10C4500001960E949E981E821D8202E310E01A83BC
:10C460000983BE016B5F7F4FCE0101960E949E98AB
:10C47000DE82CD82FA82E982BE016B5F7F4FCE0100
:10C4800001960E949E981E821D821A830983BE0116
:10C490006B5F7F4FCE0101960E949E98DE82CD8217
:10C4A000FA82E982BE016B5F7F4FCE0101960E9446
:10C4B0009E981E821D821A830983BE016B5F7F4F87
:10C4C000CE0101960E949E9880E090E0A0E0B1E449
:10C4D0008D839E83AF83B88780E090E0A8ECB2E4C0
:10C4E00089839A83AB83BC83BE016B5F7F4FCE0190
:10C4F00001960E9405EB1092E50E1092E60E109246
:10C50000E70E1092E80E0E941A8E0E94E2760E94B8
:10C5100095F78DE49CE2E1C0E4E8FCE284919F01A0
:10C520002F5F3F4F882341F02F8B388F0E947D482B
:10C530002F89388DF901F2CF60E084E49CE20E94FB
:10C5400082C08D829E82AF82B88649825A826B8277
:10C550007C82BE016B5F7F4FCE0101960E9405EB8E
:10C560001A8A19821A821B821C82FCE0F98B1D82B6
:10C570009E012E5E3F4FAE014F5F5F4FBE016F5E6B
:10C580007F4FCE0105960E940CEB33CF80E090E008
:10C59000A0E0B1E48D839E83AF83B88720E030E0D4
:10C5A00040EA50E46091E10E7091E20E8091E30E5A
:10C5B0009091E40E0F94CC1A69837A838B839C83C9
:10C5C000BE016B5F7F4FCE0101960E9405EB04E038
:10C5D00010E0812C912C20E8A22E2FE3B22E412CCA
:10C5E000512C30E2632E31E4732EA2C060E082E170
:10C5F0009CE20E9482C080E7C82E83E0D82EDE82B3
:10C60000CD8299E1E92EF12CFA82E982BE016B5FBD
:10C610007F4FCE0101960E949E981E821D8202E3EA
:10C6200010E01A830983BE016B5F7F4FCE01019634
:10C630000E949E98DE82CD82FA82E982BE016B5F03
:10C640007F4FCE0101960E949E981E821D821A8302
:10C650000983BE016B5F7F4FCE0101960E949E98B9
:10C66000DE82CD82FA82E982BE016B5F7F4FCE010E
:10C6700001960E949E981E821D821A830983BE0124
:10C680006B5F7F4FCE0101960E949E9880E090E004
:10C69000A0E0B1E48D839E83AF83B88780E090E013
:10C6A000A8ECB2E489839A83AB83BC83BE016B5F41
:10C6B0007F4FCE0101960E9405EB1092E50E10927D
:10C6C000E60E1092E70E1092E80E0E941A8E0E945B
:10C6D000E2760E9495F783E09CE20E94C29260E0BD
:10C6E0008AEF9BE20E9482C08D829E82AF82B886D2
:10C6F00049825A826B827C82BE016B5F7F4FCE0182
:10C7000001960E9405EB1A8A19821A821B821C82EA
:10C710008CE0898B1D829E012E5E3F4FAE014F5FE4
:10C720005F4FBE016F5E7F4FCE0105960E940CEBFE
:10C7300060E070E080E792E40E94A3ED882319F1A5
:10C74000015011090115110569F4E1E2FCE284913F
:10C750008F010F5F1F4F882309F448CF0E947D4847
:10C76000F801F5CFEAE3FCE284919F012F5F3F4F90
:10C77000882309F4B4CF2F8B388F0E947D482F89EE
:10C78000388DF901F1CF8090E10E9090E20EA090EB
:10C79000E30EB090E40E2091620430916304409166
:10C7A000640450916504C501B4010F94CB1A209123
:10C7B0009A0630919B0640919C0650919D060F94DD
:10C7C000CC1A3B018C019D8991111CC080E090E046
:10C7D000A0E0B1E489839A83AB83BC8320E030E09E
:10C7E00040EA50E4C501B4010F94CC1A6D837E83F6
:10C7F0008F839887BE016F5F7F4FCE0105960E94A1
:10C8000005EB09C080E00E9417ED882321F0612C20
:10C81000712C00EC1FE78091EF0680931502EE89E2
:10C82000E33008F440C0E7EBFCE284915F019FEF46
:10C83000A91AB90A882321F00E947D48F501F5CF95
:10C84000EB89FC89608171818281938143E00E9440
:10C8500088F1E2EBFCE284915F019FEFA91AB90A2B
:10C86000882321F00E947D48F501F5CFF101608118
:10C8700071818281938143E00E9488F1EDEAFCE2BC
:10C8800084915F019FEFA91AB90A882321F00E94C1
:10C890007D48F501F5CF43E0B301C8010E9488F15E
:10C8A0008AE00E947D48C0920A02D0920B02E09278
:10C8B0000C02F0920D029301A801B301C8010F947C
:10C8C000781D8823F9F060E08EE99CE20E9482C026
:10C8D000E7E9FBE484917F019FEFE91AF90A8823D5
:10C8E00021F00E947D48F701F5CFEEE8FCE284914B
:10C8F0007F019FEFE91AF90A882321F00E947D4801
:10C90000F701F5CFB301C80168960FB6F894DEBF02
:10C910000FBECDBFDF91CF911F910F91FF90EF9090
:10C92000DF90CF90BF90AF909F908F907F906F904F
:10C930005F904F903F902F9008952F923F924F928B
:10C940005F926F927F928F929F92AF92BF92CF929F
:10C95000DF92EF92FF920F931F93CF93DF93CDB7A8
:10C96000DEB7C150D1400FB6F894DEBF0FBECDBFC9
:10C970000E94C97581110C942373FE0131968CE3DA
:10C98000DF011D928A95E9F7C0909906C652DF4FE4
:10C99000C882CA5DD0408AE40E94144B882321F0EB
:10C9A0000E94CBAC0C94237386E50E94214C882313
:10C9B00049F00E945E49CC52DF4F79836883C45DA1
:10C9C000D04006C0CC52DF4F19821882C45DD040DF
:10C9D000CC52DF4F28813981C45DD04025303105EC
:10C9E00070F0ECE8FEE284918F010F5F1F4F882307
:10C9F00011F40C9423730E947D48F801F4CF84E471
:10CA00000E94144B882341F00E947F49C152DF4F9E
:10CA10008883CF5DD04005C0C152DF4F1882CF5D03
:10CA2000D040CC52DF4F48815981C45DD040433063
:10CA300051056CF484E50E94144B882379F00E9420
:10CA40007F49C352DF4F8883CD5DD0400CC051E099
:10CA5000C352DF4F5883CD5DD04005C0C352DF4F76
:10CA60001882CD5DD04088E50E94214C882321F0BA
:10CA70000E945E49162F01C012E089E50E94214CF8
:10CA8000882321F00E945E49062F01C002E080E564
:10CA90000E94214C811107C0CD52DF4F1883C35D26
:10CAA000D040202E08C00E945E49CD52DF4F6883DF
:10CAB000C35DD040262ECD52DF4F8881C35DD0406C
:10CAC000823018F4E7E5FEE204C091E0921568F0C8
:10CAD000F9CF84918F010F5F1F4F882311F40C94BD
:10CAE00023730E947D48F801F4CF83E50E94214C16
:10CAF000882319F00E948E4904C060E070E88BEB37
:10CB000095E420E030E040E752E40F94A81B6093E6
:10CB10001602709317028093180290931902C09026
:10CB20005A04D0905B04E0905C04F0905D048CE4C7
:10CB30000E94214C811108C020E030E0A901C7010A
:10CB4000B6010F94CC1A02C00E948E490F94101C9B
:10CB50006B017C01CA52DF4F79836883C65DD04088
:10CB600080905A0490905B04A0905C04B0905D04A7
:10CB700082E50E94214C811109C020E030E044E2AE
:10CB800053E4C501B4010F94CC1A02C00E948E492F
:10CB90000F94101C4B015C01CD53DF4F79836883E8
:10CBA000C35CD04040905E0450905F04609060048D
:10CBB0007090610486E40E94214C811109C020E03C
:10CBC00030E040EC50E4C301B2010F94CB1A02C034
:10CBD0000E948E490F94101CC954DF4F68837983DB
:10CBE0008A839B83C75BD040C954DF4FA881B9813A
:10CBF000C75BD040C052DF4FB983A883C05ED0402E
:10CC000040905E0450905F046090600470906104F6
:10CC100082E40E94214C811109C020E030E042E210
:10CC200053E4C301B2010F94CC1A02C00E948E4992
:10CC30000F94101CC554DF4F688379838A839B83CC
:10CC4000CB5BD040C554DF4FE881F981CB5BD0404E
:10CC5000C553DF4FF983E883CB5CD040B60188270A
:10CC600077FD8095982F0F949F16CA51DF4F6883E8
:10CC700079838A839B83C65ED04040905A0450904B
:10CC80005B0460905C0470905D0420E030E0A901DA
:10CC9000C301B2010F94CC1A9B01AC01CA51DF4F02
:10CCA000688179818A819B81C65ED0400F949916F4
:10CCB00087FD13C021E0C4010997CA52DF4F4881A4
:10CCC0005981C65DD040481759070CF420E0C15483
:10CCD000DF4F2883CF5BD04006C051E0C154DF4F07
:10CCE0005883CF5BD040B401882777FD8095982F7B
:10CCF0000F949F164B015C0120E030E045E253E4C5
:10CD0000C301B2010F94CC1A9B01AC01C501B4015F
:10CD10000F94F21C181684F089E0C80ED11C81E033
:10CD2000CD53DF4FE880F980C35CD040CE14DF04E0
:10CD30000CF480E0382E02C033243394C954DF4F02
:10CD400028813981C75BD040B901882777FD80955C
:10CD5000982F0F949F162B013C01C0905E04D09039
:10CD60005F04E0906004F090610420E030E040EC6B
:10CD700050E4C701B6010F94CB1A9B01AC01C3016B
:10CD8000B2010F94991601E087FD11C0C554DF4F21
:10CD900088819981CB5BD0400997C052DF4F488191
:10CDA0005981C05ED040481759070CF400E0C554C3
:10CDB000DF4FA881B981CB5BD040BD01882777FDCB
:10CDC0008095982F0F949F164B015C0120E030E076
:10CDD0004FE353E4C701B6010F94CC1A9B01AC0199
:10CDE000C501B4010F94F21C18169CF0C954DF4F12
:10CDF00088819981C75BD040099611E0C553DF4F08
:10CE0000C880D980CB5CD0408C159D051CF410E007
:10CE100001C011E0C154DF4FD880CF5BD040D110AA
:10CE20000CC0332029F088E49EE20E9484480BC0A5
:10CE3000011109C011110DC016C080E59EE20E94CB
:10CE400084483110F0CF002321F080E49EE20E945C
:10CE50008448112311F40C94237389E39EE20E9409
:10CE600084480C942373CC52DF4FE880F980C45D72
:10CE7000D040EF28F9F0E2E2FEE284918F010F5FEB
:10CE80001F4F882321F00E947D48F801F6CFC15240
:10CE9000DF4FF880CF5DD040FF2061F0E9E0FEE297
:10CEA00084918F010F5F1F4F882321F00E947D48DE
:10CEB000F801F6CF0E9495F710929906C152DF4F04
:10CEC000C880CF5DD040C1100AC00E94E2C788EF81
:10CED00096E00E94C0BD0E94B54D0E94FFFF81E018
:10CEE0000E9417ED882349F0C652DF4FD880CA5DF3
:10CEF000D040D09299060C9423730E94575085E439
:10CF00000E94144B882341F00E947F49C451DF4F97
:10CF10008883CC5ED04005C0C451DF4F1882CC5E00
:10CF2000D040CD52DF4FF880C35DD040EF2CF12CC4
:10CF3000C251DF4FF982E882CE5ED040C22CD12CA4
:10CF4000C051DF4FD982C882C05FD040CD52DF4F81
:10CF5000F880C35DD040F29C70011124C552DF4FB0
:10CF6000F982E882CB5DD040CD52DF4F2881C35D8E
:10CF7000D0402170C153DF4F2883CF5CD040EE0CEE
:10CF8000FF1CC651DF4FF982E882CA5ED0402CEF09
:10CF9000A70124036001259FD00C1124CC50DF4F42
:10CFA000D982C882C45FD040C552DF4FE880F98083
:10CFB000CB5DD040EE0CFF1CEE0CFF1CCE50DF4FC3
:10CFC000F982E882C25FD040C554DF4F19821882CF
:10CFD000CB5BD0402FEF3FEFC954DF4F398328831D
:10CFE000C75BD040CD53DF4FC880D980C35CD040F1
:10CFF000CA52DF4FE880F980C65DD040CE18DF0806
:10D00000CD53DF4FD982C882C35CD040C553DF4FB8
:10D01000C880D980CB5CD040C052DF4FE880F98017
:10D02000C05ED040CE18DF08C553DF4FD982C8821A
:10D03000CB5CD040C953DF4F288139814A815B8165
:10D04000C75CD040CA01B9010F94781D811120C37B
:10D05000C153DF4FC880CF5CD040CC2069F0CA52AA
:10D06000DF4F2882C65DD04021E0C052DF4F2883C9
:10D07000C05ED040312C0FC033243A94320C3FEFC5
:10D08000C052DF4F3883C05ED0404FEFCA52DF4FEF
:10D090004883C65DD04081E0C153DF4FC880CF5C7C
:10D0A000D040C826C153DF4FC882CF5CD0409E011C
:10D0B000235C3F4FC954DF4F88819981C75BD040C3
:10D0C0000196C651DF4FC880D980CA5ED0408C0D12
:10D0D0009D1D880F991F880F991F280F391FC15454
:10D0E000DF4F39832883CF5BD040C251DF4F288187
:10D0F0003981CE5ED04021503109CA50DF4F39838B
:10D100002883C65FD040C554DF4FC880D980CB5B31
:10D11000D040EE24D7FCE094FE2CC850DF4FC882EC
:10D12000D982EA82FB82C85FD040C051DF4F28819C
:10D130003981C05FD04021503109C450DF4F39835D
:10D140002883CC5FD040C554DF4FC880D980CB5BEB
:10D15000D040CC0CDD1CC250DF4FD982C882CE5FDC
:10D16000D040CA52DF4FD880C65DD0403D1409F48C
:10D1700079C2CD53DF4F88819981C35CD040CA50BA
:10D18000DF4F68817981C65FD0400F94A81D882742
:10D1900077FD8095982F0F949F166B017C01C850E6
:10D1A000DF4F688179818A819B81C85FD0400F946D
:10D1B0009F169B01AC01C701B6010F94FE169B019F
:10D1C000AC01CA51DF4F688179818A819B81C65E3B
:10D1D000D0400F94CC1A4B015C01C553DF4F8881BE
:10D1E0009981CB5CD040C450DF4F68817981CC5F9E
:10D1F000D0400F94A81D882777FD8095982F0F9415
:10D200009F166B017C01632D772767FD7095872F33
:10D21000972F0F949F169B01AC01C701B6010F9485
:10D22000FE169B01AC01C301B2010F94CC1A6B0135
:10D230007C0120E030E0A901C501B4010F949916EA
:10D2400087FF04C020E030E0A90104C020E030E006
:10D2500040E05FE3C501B4010F94CC1A0F94411C68
:10D26000C355DF4F688379838A839B83CD5AD0402F
:10D2700020E030E0A901C701B6010F94991687FF9D
:10D2800004C020E030E0A90104C020E030E040E02C
:10D290005FE3C701B6010F94CC1A0F94411CC75528
:10D2A000DF4F688379838A839B83C95AD040C954EE
:10D2B000DF4F28813981C75BD0402F5F3F4FC95472
:10D2C000DF4F39832883C75BD040C250DF4FE881EE
:10D2D000F981CE5FD040E30DF11D37FCFA95EE0FDA
:10D2E000FF1F41EA50E04C0F5D1FE40FF51F318333
:10D2F0002083CC52DF4F2881C45DD040C451DF4F22
:10D300004881CC5ED040BE0167557F4FCE0183552A
:10D310009F4F0E943E61C953DF4F688379838A83A0
:10D320009B83C75CD0409B01AC010F94781D882380
:10D3300041F0C652DF4FC880CA5DD040C092990606
:10D3400091C1C953DF4F288139814A815B81C75C14
:10D35000D040CE51DF4F688179818A819B81C25E46
:10D36000D0400F94CC1ACE51DF4F688379838A83E3
:10D370009B83C25ED040C954DF4FE881F981C75B0F
:10D38000D040EE0FFF1FEE0FFF1F4DE6E42EF12CF5
:10D39000EC0EFD1EEE0DFF1DC953DF4FC880D98076
:10D3A000EA80FB80C75CD040C082D182E282F382F7
:10D3B000C355DF4F88809980AA80BB80CD5AD0406A
:10D3C000C154DF4FE881F981CF5BD040CC50DF4FB3
:10D3D000E880F980C45FD040EE0DFF1D808291820D
:10D3E000A282B382C755DF4FC880D980EA80FB8014
:10D3F000C95AD040CE50DF4F28813981C25FD0401A
:10D40000E20FF31FC082D182E282F382C154DF4F68
:10D41000E881F981CF5BD04080E090E0A0E8BFE3F5
:10D4200081939193A193B193C154DF4FF983E88322
:10D43000CF5BD040A501940169817A818B819C8169
:10D440000F94CC1A69837A838B839C83A7019601FE
:10D450006D817E818F8198850F94CC1A6D837E8338
:10D460008F839887C953DF4F288139814A815B8137
:10D47000C75CD04069857A858B859C850F94CC1AD2
:10D4800069877A878B879C87A5019401C501B401C0
:10D490000F94FE169B01AC016D857E858F85988962
:10D4A0000F94CC1A6D877E878F87988BA701960182
:10D4B000C701B6010F94FE169B01AC0169897A89F8
:10D4C0008B899C890F94CC1A698B7A8B8B8B9C8B64
:10D4D000C953DF4F288139814A815B81C75CD040C5
:10D4E000CA01B9010F94FE169B01AC016D897E89BA
:10D4F0008F89988D0F94CC1A6D8B7E8B8F8B988F24
:10D50000A7019601C501B4010F94FE169B01AC0161
:10D51000698D7A8D8B8D9C8D0F94CC1A698F7A8F43
:10D520008B8F9C8FC953DF4F288139814A815B8162
:10D53000C75CD040C501B4010F94FE169B01AC013D
:10D540006D8D7E8D8F8D98A10F94CC1A6D8F7E8FEF
:10D550008F8F98A3C953DF4F288139814A815B811E
:10D56000C75CD040C701B6010F94FE169B01AC0109
:10D5700069A17AA18BA19CA10F94CC1A69A37AA36B
:10D580008BA39CA3E894B7F81DA10EA1FFA1C652DE
:10D59000DF4FF883CA5DD04028A5C351DF4F2883F1
:10D5A000CD5ED040212F302F4F2FC351DF4F5881F8
:10D5B000CD5ED040C501B4010F94F21C18162CF4B6
:10D5C000182D092D3A2D2B2D0AC0C652DF4F388158
:10D5D000CA5DD040C351DF4F2881CD5ED040812F3E
:10D5E000902FA32FB22F8DA39EA3AFA3B8A7460160
:10D5F0005701E894B7F819A50AA5FBA4ECA4212FBC
:10D60000302F4F2D5E2DC501B4010F94F21C18165A
:10D6100024F4182D092DFA2CEB2C812F902FAF2DEF
:10D62000BE2D89A79AA7ABA7BCA720E030E040E8B1
:10D630005FE369AD7AAD8BAD9CAD0F94CC1A69AF49
:10D640007AAF8BAF9CAF80E00F94C104C052DF4F24
:10D65000C880C05ED0403C0CC652DF4F1882CA5D05
:10D66000D0407FCDC554DF4F28813981CB5BD0407E
:10D670002F5F3F4FC554DF4F39832883CB5BD040AA
:10D68000CD52DF4FC880C35DD0402C1508F4D2CCFA
:10D6900080E00E9417ED882341F0C652DF4FD8800A
:10D6A000CA5DD040D0929906C5C7C953DF4F2881C3
:10D6B00039814A815B81C75CD040CA01B9010F94AE
:10D6C000781D8111B7C789AC9AACABACBCAC20E07B
:10D6D00030E0A901C501B4010F949916882309F41B
:10D6E00008C2A501940169817A818B819C810F9484
:10D6F000A81BC954DF4F688379838A839B83C75BE8
:10D70000D04069837A838B839C83A50194016D81CA
:10D710007E818F8198850F94A81BC554DF4F688345
:10D7200079838A839B83CB5BD0406D837E838F8399
:10D730009887A501940169857A858B859C850F94CE
:10D74000A81BC154DF4F688379838A839B83CF5B97
:10D75000D04069877A878B879C87A50194016D8566
:10D760007E858F8598890F94A81B6B017C01C95415
:10D77000DF4F288139814A815B81C75BD040CA0174
:10D78000B9010F94FE169B01AC01C701B6010F94BD
:10D79000CB1AC553DF4F688379838A839B83CB5C25
:10D7A000D0406D877E878F87988BA501940169890A
:10D7B0007A898B899C890F94A81B6B017C01C554C5
:10D7C000DF4F288139814A815B81CB5BD040CA0120
:10D7D000B9010F94FE169B01AC01C701B6010F946D
:10D7E000CB1AC153DF4F688379838A839B83CF5CD5
:10D7F000D040698B7A8B8B8B9C8BA50194016D89B2
:10D800007E898F89988D0F94A81B6B017C01C15470
:10D81000DF4F288139814A815B81CF5BD040CA01CB
:10D82000B9010F94FE169B01AC01C701B6010F941C
:10D83000CB1A6D8B7E8B8F8B988FA5019401698D90
:10D840007A8D8B8D9C8D0F94A81B6B017C01C55428
:10D85000DF4F288139814A815B81CB5BD040C9543D
:10D86000DF4F688179818A819B81C75BD0400F94AB
:10D87000FE169B01AC01C701B6010F94CB1ACD5324
:10D88000DF4F688379838A839B83C35CD040698F31
:10D890007A8F8B8F9C8FA501940169A17AA18BA1AE
:10D8A0009CA10F94A81B6B017C01C154DF4F288100
:10D8B00039814A815B81CF5BD040C554DF4F68819D
:10D8C00079818A819B81CB5BD0400F94FE169B01AE
:10D8D000AC01C701B6010F94CB1A6B017C0169A39F
:10D8E0007AA38BA39CA3A50194016D8D7E8D8F8D52
:10D8F00098A10F94A81B4B015C01C154DF4F2881F4
:10D9000039814A815B81CF5BD040C954DF4F688148
:10D9100079818A819B81C75BD0400F94FE169B0161
:10D92000AC01C501B4010F94CB1A4B015C016D8FA2
:10D930007E8F8F8F98A3C153DF4F288139814A8111
:10D940005B81CF5CD040C553DF4F688179818A818C
:10D950009B81CB5CD0400F94FE162B013C01CD5334
:10D96000DF4F288139814A815B81C35CD040CA0185
:10D97000B9010F94FE169B01AC01C301B2010F94D3
:10D98000CB1ACA52DF4F688379838A839B83C65D33
:10D99000D0402B013C01E89477F829A53AA54BA586
:10D9A0005CA56DA17EA18FA198A50F94CC1A2FEF35
:10D9B00036EE4BED5EE20F94FE169B01AC01C30107
:10D9C000B2010F94991618160CF093C0CD53DF4F87
:10D9D000288139814A815B81C35CD040C701B6018F
:10D9E0000F94FE162B013C01C153DF4F2881398172
:10D9F0004A815B81CF5CD040C501B4010F94FE1613
:10DA00009B01AC01C301B2010F94CB1ACA52DF4F84
:10DA1000288139814A815B81C65DD0400F94A81B63
:10DA20002B013C016DA77EA78FA798ABCD53DF4F8D
:10DA3000288139814A815B81C35CD040C501B40132
:10DA40000F94FE164B015C01C553DF4F28813981CD
:10DA50004A815B81CB5CD040C701B6010F94FE16B2
:10DA60009B01AC01C501B4010F94CB1ACA52DF4F20
:10DA7000288139814A815B81C65DD0400F94A81B03
:10DA80006B017C0169AB7AAB8BAB9CABC954DF4FAC
:10DA9000288139814A815B81C75BD040C301B201D3
:10DAA0000F94FE169B01AC01C154DF4F6881798150
:10DAB0008A819B81CF5BD0400F94CC1A4B015C01D3
:10DAC000C554DF4F288139814A815B81CB5BD040CF
:10DAD000C701B6010F94FE169B01AC01C501B4014C
:10DAE0000F94CC1ADC01CB01B0588DAB9EABAFAB21
:10DAF000B8AFCDA4DEA4EFA4F8A82601370177FAC9
:10DB0000709477F8709489A89AA8ABA8BCA82DA99E
:10DB10003EA94FA958ADC954DF4F288339834A83A2
:10DB20005B83C75BD040C552DF4F48815981CB5DD5
:10DB3000D040BA01882777FD8095982F0F949F16C3
:10DB40009B01AC01CE51DF4F688179818A819B8135
:10DB5000C25ED0400F94A81BC153DF4F6883798306
:10DB60008A839B83CF5CD040CC52DF4F88819981E0
:10DB7000C45DD040892B09F460C0E3EFFDE28491DD
:10DB80008F010F5F1F4F882321F00E947D48F8010D
:10DB9000F6CF48E0C301B2010E9488F1EEEEFDE24B
:10DBA00084918F010F5F1F4F882321F00E947D48D1
:10DBB000F801F6CF48E0C501B40190580E9488F101
:10DBC000E9EEFDE284918F010F5F1F4F882321F062
:10DBD0000E947D48F801F6CFC954DF4F68817981F2
:10DBE0008A819B81C75BD040905848E00E9488F1B1
:10DBF0008AE00E947D48CC52DF4FA881B981C45D84
:10DC0000D0401397D4F0E0EDFDE284918F010F5FD7
:10DC10001F4F882321F00E947D48F801F6CF48E08D
:10DC2000C153DF4F688179818A819B81CF5CD0406D
:10DC30000E9488F18AE00E947D48C152DF4FB8817E
:10DC4000CF5DD040B111D1C1CB56DF4FC882D98250
:10DC5000EA82FB82C559D040C756DF4F888299823D
:10DC6000AA82BB82C959D040C12CD12C20E8E22E17
:10DC70002FE3F22EC356DF4FC882D982EA82FB829D
:10DC8000CD59D040CE018B569F4F0E94347EC7574E
:10DC9000DF4FC882D982EA82FB82C958D040C3577D
:10DCA000DF4F188219821A821B82CD58D040CF567E
:10DCB000DF4F488259826A827B82C159D040CE01AF
:10DCC00087579F4F0E94347ECB56DF4FC880D98044
:10DCD000EA80FB80C559D040C954DF4FC882D98241
:10DCE000EA82FB82C75BD040C756DF4F488059802D
:10DCF0006A807B80C959D040C356DF4F88809980A5
:10DD0000AA80BB80CD59D040C757DF4FC880D9808B
:10DD1000EA80FB80C958D040C554DF4FC882D98201
:10DD2000EA82FB82CB5BD040C357DF4FC880D980EB
:10DD3000EA80FB80CD58D040C154DF4FC882D982E1
:10DD4000EA82FB82CF5BD040CF56DF4FC880D980BC
:10DD5000EA80FB80C159D040A7019601C301B201FE
:10DD60000F94FE16CD53DF4F688379838A839B839C
:10DD7000C35CD040C154DF4F288139814A815B8127
:10DD8000CF5BD040C501B4010F94FE169B01AC01DE
:10DD9000CD53DF4F688179818A819B81C35CD040FC
:10DDA0000F94CB1AC358DF4F688379838A839B8390
:10DDB000CD57D040C554DF4F288139814A815B81DE
:10DDC000CB5BD040C501B4010F94FE164B015C0142
:10DDD000A7019601C954DF4F688179818A819B81AF
:10DDE000C75BD0400F94FE169B01AC01C501B40186
:10DDF0000F94CB1ACF57DF4F688379838A839B8335
:10DE0000C158D040C154DF4F288139814A815B819C
:10DE1000CF5BD040C954DF4F688179818A819B8173
:10DE2000C75BD0400F94FE166B017C01C554DF4FD9
:10DE3000288139814A815B81CB5BD040C301B2012B
:10DE40000F94FE169B01AC01C701B6010F94CB1ACB
:10DE5000CB57DF4F688379838A839B83C558D04033
:10DE6000CE0183589F4F0E94347EC757DF4F888072
:10DE70009980AA80BB80C958D040C357DF4FC88063
:10DE8000D980EA80FB80CD58D040CF56DF4F488004
:10DE900059806A807B80C159D040C358DF4F2881A8
:10DEA00039814A815B81CD57D040C954DF4F2883E7
:10DEB00039834A835B83C75BD040CF57DF4F88816C
:10DEC0009981AA81BB81C158D040C554DF4F888356
:10DED0009983AA83BB83CB5BD040CB57DF4F28818C
:10DEE00039814A815B81C558D040C154DF4F2883B6
:10DEF00039834A835B83CF5BD040CB56DF4F0881A9
:10DF000019812A813B81C559D040C756DF4F4881CE
:10DF100059816A817B81C959D040C356DF4F8881BE
:10DF20009981AA81BB81CD59D0408092D411909221
:10DF3000D511A092D611B092D711C092D811D0921B
:10DF4000D911E092DA11F092DB114092DC1150927B
:10DF5000DD116092DE117092DF11C954DF4FC8806D
:10DF6000D980EA80FB80C75BD040C092E011D0929C
:10DF7000E111E092E211F092E311C554DF4FC88045
:10DF8000D980EA80FB80CB5BD040C092E411D09274
:10DF9000E511E092E611F092E711C154DF4FC8801D
:10DFA000D980EA80FB80CF5BD040C092E811D0924C
:10DFB000E911E092EA11F092EB110093EC11109349
:10DFC000ED112093EE113093EF114093F011509327
:10DFD000F1116093F2117093F3118093F411909307
:10DFE000F511A093F611B093F711C352DF4FD8800B
:10DFF000CD5DD040DD2009F47EC2EDE0FDE28491EC
:10E000008F010F5F1F4F882321F00E947D48F80188
:10E01000F6CF44244A94420C542CC554DF4F188246
:10E02000CB5BD04020ECC154DF4F2883CF5BD04086
:10E0300039E7CD53DF4F3883C35CD04044E4C55348
:10E04000DF4F4883CB5CD040CE018B569F4FCF54DF
:10E05000DF4F99838883C15BD040DE01A757BF4F54
:10E06000CD54DF4FB983A883C35BD040FE01E35892
:10E07000FF4FCB54DF4FF983E883C55BD04057FC9B
:10E0800029C1652C660C770811EAE12EF12CEC0E03
:10E09000FD1E6E0C7F1C212C312CC954DF4F1882C1
:10E0A000C75BD040F301E20DF31DC080D180C352A5
:10E0B000DF4FD982C882CD5DD0408601000F111F8D
:10E0C000000F111FEDE6F0E0EC0FFD1FE00FF11F58
:10E0D00080809180A280B380C153DF4F2881398135
:10E0E0004A815B81CF5CD040C501B4010F94CB1A4B
:10E0F0006B017C01E1E0F0E0EC0FFD1FE00FF11F90
:10E1000084AD95ADA6ADB7ADCB56DF4F888399836F
:10E11000AA83BB83C559D040C352DF4FE881F98140
:10E12000CD5DD040C552DF4F28813981CB5DD040D5
:10E13000E20FF31FEE0FFF1FEE0FFF1F41E050E055
:10E140004C0F5D1FE40FF51F84AD95ADA6ADB7ADC7
:10E15000C757DF4F88839983AA83BB83C958D040B0
:10E16000C358DF4F188219821A821B82CD57D040C4
:10E17000CA54DF4F5881C65BD0405F93CB54DF4F0A
:10E180008881C55BD0408F93CC54DF4F9881C45BAE
:10E19000D0409F93CD54DF4FA881C35BD040AF9355
:10E1A000CE54DF4FB881C25BD040BF93CF54DF4F16
:10E1B000E881C15BD040EF932DB73EB724523109BF
:10E1C0000FB6F8943EBF0FBE2DBFADB7BEB71196C8
:10E1D000E4EDF1E184E201900D928A95E1F70E946D
:10E1E000DBBCC358DF4F288139814A815B81CD5721
:10E1F000D040C501B4010F94CB1A5B018C010FB65E
:10E20000F894DEBF0FBECDBF9B01AC01C554DF4FFC
:10E210006881CB5BD040C154DF4F7881CF5BD04069
:10E22000CD53DF4F8881C35CD040C553DF4F988109
:10E23000CB5CD0400F94F21C1816A4F4C554DF4FE9
:10E24000A882CB5BD040C154DF4FB882CF5BD040B7
:10E25000CD53DF4F0883C35CD040C553DF4F1883D5
:10E26000CB5CD04020E030E0A901C701B6010F949B
:10E27000F21C87FD0CC0EAE0FDE284918F010F5F84
:10E280001F4F882339F00E947D48F801F6CF80E2C5
:10E290000E947D4845E0C701B6010E9488F1C9543B
:10E2A000DF4F5881C75BD0405F5FC954DF4F588351
:10E2B000C75BD04084E0280E311CCD52DF4FC880B0
:10E2C000C35DD0405C1508F4EDCE8AE00E947D4825
:10E2D0005A94D5CE8AE00E947D48CC52DF4F2881E7
:10E2E0003981C45DD0402430310509F004C1E1EE2C
:10E2F000FCE284918F010F5F1F4F811112C0AE01AC
:10E300004B565F4FCF54DF4F59834883C15BD0409A
:10E310001E0159E8250E311C3E018DE7680E711C67
:10E320001AC00E947D48F801E4CF80E20E947D4837
:10E3300045E0C501B4010E9488F1D3940C5F1F4FE2
:10E34000CD52DF4FF881C35DD040DF16A8F08AE0E0
:10E350000E947D484A9447FCCAC0E42CEE0CFF089A
:10E36000E1EACE2ED12CCC0EDD1EEC0CFD1C00E023
:10E3700010E0D12CF4E2CF2EF701E00FF11F019055
:10E38000F081E02D5F01AA0CBB1CAA0CBB1CA1E014
:10E39000B0E0AC0FBD1FAA0DBB1DDC968D919D9109
:10E3A0000D90BC91A02DCB56DF4F88839983AA8313
:10E3B000BB83C559D040C552DF4FA881B981CB5D21
:10E3C000D040EA0FFB1FEE0FFF1FEE0FFF1F21E0F3
:10E3D00030E02C0F3D1FE20FF31F84AD95ADA6ADCD
:10E3E000B7ADF10180839183A283B383D3011D92E2
:10E3F0001D921D921C9213977F926F923F922F92C3
:10E40000CE54DF4FB881C25BD040BF93CF54DF4FB3
:10E41000E881C15BD040EF932DB73EB7245231095C
:10E420000FB6F8943EBF0FBE2DBFADB7BEB7119665
:10E43000E4EDF1E18C2D01900D928A95E1F70E94B7
:10E44000DBBCEDE6F0E0EC0FFD1FEA0DFB1DD30198
:10E450002D913D914D915C9160817181828193817B
:10E460000F94CB1AC554DF4F2881CB5BD040C154E9
:10E47000DF4F3881CF5BD040CD53DF4F4881C35C45
:10E48000D040C553DF4F5881CB5CD0400F94CB1A9E
:10E490004B015C010FB6F894DEBF0FBECDBF20E08C
:10E4A00030E0A9010F94F21C87FD3FCFEEEDFCE2B6
:10E4B00084919F012F5F3F4F882309F439CFC050CB
:10E4C000DF4F2883C050D140CF5FDE4F3883C1502B
:10E4D000D1400E947D48C050DF4F2881C050D140BC
:10E4E000CF5FDE4F3881C150D140F901E1CF8AE0E2
:10E4F0000E947D4808C0CC52DF4FE880F980C45D9F
:10E50000D040EF2821F08FEB9CE20F944B0FC152CB
:10E51000DF4FF880CF5DD040F11085C08CE0E9ED91
:10E52000FEE0DE01A358BF4F01900D928A95E1F7FE
:10E5300081E080939906CE0183589F4F0E94C0BD11
:10E54000C355DF4F288139814A815B81CD5AD04044
:10E550006091D90E7091DA0E8091DB0E9091DC0EF5
:10E560000F94CB1A6B017C012DEB37E346E855EB9A
:10E570000F94F21C87FD4BC02DEB37E346E855E3C3
:10E58000C701B6010F94991618160CF440C0C75570
:10E59000DF4F288139814A815B81C95AD04060911F
:10E5A000DD0E7091DE0E8091DF0E9091E00E0F94E3
:10E5B000CB1A6B017C012DEB37E346E855EB0F944A
:10E5C000F21C87FD24C02DEB37E346E855E3C70175
:10E5D000B6010F9499161816D4F0C953DF4F28814D
:10E5E00039814A815B81C75CD0406091E10E7091B6
:10E5F000E20E8091E30E9091E40E0F94CB1ACB576C
:10E60000DF4F688379838A839B83C558D0408CE031
:10E61000FE01E358FF4FA9EDBEE001900D928A95EF
:10E62000E1F781E005C0C652DF4F8881CA5DD04066
:10E63000809399060E943E500F948B0F809199060B
:10E6400081110E94FFFFCF5FDE4F0FB6F894DEBF4F
:10E650000FBECDBFDF91CF911F910F91FF90EF9033
:10E66000DF90CF90BF90AF909F908F907F906F90F2
:10E670005F904F903F902F900895FB014081FC01E7
:10E6800020813181342768E0A901440F551F37FDEF
:10E6900007C09A016150C1F7FC01318320830895BE
:10E6A0009A01F1E22F27F0E13F27F4CF0F931F9358
:10E6B000CF93DF93EC0189018C81833039F0E9E05D
:10E6C000440F551F661F771FEA95D1F79A01AB01DA
:10E6D00068E1CE010E94694F882311F086E034C0C2
:10E6E0008EEF8EBD80E090E00DB407FEFDCFF80107
:10E6F000E80FF91F20812EBD0DB407FEFDCF21814B
:10E700002EBD0296811522E0920771F70DB407FE27
:10E71000FDCF8FEF0E9471488FEF0E9471480E94D9
:10E7200076488B838F71853031F083E18983CE0108
:10E730000E94414F0AC068E572E0CE010E94514F2D
:10E74000182F811107C087E18983CE010E94414FB4
:10E7500010E012C020E030E0A9016DE0CE010E947F
:10E76000694F811104C00E947648882311F086E128
:10E77000EBCFCE010E94414F812FDF91CF911F91AE
:10E780000F910895CF93809191078823A9F140912B
:10E7900092075091930760919407709195072AE62C
:10E7A00034E080918F079091900780DFC82F8823F5
:10E7B00021F14091B70E5091B80E6091B90E709151
:10E7C000BA0E411551056105710589F02AE634E05C
:10E7D00080918F079091900769DF882359F01092FC
:10E7E000B70E1092B80E1092B90E1092BA0E109287
:10E7F00091078C2FC82F01C0C1E08C2FCF910895B5
:10E80000EF92FF920F931F93CF93DF93EC01890157
:10E810008C81833039F0F9E0440F551F661F771F54
:10E82000FA95D1F79A01AB0161E1CE010E94694FDF
:10E83000882331F084E08983CE010E94414F41C09A
:10E840000E94454F7B010E9476488B838F3F49F49D
:10E850000E94454F6E197F096D327140A0F381E12E
:10E8600003C08E3F49F08FE08983CE010E94414F63
:10E870008FEF0E94714825C08FEF8EBDF80180E0B8
:10E8800090E02FEF0DB407FEFDCF3EB531932EBDC6
:10E8900001968F3F31E09307A9F70DB407FEFDCF36
:10E8A0008EB5F801E150FE4F80830E9476480E94A9
:10E8B0007648CE010E94414F8FEF0E94714881E05F
:10E8C00001C080E0DF91CF911F910F91FF90EF90F9
:10E8D0000895CF92DF92EF92FF92CF936B017C016C
:10E8E000C42F8091920790919307A0919407B091C3
:10E8F00095078C159D05AE05BF05C1F043DF81115D
:10E9000002C080E017C02AE634E0B701A60180917A
:10E910008F079091900774DF882399F3C092920734
:10E92000D0929307E0929407F092950781E0C1118D
:10E9300080939107CF91FF90EF90DF90CF90089553
:10E940008F929F92AF92BF92CF92DF92EF92FF92FF
:10E950000F931F93CF93DF93EC016A017B01890131
:10E9600089859A85AB85BC850196A11DB11D84174B
:10E970009507A607B70710F480E054C08F8980314F
:10E9800029F49927872F762F652F0BC08032A1F7A6
:10E99000CB01BA0127E096958795779567952A95DB
:10E9A000D1F78B889C88AD88BE88680D791D8A1D3B
:10E9B0009B1D8090920790909307A0909407B09031
:10E9C0009507681579058A059B0581F48F89803143
:10E9D00091F4DD24EE24FF24F601EE0FFF1FE6592B
:10E9E000FB4F80819181A0E0B0E016C040E071DF74
:10E9F0008111ECCFC1CFE894C7F8DD24EE24FF24C9
:10EA0000F601EE0FFF1FEE0FFF1FE659FB4F80814F
:10EA10009181A281B381BF70F80180839183A28329
:10EA2000B38381E0DF91CF911F910F91FF90EF9021
:10EA3000DF90CF90BF90AF909F908F9008954F92AE
:10EA40005F926F927F928F929F92AF92BF92CF927E
:10EA5000DF92EF92FF920F931F93CF93DF93EC011E
:10EA60004A015B01280139014230510561057105F8
:10EA700008F462C049855A856B857C854F5F5F4F7E
:10EA80006F4F7F4F481559056A057B0508F454C040
:10EA90008F89803129F4FF24EB2CDA2CC92C0CC08F
:10EAA000803209F049C07501640167E0F694E7948B
:10EAB000D794C7946A95D1F74B895C896D897E8913
:10EAC000C40ED51EE61EF71E41E0C701B60101DFE8
:10EAD000882391F19F89903159F49924AA24BB2469
:10EAE000F401EE0FFF1FE659FB4F5182408210C028
:10EAF000E89487F89924AA24BB24F401EE0FFF1FA1
:10EB0000EE0FFF1FE659FB4F4082518262827382F3
:10EB10009A89923090F04D815E816F8178854C0D9D
:10EB20005D1D6E1D7F1D4093B70E5093B80E609310
:10EB3000B90E7093BA0E01C080E0DF91CF911F91A2
:10EB40000F91FF90EF90DF90CF90BF90AF909F908C
:10EB50008F907F906F905F904F900895CF93DF9349
:10EB6000CDB7DEB78091B206811110C09E01275F3C
:10EB70003F4F4F81588562E470E08FE492E00F943C
:10EB800061160E9453C083E08093B002DF91CF9161
:10EB90000895FF920F931F93CF93DF93C0915F0768
:10EBA00081E0C827D0916007D827F0906107F82648
:10EBB000C11102C0DD2319F0EEECFBE404C0F1103A
:10EBC000FBCF80E077C084918F010F5F1F4F8823B8
:10EBD00021F00E947D48F801F6CFEBEFFEE2849130
:10EBE0008F010F5F1F4F882321F00E947D48F8019D
:10EBF000F6CFCC2361F0E9EFFEE284918F010F5F45
:10EC00001F4F882321F00E947D48F801F6CFDD23B5
:10EC100061F0E7EFFEE284918F010F5F1F4F8823C1
:10EC200021F00E947D48F801F6CFF11003C0EDEE0F
:10EC3000FEE20CC0E5EFFEE284918F010F5F1F4FF3
:10EC40008823A9F30E947D48F801F6CF84918F01B3
:10EC50000F5F1F4F882321F00E947D48F801F6CFF7
:10EC6000FF2019F04DEC53E002C042E054E0DD23F8
:10EC700019F02FEC33E002C022E034E0CC2319F08D
:10EC800081ED93E002C082E094E05F934F933F9365
:10EC90002F939F938F938BED9EE29F938F931F9261
:10ECA0005DDF8DB79EB709960FB6F8949EBF0FBE75
:10ECB0008DBF81E0DF91CF911F910F91FF9008955B
:10ECC00080913C128150823010F080E008951092C3
:10ECD0003C120E94454F60934512709346128093F8
:10ECE00047129093481281E008950F931F938091EB
:10ECF0003C12813019F40E94454F08C060914512C2
:10ED000070914612809147129091481200914112E1
:10ED1000109142122091431230914412601B710BEA
:10ED2000820B930B28EE33E040E050E00F946E1A14
:10ED300080913D1290913E12A0913F12B0914012ED
:10ED4000280F391F4A1F5B1FCA01B9011F910F917C
:10ED5000089580913C12813099F1823051F4C5DFE1
:10ED600060933D1270933E1280933F129093401235
:10ED700018C0109241121092421210924312109237
:10ED8000441210924512109246121092471210929D
:10ED9000481210923D1210923E1210923F121092A1
:10EDA000401281E080933C120E94454F60934112D3
:10EDB00070934212809343129093441281E008951D
:10EDC00080E00895CF92DF92EF92FF92C090E50E1F
:10EDD000D090E60EE090E70EF090E80E20918A07C2
:10EDE00030918B0740918C0750918D07C701B60178
:10EDF0000F94FE160F94FD1C609318127093191255
:10EE000080931A1290931B12C701B6010F94101C25
:10EE10002FB7F8946093660E7093670E8093680E18
:10EE20009093690E2FBF109208121092091210923F
:10EE30000A1210920B12FF90EF90DF90CF9008957E
:10EE400080913C12813079F482E080933C120E94E0
:10EE5000454F6093451270934612809347129093EA
:10EE6000481281E0089580E00895E82FF0E0E0582E
:10EE7000F64B849190E0FC013797EC30F105F8F403
:10EE8000EC57FF4F0D94BB1D8091B100887F8460CB
:10EE90008093B100089580919100887F8460809371
:10EEA000910008958091A100887F84608093A100E3
:10EEB000089580912101887F8460809321010895C5
:10EEC0008F929F92AF92BF92CF92DF92EF92FF927A
:10EED0000F931F93CF93DF931F921F92CDB7DEB78F
:10EEE0007C0149018091CE10811147C08B015B01EB
:10EEF000A40EB51E0A151B0509F43FC0F701C0801A
:10EF0000D180F80161918F016983C6016A830F94F2
:10EF10004F196A81681729F1C6010F945719C60164
:10EF20000F944F1999818917E1F0EEECFBE484917D
:10EF30008F010F5F1F4F882321F00E947D48F80149
:10EF4000F6CFE1ECFEE284918F010F5F1F4F882323
:10EF500021F00E947D48F801F6CF81E08093CE1029
:10EF60000CC0BE016F5F7F4FC40187DBF70180815A
:10EF70009181019691838083BDCF0F900F90DF9197
:10EF8000CF911F910F91FF90EF90DF90CF90BF90A6
:10EF9000AF909F908F900895AF92BF92CF92DF92E3
:10EFA000EF92FF920F931F93CF93DF931F92CDB7F2
:10EFB000DEB78C016B017A0159018091CE1081116D
:10EFC0001BC0F801808191810F944F198983F6014C
:10EFD00081936F01BE016F5F7F4FC5014EDBF8016A
:10EFE000408151814F5F5F4F51834083F1E0EF1AC1
:10EFF000F108E114F10429F70F90DF91CF911F91EF
:10F000000F91FF90EF90DF90CF90BF90AF90089559
:10F01000CF92DF92EF92FF920F931F93CF93DF93E4
:10F020007C018B016A01E9010E9416C183E0809393
:10F03000B002F0929810E0929710109396100093FF
:10F0400095101092911010929210109293101092AD
:10F050009410A601662757FD6095762F40938D107A
:10F0600050938E1060938F1070939010F8018081F0
:10F070009181AA2797FDA095BA2F8093851190932F
:10F080008611A0938711B093881186EB92E9909333
:10F090004E0280934D02D0932E07C0932D071092FD
:10F0A0002C07DF91CF911F910F91FF90EF90DF9090
:10F0B000CF900895CF92DF92EF92FF920F931F931C
:10F0C000CF93DF9300D01F92CDB7DEB77C018B01C9
:10F0D000CA01B90129837A838B839C830E9416C15C
:10F0E00023E02093B002F0929810E09297101093D2
:10F0F0009610009395102AE037ED43E25CE36981B6
:10F100007A818B819C810F94FE160F94101C609362
:10F1100091107093921080939310909394100F9489
:10F120009F166B017C019B01AC0160E070E887E7F2
:10F1300094E40F94CB1A0F94101C60938D1070936D
:10F140008E1080938F10909390102AE037ED43E259
:10F150005CE3F80160817181828193810F94FE16D6
:10F16000A70196010F94CB1A0F94151C609385117B
:10F170007093861180938711909388118CEF9FE88C
:10F1800090934E0280934D020F900F900F900F902E
:10F19000DF91CF911F910F91FF90EF90DF90CF9073
:10F1A00008950F931F93CF93DF938C01EB010E947F
:10F1B00016C183E08093B0021093981000939710CB
:10F1C000D0939610C093951084EF91E0A0E0B0E04A
:10F1D0008093911090939210A0939310B0939410F9
:10F1E00088EE9FE3AFE0B0E080938D1090938E1097
:10F1F000A0938F10B093901020E030E048EC52E4E0
:10F20000688179818A819B810F94FE1620E030E02D
:10F210004AEF53E40F94CB1A0F94151C6093851199
:10F220007093861180938711909388118FEA90E9EB
:10F2300090934E0280934D028BEF99EE90932E07A0
:10F2400080932D0710922C07DF91CF911F910F9182
:10F250000895CF92DF92EF92FF920F931F93CF9377
:10F26000DF9300D01F92CDB7DEB77C018B012983DD
:10F270003A834B835C830E9416C183E08093B00283
:10F28000F0929810E09297101093961000939510BA
:10F2900029813A814B815C81CA01B9010F949D1685
:10F2A0002AE037ED43E25CE30F94FE160F94101C46
:10F2B0006093911070939210809393109093941098
:10F2C0000F949F166B017C019B01AC0160E070E81C
:10F2D00087E794E40F94CB1A0F94101C60938D1061
:10F2E00070938E1080938F1090939010F80160812E
:10F2F0007181828193810F949D162AE037ED43E25C
:10F300005CE30F94FE16A70196010F94CB1A0F949D
:10F31000151C6093851170938611809387119093CB
:10F3200088118EE39FE890934E0280934D0289ED01
:10F330009CEB90932E0780932D0710922C070F9033
:10F340000F900F900F90DF91CF911F910F91FF9031
:10F35000EF90DF90CF9008958F929F92AF92BF92DF
:10F36000CF92DF92EF92FF92CF9320E030E04AE716
:10F3700054E4FC0160817181828193810F94FE16B7
:10F380000F94101C6B017C016115710581059105BD
:10F3900061F097FF0AC0F094E094D094C094C11C2F
:10F3A000D11CE11CF11C8DE201C080E28093CC06EF
:10F3B000C701B60128EE33E040E050E00F94901A08
:10F3C000EAE08E2E912CA12CB12CCA01B901A50125
:10F3D00094010F94901A605D6093CD068EE2809345
:10F3E000CE06C701B60124E630E040E050E00F94BD
:10F3F000901ACA01B901A50194010F94901A605D99
:10F400006093CF06C701B601A50194010F94901A2D
:10F41000C62FCA01B901A50194010F94901A605D2D
:10F420006093D006C05DC093D1068CEC96E0CF917E
:10F43000FF90EF90DF90CF90BF90AF909F908F9014
:10F4400008950F931F93CF93DF931F921F92CDB711
:10F45000DEB7FC0184918F010F5F1F4F811102C045
:10F460008B0108C069837A830E947D48F801698115
:10F470007A81F0CFD8018D918D01882319F00E94F7
:10F480007D48F8CF0F900F90DF91CF911F910F9192
:10F4900008950F931F93CF93DF938C01EEECFBE461
:10F4A0008491EF012196882321F00E947D48FE017E
:10F4B000F7CFB80184EB9EE2C4DF82E20E947D4870
:10F4C0008AE00E947D4881E0DF91CF911F910F91EA
:10F4D00008958F929F92AF92BF92CF92DF92EF9258
:10F4E000FF92CF93FC01C080D180E280F38020E0C6
:10F4F00030E0A901C701B6010F94991687FF08C033
:10F50000C701B601905820E030E048EC52E406C054
:10F5100020E030E048EC52E4C701B6010F94FE163B
:10F520000F94101C6B017C01603AF6E87F07F1E054
:10F530008F07910584F020EA36E841E050E00F940F
:10F54000901ACA01B9012AE030E040E050E00F947F
:10F55000901A605D01C060E26093CB0680E1C8163E
:10F5600087E2D806E104F10494F0C701B60120E176
:10F5700037E240E050E00F94901ACA01B9012AE046
:10F5800030E040E050E00F94901A605D01C060E20E
:10F590006093CC06E8EECE16E3E0DE06E104F1046B
:10F5A00094F0C701B60128EE33E040E050E00F943C
:10F5B000901ACA01B9012AE030E040E050E00F940F
:10F5C000901A605D01C060E26093CD06C701B6018C
:10F5D00024E630E040E050E00F94901AFAE08F2EDD
:10F5E000912CA12CB12CCA01B901A50194010F9451
:10F5F000901A605D6093CE068EE28093CF06C701BD
:10F60000B601A50194010F94901AC62FCA01B90141
:10F61000A50194010F94901A605D6093D006C05DBF
:10F62000C093D1068BEC96E0CF91FF90EF90DF90E6
:10F63000CF90BF90AF909F908F9008958F929F92A0
:10F64000AF92BF92CF92DF92EF92FF92CF9320E0E2
:10F6500030E048EC52E4FC01608171818281938149
:10F660000F94FE160F94101C6B017C0197FF0AC0CB
:10F67000F094E094D094C094C11CD11CE11CF11C06
:10F680008DE201C08BE28093CB06C701B60120E179
:10F6900037E240E050E00F94901AAAE08A2E912CB5
:10F6A000A12CB12CCA01B901A50194010F94901AA3
:10F6B000605D6093CC06C701B60128EE33E040E000
:10F6C00050E00F94901ACA01B901A50194010F945A
:10F6D000901A605D6093CD06C701B60124E630E064
:10F6E00040E050E00F94901ACA01B901A5019401BD
:10F6F0000F94901A605D6093CE068EE28093CF06E1
:10F70000C701B601A50194010F94901AC62FCA0132
:10F71000B901A50194010F94901A605D6093D00621
:10F72000C05DC093D1068BEC96E0CF91FF90EF9037
:10F73000DF90CF90BF90AF909F908F9008958F9261
:10F740009F92AF92BF92CF92DF92EF92FF92FC0115
:10F75000C080D180E280F38020E030E0A901C701C1
:10F76000B6010F94991687FF04C0C701B6019058DF
:10F7700002C0C701B6010F94101C6B017C016031FF
:10F78000F7E27F078105910584F020E137E240E050
:10F7900050E00F94901ACA01B9012AE030E040E02D
:10F7A00050E00F94901A605D01C060E26093CD0656
:10F7B00088EEC81683E0D806E104F10494F0C7018E
:10F7C000B60128EE33E040E050E00F94901ACA01F1
:10F7D000B9012AE030E040E050E00F94901A605DFB
:10F7E00001C060E26093CE06E4E6CE16D104E104E7
:10F7F000F10494F0C701B60124E630E040E050E0A7
:10F800000F94901ACA01B9012AE030E040E050E0BC
:10F810000F94901A605D01C060E26093CF06FAE039
:10F82000CF16D104E104F1049CF0BAE08B2E912CA8
:10F83000A12CB12CC701B601A50194010F94901A17
:10F84000CA01B901A50194010F94901A605D01C02D
:10F8500060E26093D006C701B6012AE030E040E0E4
:10F8600050E00F94901A605D6093D1068DEC96E0A5
:10F87000FF90EF90DF90CF90BF90AF909F908F90D0
:10F88000089520E030E040E251E4FC0160817181A4
:10F89000828193810F94FE160F94101C9B0177FFB9
:10F8A00006C022273327261B370B8DE201C08BE2CF
:10F8B0008093CC06C90168EE73E00F94A81DCB01BC
:10F8C000EAE0F0E0BF010F94A81D805D8093CD06B3
:10F8D000C90164E670E00F94A81DCB01BF010F942D
:10F8E000A81D805D8093CE06C901BF010F94A81D9D
:10F8F000282FCB01BF010F94A81D805D8093CF06F8
:10F900008EE28093D006205D2093D1068CEC96E0A9
:10F910000895492F441F4427441F29F022273327E5
:10F92000281B390B01C09C01883E9340ACF0C901F3
:10F9300068EE73E00F94A81DCB01EAE0F0E0BF0190
:10F940000F94A81D805D8093CE06C90164E670E027
:10F950000F94A81DCB0112C024363105B4F0442306
:10F9600011F08DE201C080E28093CE06C90164E609
:10F9700070E00F94A81DCB01EAE0F0E0BF010F9406
:10F98000A81D805D8093CF0611C080E28093CE06D3
:10F990008093CF062A3031059CF0442311F08DE28C
:10F9A00001C080E28093CF06EAE0F0E0C901BF0128
:10F9B0000F94A81DCB01BF010F94A81D805D05C049
:10F9C000442311F08DE201C080E28093D006C9018A
:10F9D0006AE070E00F94A81D805D8093D1068EECE4
:10F9E00096E008959C0197FD0EC08436910584F041
:10F9F00064E670E00F94A81DCB016AE070E00F94FC
:10FA0000A81D805D06C03195219531098DE201C0A8
:10FA100080E28093CF062A30310564F0EAE0F0E01E
:10FA2000C901BF010F94A81DCB01BF010F94A81DF0
:10FA3000805D01C080E28093D006C9016AE070E079
:10FA40000F94A81D805D8093D1068FEC96E00895F9
:10FA5000CF92DF92EF92FF920F931F93CF93DF939A
:10FA6000E0918D0EF0918E0E82819381A481B581FB
:10FA7000181619061A061B06E4F580918C0E909153
:10FA800005074091040780FF15C083B182958695D4
:10FA90008695837051E08527282F21709E7F292B22
:10FAA00020930507942F9170922319F180910A0FEA
:10FAB00081601AC086B1292F30E0992787FD909583
:10FAC00080959095990F880B982F822793278071A6
:10FAD00099278227932780930507942F9071982365
:10FAE00041F080910A0F806180930A0F80E00E94AC
:10FAF000BFC7E0918D0EF0918E0E86819781A08513
:10FB0000B185181619061A061B060CF049C090910B
:10FB10008C0E809105073091040791FF1FC023B11F
:10FB200090E022952695277041E0242720FBCC24E5
:10FB3000C0F8D12CD194C194D108C826D92622E08E
:10FB4000C222DD24C826D926C0920507832F8270E1
:10FB50008C2131F180910A0F82601DC020B190E0AC
:10FB60002695269541E0242720FBEE24E0F8F12C91
:10FB7000F194E194F108E826F92620E2E222FF243C
:10FB8000E826F926E0920507832F80728E2141F046
:10FB900080910A0F806280930A0F81E00E94BFC7A4
:10FBA000E0918D0EF0918E0E82859385A485B585AA
:10FBB000181619061A061B060CF049C090918C0EF7
:10FBC0008091050792FF22C09091CC0E992309F4F1
:10FBD0003EC023B190E022952F7031E02327022F01
:10FBE000017010E01195019511090827192704707B
:10FBF00011270827192700930507809104078470AF
:10FC0000802329F180910A0F84601CC020B190E00C
:10FC1000269531E023272170C22F20E0D22FD195E5
:10FC2000C195D109C827D927C074DD27C827D9278E
:10FC3000C09305078091040780748C2341F0809164
:10FC40000A0F806480930A0F82E00E94BFC78091F0
:10FC5000050780930407DF91CF911F910F91FF90CB
:10FC6000EF90DF90CF9008954F925F926F927F92C6
:10FC70008F929F92AF92BF92CF92DF92EF92FF92BC
:10FC80000F931F93CF93DF9300D01F92CDB7DEB7B2
:10FC90008C01DC014D905D906D907C9013971496D3
:10FCA0008D909D90AD90BC90179718968D919D91D9
:10FCB0000D90BC91A02D89839A83AB83BC83A30153
:10FCC0009201C301B2010F94FE166B017C01A501E4
:10FCD0009401C501B4010F94FE169B01AC01C7014C
:10FCE000B6010F94CC1A6B017C0129813A814B81BA
:10FCF0005C81CA01B9010F94FE169B01AC01C701DA
:10FD0000B6010F94CC1A0F94371D9B01AC0160E033
:10FD100070E080E89FE30F94A81B6B017C019B01BE
:10FD2000AC01C301B2010F94FE16F8016083718328
:10FD300082839383A7019601C501B4010F94FE1637
:10FD4000D80114966D937D938D939C931797A7017B
:10FD5000960169817A818B819C810F94FE16F8014E
:10FD600060877187828793870F900F900F900F9015
:10FD7000DF91CF911F910F91FF90EF90DF90CF9087
:10FD8000BF90AF909F908F907F906F905F904F90BB
:10FD900008952F923F924F925F926F927F928F922F
:10FDA0009F92AF92BF92CF92DF92EF92FF920F930A
:10FDB0001F93CF93DF93CDB7DEB7C857D1090FB6E6
:10FDC000F894DEBF0FBECDBF5B014A013901EBAA3B
:10FDD000FFAE21960FAF219722961FAF2297CFA695
:10FDE00020917E0730917F074091800750918107D5
:10FDF000DC016D917D918D919C910F94FE160F9475
:10FE0000FD1CE0966CAF7DAF8EAF9FAFE097209169
:10FE10008207309183074091840750918507F5014F
:10FE200060817181828193810F94FE160F94FD1C75
:10FE3000E4966CAF7DAF8EAF9FAFE49720918607BD
:10FE4000309187074091880750918907D4016D91BF
:10FE50007D918D919C910F94FE160F94FD1CE89658
:10FE60006CAF7DAF8EAF9FAFE89720918A0730913E
:10FE70008B0740918C0750918D07F3016081718150
:10FE8000828193810F94FE160F94FD1C69966CAFCE
:10FE90007DAF8EAF9FAF699780910C1290910D123C
:10FEA000A0910E12B0910F12E096CCACDDACEEAC8E
:10FEB000FFACE097C81AD90AEA0AFB0A809110122F
:10FEC00090911112A0911212B0911312E4968CAC81
:10FED0009DACAEACBFACE497881A990AAA0ABB0ADB
:10FEE0008091141290911512A0911612B0911712D0
:10FEF000E8962CAD3DAD4EAD5FADE897281B390BB4
:10FF00004A0B5B0B2BAF3CAF4DAF5EAF8091BE0693
:10FF100083FF0EC069964CAD5DAD6EAD7FAD699748
:10FF2000409318125093191260931A1270931B1277
:10FF30008091181290911912A0911A12B0911B126F
:10FF400069964CAC5DAC6EAC7FAC6997481A590AA7
:10FF50006A0A7B0A09F495C080917706811141C035
:10FF60006091120270911302882777FD8095982F77
:10FF70000F949F169B01AC016091900670919106C1
:10FF800080919206909193060F94991687FF29C04D
:10FF900069966CAD7DAD8EAD9FAD6997609318127B
:10FFA0007093191280931A1290931B12EEECFBE4DB
:10FFB00084918F010F5F1F4F882321F00E947D489D
:10FFC000F801F6CFE0E2FFE284918F010F5F1F4F4F
:10FFD000882321F00E947D48F801F6CF412C512C56
:10FFE00032014BA65CA66DA67EA677FE0BC08827C5
:10FFF0009927DC0184199509A609B7098BA79CA745
:020000021000EC
:10000000ADA7BEA760918A0770918B0780918C077E
:1000100090918D070F94101C9B01AC01A8ECB0E0EF
:100020000F94AC1A2BA53CA54DA55EA562177307CE
:10003000840795074CF569964CAD5DAD6EAD7FAD0F
:100040006997409318125093191260931A12709383
:100050001B12EEECFBE484918F010F5F1F4F88238E
:1000600021F00E947D48F801F6CFE1E0FFE28491A3
:100070008F010F5F1F4F882321F00E947D48F801F8
:10008000F6CF412C512C3201D701C6018827B7FD8C
:1000900083959927AA27BB278BA7B7FE03C0582FA4
:1000A00052605BA76BAD7CAD8DAD9EAD97FF03C07D
:1000B0007BA574607BA777FE03C08BA588608BA7A8
:1000C0009FA5092F10E0C301B2010F949F16F801FC
:1000D000EE0FFF1FEE0FFF1FE15FF84F2081318110
:1000E000428153810F94FE162B013C01F801EE0F63
:1000F000FF1FE455FD4F60817181882777FD809552
:10010000982F0F949F169B01AC01C301B2010F946D
:10011000FE162AE037ED43E25CE30F94FE162B0156
:100120003C0120E030E0A9010F94F21C18164CF4B9
:1001300020E030E040E05FE3C301B2010F94CC1A4D
:1001400008C0A301920160E070E080E09FE30F949B
:10015000CB1A0F94101C6FAB78AF89AF9AAFA091F8
:100160001C12AF5FAF706596AFAF659780911D129F
:100170006596BFAD65978B1304C080E00F94C104F2
:10018000F5CF80911C12EDE48E9F10011124910196
:100190002657364F1901D9011C92EBA59296EC9384
:1001A00097018601F7FE07C00027112798010C1957
:1001B0001D092E093F09D10112960D931D932D9310
:1001C0003C9315978BA69CA6ADA6BEA6B7FE0BC00A
:1001D00044275527BA01481959096A097B094BA7D1
:1001E0005CA76DA77EA76BA57CA58DA59EA5D1015B
:1001F00016966D937D938D939C9319974BAD5CAD43
:100200006DAD7EAD77FF07C07095609550954195B7
:100210005F4F6F4F7F4FF101428753876487758728
:100220008FA998ADA9ADBAAD86879787A08BB18B02
:100230008BA59CA5ADA5BEA580179107A207B30706
:1002400014F4D901C80184179507A607B70714F459
:10025000DB01CA014FA958AD69AD7AAD48175907FE
:100260006A077B0714F0DB01CA01F101828B938BD3
:10027000A48BB58B0697A105B10510F40C94E98AFF
:1002800080915E1190915F11E95BFF4F91838083B4
:10029000EFA5D1011196EC93012B022B032B09F052
:1002A0001798F10186819781A085B185892B8A2BCA
:1002B0008B2B09F01698F10182859385A485B5856D
:1002C000892B8A2B8B2B09F015982FA938AD49ADB6
:1002D0005AAD232B242B252BD9F080910E07882390
:1002E00019F0815080930E073FA5311104C0149876
:1002F00080E280930E07B0916907BBA7E0916A077F
:10030000EFA700916B0710916C072B2F3E2F0CC0AD
:10031000309165073BA7409166074FA7009167079B
:1003200010916807232F342FA8016BA97FAD219668
:100330008FAD219722969FAD22970F94991687FD36
:1003400002C00C94DD8AC701B6010F949F1620915C
:10035000EE0E3091EF0E4091F00E5091F10E0F9491
:10036000FE166BAB7CAB8DAB9EAB698B7A8B8B8BAC
:100370009C8BC501B4010F949F162091F20E309111
:10038000F30E4091F40E5091F50E0F94FE164B01B2
:100390005C016D8B7E8B8F8B988F6BAD7CAD8DAD43
:1003A0009EAD0F949F162091F60E3091F70E40915E
:1003B000F80E5091F90E0F94FE166B017C01698FB7
:1003C0007A8F8B8F9C8F2091FA0E3091FB0E40918B
:1003D000FC0E5091FD0EC301B2010F94FE166D8FFD
:1003E0007E8F8F8F98A3D10112964D905D906D9066
:1003F0007C901597B6E04B165104610471040CF51E
:10040000F1014680578060847184F6E04F165104F4
:1004100061047104B4F4D1011A964D905D906D9011
:100420007C901D97B6E04B165104610471044CF4A6
:10043000DC01CB01BF77F10187A790ABA1ABB2ABD9
:100440002DC02BA93CA94DA95EA9CA01B9010F94E1
:10045000FE162B013C01A5019401C501B4010F94C6
:10046000FE169B01AC01C301B2010F94CC1A4B01E3
:100470005C01A7019601C701B6010F94FE169B010E
:10048000AC01C501B4010F94CC1A0F94371DD101F2
:100490009F966D937D938D939C93D297F10127A5A1
:1004A00030A941A952A960E070E080E89FE30F9471
:1004B000A81B27966CAF7DAF8EAF9FAF27979B0190
:1004C000AC016BA57FA5C8010F94FE162B013C0162
:1004D0000E94AE4D2C968FAF2C97A301920160E045
:1004E00074E284E799E40F94A81B0F94FD1C6B0140
:1004F0007C012C968FAD2C978250863008F044C03A
:100500008091DB109091DC10A091DD10B091DE1095
:10051000C816D906EA06FB06B8F5BC01CD016C1970
:100520007D098E099F09660F771F881F991F2C96DA
:10053000FFAD2C970F2F10E020E030E0A9019801CB
:100540000F946E1ACA01B9010F949D160F94FD1CE9
:100550006C0D7D1D8E1D9F1D0F949D169B01AC0182
:1005600060E074E284E799E40F94A81B2B013C013E
:100570009B01AC0160E074E284E799E40F94A81B4E
:100580000F94FD1C6B017C012FB7F89480918609B4
:1005900090918709A0918809B09189098C0D9D1DC2
:1005A000AE1DBF1D8093860990938709A09388098B
:1005B000B09389092FBFD1019F962D913D914D9107
:1005C0005C91D2976F962CAF3DAF4EAF5FAF6F97F8
:1005D000A30192016F966CAD7DAD8EAD9FAD6F970F
:1005E0000F94FE162B966CAF7DAF8EAF9FAF2B97FF
:1005F000F10163A374A385A396A322893389448957
:1006000055892BA73CA74DA75EA7CA01B9010F9436
:100610009D166BAF7CAF8DAF9EAFA30192010F947F
:10062000FE160F94921B0F94151C6B017C01F101B7
:1006300067AB70AF81AF92AF9E012F5E3F4F2396A5
:100640003FAF2EAF23974DE657E064965FAF4EAFB6
:100650006497BE016F5D7F4F7AA769A7CE010196AF
:1006600062969FAF8EAF62971FA61BAA90E89FAFBE
:10067000AFE32196AFAF21972396EEADFFAD239761
:1006800061917191819191912396FFAFEEAF239784
:10069000A30192010F94FE166296AEADBFAD6297B4
:1006A0006D937D938D939D936296BFAFAEAF62972E
:1006B0009B01AC015F7760962CAF3DAF4EAF5FAF53
:1006C00060976496AEADBFAD64978D909D90AD90F0
:1006D000BD906496BFAFAEAF6497A50194016096DC
:1006E0006CAD7DAD8EAD9FAD60970F94F21C18166A
:1006F00014F560962CAD3DAD4EAD5FAD6097C50174
:10070000B4010F94A81B162F072FB82EA92E262F41
:10071000372F482F592F6FA57BA98FAD21969FADFD
:1007200021970F94F21C181634F41FA70BABBFAE21
:100730002196AFAE21972396EEADFFAD239729A565
:100740003AA5E217F30709F097CF20E030E040E840
:100750005FE36FA57BA98FAD21969FAD21970F9485
:10076000991687FF45C05E0131E1A30EB11C8E01D1
:100770000F5F1F4F2FA53BA94FAD21965FAD21976E
:10078000D8016D917D918D919C910F94FE16F80189
:1007900061937193819391938F01EA15FB0551F752
:1007A0002FA53BA94FAD21965FAD21972B966CAD40
:1007B0007DAD8EAD9FAD2B970F94FE16D101939614
:1007C0006D937D938D939C939697C701B6010F947B
:1007D0009D162FA53BA94FAD21965FAD21970F9494
:1007E000FE160F94151CF10167AB70AF81AF92AF8D
:1007F00027962CAD3DAD4EAD5FAD27976BAD7CAD73
:100800008DAD9EAD0F94FE166BAB7CAB8DAB9EABEE
:10081000D10112968D909D90AD90BC901597169633
:100820004D905D906D907C9019971A962D913D9109
:100830004D915C911D972FA738AB49AB5AAB8114F2
:100840009104A104B104B1F4411451046104710490
:1008500089F4232B242B252B69F4209179113091D5
:100860007A1140917B1150917C110F94FE160F94D8
:10087000921B00C22FA938AD49AD5AAD232B242BB2
:10088000252B49F060917D1170917E1180917F112F
:100890009091801108C060917511709176118091CE
:1008A0007711909178112BA93CA94DA95EA90F94BD
:1008B000FE160F94921B0F94151C6B017C01809106
:1008C0000A0790910B07A0910C07B0910D07F10159
:1008D00046855785608971894FAB58AF69AF7AAF4C
:1008E0002BA53CA54DA55EA582179307A407B507C8
:1008F00008F4CCC081149104A104B10471F12091D9
:10090000BE103091BF104091C0105091C1102C15F5
:100910003D054E055F0508F56BA57CA58DA59EA53B
:100920000F945F1A6BAF7CAF8DAF9EAFA70196019E
:10093000C501B4010F945F1A2BAD3CAD4DAD5EAD5A
:10094000261737074807590740F4CA01B901A5011E
:1009500094010F946E1A69017A01411451046104E3
:10096000710441F12091C2103091C3104091C41024
:100970005091C5102C153D054E055F05D8F46BA5AB
:100980007CA58DA59EA50F945F1A4B015C01A70164
:100990009601C301B2010F945F1A86169706A80646
:1009A000B90640F4C501B401A30192010F946E1A77
:1009B00069017A014FA558A969A97AA9452B462B47
:1009C000472B61F12091C6103091C7104091C8109B
:1009D0005091C9102C153D054E055F05F8F46BA527
:1009E0007CA58DA59EA50F945F1A4B015C01A70104
:1009F00096016FA578A989A99AA90F945F1A8616FE
:100A00009706A806B90650F4C501B4012FA538A968
:100A100049A95AA90F946E1A69017A016FA978AD94
:100A200089AD9AAD672B682B692B09F427C12091FA
:100A3000CA103091CB104091CC105091CD102C1594
:100A40003D054E055F0508F019C16BA57CA58DA578
:100A50009EA50F945F1A4B015C01A70196016FA937
:100A600078AD89AD9AAD0F945F1A86169706A806E1
:100A7000B90608F003C1C501B4012FA938AD49ADCD
:100A80005AAD0F946E1A69017A01F8C0811491046D
:100A9000A104B104D9F16091BE107091BF10809192
:100AA000C0109091C1106C157D058E059F0570F5E5
:100AB0000F949D162BAD3CAD4DAD5EAD0F94FE1663
:100AC0006BA77CA78DA79EA7C501B4010F949F16A5
:100AD0004B015C01C701B6010F949D16A50194015D
:100AE0000F94FE162BA53CA54DA55EA50F94F21CF8
:100AF000181664F4A50194016BA57CA58DA59EA58F
:100B00000F94A81B0F94151C6B017C014114510418
:100B100061047104A9F16091C2107091C3108091B9
:100B2000C4109091C5106C157D058E059F0540F58C
:100B30000F949D162BAD3CAD4DAD5EAD0F94FE16E2
:100B40004B015C01C301B2010F949F162B013C01C4
:100B5000C701B6010F949D16A30192010F94FE16D2
:100B6000A50194010F94F21C181654F4A3019201EC
:100B7000C501B4010F94A81B0F94151C6B017C01D7
:100B80008FA598A9A9A9BAA9892B8A2B8B2BB9F172
:100B90006091C6107091C7108091C8109091C910D3
:100BA0006C157D058E059F0550F50F949D162BAD98
:100BB0003CAD4DAD5EAD0F94FE164B015C016FA5D3
:100BC00078A989A99AA90F949F162B013C01C70106
:100BD000B6010F949D16A30192010F94FE16A50174
:100BE00094010F94F21C181654F4A3019201C5014C
:100BF000B4010F94A81B0F94151C6B017C012FA945
:100C000038AD49AD5AAD232B242B252BB9F160917A
:100C1000CA107091CB108091CC109091CD106C15B2
:100C20007D058E059F0550F50F949D162BAD3CADAF
:100C30004DAD5EAD0F94FE164B015C016FA978AD12
:100C400089AD9AAD0F949F162B013C01C701B601E7
:100C50000F949D16A30192010F94FE16A501940115
:100C60000F94F21C181654F4A3019201C501B401AB
:100C70000F94A81B0F94151C6B017C01F101ED5B17
:100C8000FF4FC082D182E282F382C701B6010F9486
:100C90009D166B017C012BA93CA94DA95EA90F945F
:100CA000A81BA3966CAF7DAF8EAF9FAFA397D1016A
:100CB000D3966D937D938D939C93D69720E030E0EF
:100CC00040E85BE4C701B6010F94FE1620E034E271
:100CD00044EF59E40F94A81B0F94101CF101668F88
:100CE000778F80A391A3F3A1FBAFD1019496BC9120
:100CF000BFA7F101F5A1FBABD1019696BC91BFAFA7
:100D00002E01E1E14E0E511C29E930E13CA72BA751
:100D1000AE014F5F5F4F3A015BAD21965FAF219708
:100D20006FA522966FAF22972496FFAF249728963F
:100D3000BFAF289710E0D3018D909D90AD90BD90EE
:100D40003D01E894B7F8EBA5FCA5C190D190E190E6
:100D5000F190FCA7EBA7A7019601C501B4010F9480
:100D6000F21C18160CF042C0112399F12BAD3FA5CF
:100D70004BA95FADC701B6010F94FE166B017C0154
:100D800021962FAD219722963FAD229724964FAD05
:100D9000249728965FAD2897C501B4010F94FE16DD
:100DA000A70196010F94F21C1816FCF4A5019401FA
:100DB000C701B6010F94A81B21966FAF2197229609
:100DC0007FAF229724968FAF249728969FAF2897BE
:100DD0000CC02196CFAE21972296DFAE22972496A3
:100DE000EFAE24972896FFAE289711E0641475049F
:100DF00009F0A1CF2C96FFAD2C97F23008F485C1F5
:100E00002091F8112BA73091F9113FAB0091FA1105
:100E10001091FB1127E137EB41ED58E36BA57FA95A
:100E2000C8010F94F21C18160CF06FC141E0A49693
:100E30004FAFA4972BAD3FA54BA95FAD6BA57FA985
:100E4000C8010F94F21C18169CF0A4961FAEA4972C
:100E50002BAD3FA54BA95FAD6BA57FA9C8010F9432
:100E6000A81BAC966CAF7DAF8EAF9FAFAC9715C093
:100E70002BA53FA9A8016BAD7FA58BA99FAD0F94B2
:100E8000A81BAC966CAF7DAF8EAF9FAFAC975BAD40
:100E90005BA76FA56FAB0BA91FAD8CEF91E16B96B4
:100EA0009FAF8EAF6B97A9E9B0E1A696BFAFAEAF8B
:100EB000A697FE013196A896FFAFEEAFA897412CFA
:100EC000512C40E8642E4FE3742E63961FAE639757
:100ED0006B96AEADBFAD6B97CD90DD90ED90FD9074
:100EE0006B96BFAFAEAF6B97A896EEADFFADA89770
:100EF00081909190A190B190A896FFAFEEAFA89786
:100F0000A496FFADA497FF2361F0AC962CAD3DAD48
:100F10004EAD5FADAC97C701B6010F94FE166B01E5
:100F20007C0163962FAD6397222381F0A301920188
:100F3000C701B6010F94FE166B017C01A30192015B
:100F4000C501B4010F94FE164B015C01A50194018B
:100F5000C701B6010F94F21C20E030E0A901181679
:100F6000CCF4C501B4010F94F21C18164CF020E02B
:100F700030E0A901C701B6010F94991687FF05C09B
:100F8000A5019401C701B60118C0B7FAB094B7F82B
:100F9000B09424C0C501B4010F94991687FD09C00F
:100FA00020E030E0A901C701B6010F94F21C181629
:100FB0008CF4A7019601C501B4010F94CB1A2C96AD
:100FC0006FAF2C972D967FAF2D9761968FAF61975E
:100FD000B92E20C0F7FAF094F7F8F094A501940127
:100FE000C701B6010F94F21C18165CF42C96CFAE14
:100FF0002C972D96DFAE2D976196EFAE6197BF2CA3
:1010000009C02C968FAE2C972D969FAE2D9761968A
:10101000AFAE6197A696AEADBFADA697CD90DD9071
:10102000ED90FD90A696BFAFAEAFA697A701960133
:101030002C966FAD2C972D967FAD2D9761968FAD29
:1010400061979B2D0F94F21C1816ECF42C962FAD83
:101050002C972D963FAD2D9761964FAD61975B2DE7
:10106000C701B6010F94A81B9B01AC01C301B201DB
:101070000F94FE162B013C016396BFAD6397BF5FD3
:101080006396BFAF63976B96EEADFFAD6B97EC5079
:10109000F24109F01DCF63963FAD6397332351F0C2
:1010A000A30192016BA57FA9C8010F94FE166BA73F
:1010B0007FAB8C0124EA30E74DE75FE36BA57FA9A6
:1010C000C8010F94FE166B017C019B01AC0160917D
:1010D00006077091070780910807909109070F9400
:1010E000F21C181624F5A701960121966FAD2197E1
:1010F00022967FAD229724968FAD249728969FAD98
:1011000028970F94F21C181694F4D1018C918460E6
:101110008C932196BFAD2197BBA72296EFAD229766
:10112000EFAB24960FAD249728961FAD28978BA57B
:101130009FA9D801F10183A794A7A5A7B6A7A39655
:101140006CAD7DAD8EAD9FADA39790589B01AC016A
:101150000F94CC1A6F962CAD3DAD4EAD5FAD6F9731
:101160000F94FE169B01AC016BE077ED83E29BE3ED
:101170000F94CB1A0F94371D762E872EF82EE92E5A
:10118000262F372F482F592F6BA57FA9C8010F9401
:10119000991687FF05C09BA4AFA8B02EC12E04C02E
:1011A000972CA82CBF2CCE2C892D9A2DAB2DBC2D85
:1011B000F10187A390A7A1A7B2A7D080272D382D32
:1011C0004F2D5E2D6BAD7FA58BA99FAD0F9499160A
:1011D000181614F083E001C081E0D82AD101DC9216
:1011E00080E1FE013196ACEFB1E101900D928A955C
:1011F000E1F78BAD9FA5ABA9BFAD8093F81190939C
:10120000F911A093FA11B093FB1121968FAD21979C
:1012100022969FAD22972496AFAD24972896BFAD16
:1012200028978093060790930707A0930807B09329
:1012300009072BAD3FA54BA95FADBC01CD010F94B4
:10124000A81B6DA37EA38FA398A72BAD3FA54BA989
:101250005FAD692D7A2D8B2D9C2D0F94A81B69A352
:101260007AA38BA39CA3AE014B5D5F4FBE016F5D64
:101270007F4FC1010F94ED0C6596BFAD6597B0939C
:101280001C12E0962CAD3DAD4EAD5FADE0972093C6
:101290000C1230930D1240930E1250930F12E496DD
:1012A0004CAD5DAD6EAD7FADE497409310125093A1
:1012B00011126093121270931312E8966CAD7DAD0B
:1012C0008EAD9FADE89760931412709315128093C2
:1012D00016129093171269968CAD9DADAEADBFAD51
:1012E00069978093181290931912A0931A12B093D1
:1012F0001B120E94AE4D843048F420911D12E12C47
:10130000F12C80E090E03DE4D32EAAC090911D1214
:101310009BA7B0901C12ADEFBA0EBB2DBF70BB2EB9
:10132000C12CD12CE12CF12CFBA5BF1631F3E1141B
:10133000F10421F0F701808182FDDFCFBA94FB2D0B
:10134000FF70BF2E2DE42F9F800111240657164FEA
:10135000E114F10409F476C0C114D10409F472C097
:10136000D7019B967C909B979C968C909C979D9682
:101370009C909D979E96AC909E97272D382D492D39
:101380005A2D97966D917D918D919C919A970F947E
:101390009916882309F456C0F701608061FC46C0A5
:1013A000D60197962D903D904D905C909A97A20112
:1013B0009101672D782D892D9A2D0F949916181665
:1013C000ACF5A2019101C201B1010F94FE161B01FF
:1013D0002C01F70183A994A9A5A9B6A9BC01CD0147
:1013E00090589B01AC010F94CC1AD7019F962D9178
:1013F0003D914D915C91D2970F94FE169B01AC01EB
:10140000C201B1010F94CB1A0F94371D1B016C015F
:101410009B01AC01672D782D892D9A2D0F9499167B
:1014200087FD04C0722C832C9C2CAD2C872D982D0D
:10143000A92DBA2DF70187A390A7A1A7B2A7862D42
:1014400081608083670178016FCFD29E8001112473
:101450000657164F009749F42F5F2F70C701780188
:1014600030911C122313F1CF0EC0DC013C9131FDF1
:10147000F3CFB701E9962FAFE9970E949747E99616
:101480002FADE997E9CF009739F0FC01208121FDCC
:1014900003C0B7010E94974790901D1200E010E032
:1014A0008DE4882E892D992787FD909520911C1217
:1014B00030E08217930709F44AC0889E5001899E44
:1014C000B00C112495012657364F5901011511050D
:1014D000C1F1D8018C9180FD04C0F901808180FFA9
:1014E00030C0D8019396CD90DD90ED90FC9096970A
:1014F000A7019601F50167A170A581A592A50F949A
:10150000A81B69A37AA38BA39CA3A7019601D8016A
:1015100097966D917D918D919C919A970F94A81BB0
:101520006DA37EA38FA398A7AE014F5D5F4FBE0151
:101530006B5D7F4FC8010F94ED0CF80180818E7FA9
:1015400080839394F92DFF709F2E8501ABCF0115F9
:10155000110569F1D8019396CD90DD90ED90FC9046
:101560009697A70196016DEC7CEC8CE49DE30F94BB
:10157000A81B69A37AA38BA39CA3A7019601F801DA
:1015800067A170A581A592A50F94A81B6DA37EA34A
:101590008FA398A7AE014F5D5F4FBE016B5D7F4F7C
:1015A000C8010F94ED0CD8018C918E7F8C938091A3
:1015B0006F00826080936F000CC0FBA9FBA72FAD6A
:1015C0002FA721960FAD219722961FAD22970C943D
:1015D000A381C858DF4F0FB6F894DEBF0FBECDBF52
:1015E000DF91CF911F910F91FF90EF90DF90CF90FF
:1015F000BF90AF909F908F907F906F905F904F9033
:101600003F902F9008954F925F926F927F928F92AA
:101610009F92AF92BF92CF92DF92EF92FF920F9381
:101620001F93CF93DF93CDB7DEB72E970FB6F89405
:10163000DEBF0FBECDBF10911A021F3FE9F00E941E
:10164000454FC0901307D0901407E0901507F09015
:1016500016076C197D098E099F0997FD0DC0209111
:101660001D1280911C1230E090E001968F70992736
:101670002817390709F028C20E94FDBF80912B0767
:1016800082FF3EC080912A0781113CC091E0909377
:101690002A078091000989278093811110920009FF
:1016A00083E08093B00210922B070E94454F6C504C
:1016B0007E4F8F4F9F4F609317077093180780934B
:1016C000190790931A0788E893E19E878D8782E037
:1016D00090E09A838983BE01635F7F4FCE010196BC
:1016E0000E949E9816E0115069F08EE192E10E94EE
:1016F000D94F62E070E080E090E00E94AC4EF3CF02
:1017000010922A071091030110951170912F91707A
:10171000809129071817A9F0992309F428C20E947B
:101720000AAB80912907823029F060E088E49FE2CB
:101730000E9482C01093290783E08093B0020E9428
:10174000305D0E94454F6B017C018091250790918F
:101750002607A0912707B0912807A7019601281B0B
:10176000390B4A0B5B0B57FF05C080912407882378
:1017700009F449C2D701C6018C599F4FAF4FBF4FE3
:101780008093250790932607A0932707B0932807F7
:101790008091230718162CF480912307823074F46B
:1017A00008C080912307992781950CF490950297A2
:1017B0002CF48091811181119DC0ADC0809189115F
:1017C000882309F470C08091230718165CF4809177
:1017D0002307992787FD909597FD0196BC01759584
:1017E00067950DC080912307992787FD909597FDF8
:1017F00001969595879566277727681B790B8090CA
:10180000601190906111A0906211B09063118114E9
:101810009104A104B10429F421E030E040E050E05B
:1018200039C0882777FD8095982F0F949F162B013C
:101830003C01C701B601681979098A099B090F940F
:101840009D169B01AC01C301B2010F94A81B20E0BF
:1018500030E04AE754E40F94FE164B015C0120E0AF
:1018600030E040E253E40F94F21C87FF0FC020E009
:1018700030E046E952E4C501B4010F94F21C87FD43
:10188000CBCF2AE030E040E050E004C024E630E076
:1018900040E050E0C0926011D0926111E09262117C
:1018A000F092631104C021E030E040E050E0A091EC
:1018B0002307BB27A7FDB0950F94B61A22E030E0AE
:1018C00040E050E00F94901A80918511909186111C
:1018D000A0918711B0918811820F931FA41FB51F8B
:1018E0008093851190938611A0938711B0938811EE
:1018F00010922307D701C6018856954CAF4FBF4FB2
:1019000080931F0790932007A0932107B09322078D
:1019100081E08093B00220914D0230914E0240E56B
:10192000213A340749F480911B029FEF980F90935E
:101930001B02882309F426C12E593D4A79F480916F
:101940001C0790911B07891748F490911B022FEFF9
:10195000290F20931B02992309F424C12FB7F8946F
:101960008091860990918709A0918809B091890991
:101970002FBF4091B002411105C0209124072223BE
:1019800009F465C02AE0B695A795979587952A959D
:10199000D1F7009721E0A207B10520F08FEF9FEF6C
:1019A000A0E0B0E096958795009741F020911D0743
:1019B00030911E072817390708F049C08091240785
:1019C000811111C0423050F0443028F0443031F4DD
:1019D0001092B00203C081E08093B0020F94F70B25
:1019E00081E08093240784E00E942BD381E08093E0
:1019F000BA11E0914D02F0914E02199510928111A9
:101A000080912407882351F00E949DD291E081119A
:101A100001C090E0909324079111DCC080901D07D5
:101A200090901E07A12CB12C0E94454F6C197D0986
:101A30008E099F0986169706A806B90640F40E94EB
:101A4000454F6C197D0970931E0760931D078091A7
:101A50004D0290914E02815A904521F080919F064F
:101A6000882379F048E9C40E4AE3D41EE11CF11C36
:101A7000C0921F07D0922007E0922107F092220720
:101A80000FC080911F0790912007A0912107B0916E
:101A90002207C81AD90AEA0AFB0AF7FE0E9404C202
:101AA000809124078111AFC08091B002813049F04C
:101AB00008F4A9C0843008F0A6C081E08093B00289
:101AC000A2C01092B0029FC054E01502F001112490
:101AD000ED52FC4F20E030E040E752E4608171813C
:101AE000828193810F94A81B4B015C018091D90ED8
:101AF0009091DA0EA091DB0EB091DC0E89839A836F
:101B0000AB83BC838091DD0E9091DE0EA091DF0E41
:101B1000B091E00E8D839E83AF83B8878091E10EF4
:101B20009091E20EA091E30EB091E40E89879A871E
:101B3000AB87BC87AE01475F5F4FBE016B5F7F4FD6
:101B4000CE0101960E9431BFC12C8501740125EEA2
:101B50003EE0AE01475F5F4FBE016B5F7F4FCE013E
:101B600001960E94C97E8FEF80931A0285CD109254
:101B70004B1210924C12823009F4DCCD60E08BE302
:101B80009FE2D6CD8CE080931B0280911D0790913F
:101B90001E07019790931E0780931D0781E0809395
:101BA000B002CACE96E090931B0291E09093B002EF
:101BB0008F5F80931C07D701C6018856954CAF4FA5
:101BC000BF4F80931F0790932007A0932107B093E6
:101BD0002207C4CE80901D0790901E07A12CB12C27
:101BE0000E94454F6C197D098E099F09861697063C
:101BF000A806B90640F40E94454F6C197D09709300
:101C00001E0760931D072E960FB6F894DEBF0FBE19
